:020000040802F0
:1000000000000824A55B02083D450208434502089C
:10001000494502084F450208554502080000000006
:100020000000000000000000000000005B45020826
:10003000694502080000000077450208854502086E
:10004000F55B0208F55B0208F55B0208F55B020848
:10005000F55B0208F55B0208F55B0208F55B020838
:10006000F55B0208F55B0208F55B020891450208A2
:10007000A5450208B9450208CD450208E145020838
:10008000F545020809460208F55B02081D4602080C
:1000900031460208F55B0208F55B0208F55B0208D1
:1000A000F55B020845460208F55B0208F55B0208AD
:1000B000F55B0208F55B0208F55B0208F55B0208D8
:1000C000F55B0208F55B0208F55B0208F55B0208C8
:1000D000F55B0208594602086D460208814602088F
:1000E000F55B0208F55B020800000000F55B020802
:1000F00095460208F55B0208F55B0208F55B02080D
:10010000F55B0208F55B0208F55B0208F55B020887
:10011000A9460208BD460208F55B0208F55B020825
:10012000F55B0208F55B0208F55B0208F55B020867
:10013000F55B0208D1460208F55B0208F55B020890
:1001400000000000000000000000000000000000AF
:10015000F55B0208F55B0208F55B0208E54602085C
:10016000F55B0208F55B0208F55B0208F55B020827
:10017000F55B0208F55B0208F55B02080000000071
:10018000F55B0208F55B0208F9460208F55B020818
:10019000F55B0208F55B0208F55B0208F55B0208F7
:1001A000F55B0208F55B0208F55B0208F55B0208E7
:1001B0000D470208F55B0208F55B020821470208BB
:1001C00035470208F55B0208F55B0208F55B02089B
:1001D000F55B0208F55B0208F55B0208F55B0208B7
:1001E000F55B0208F55B0208F55B0208F55B0208A7
:1001F000F55B0208F55B0208F55B0208F55B020897
:10020000F55B0208F55B0208F55B0208F55B020886
:10021000F55B0208F55B0208F55B0208F55B020876
:10022000F55B0208F55B0208F55B020800000000C0
:10023000F55B0208F55B020800000000F55B0208B0
:10024000F55B020849470208F55B0208F55B020806
:10025000F55B0208F55B0208F55B0208F55B020836
:10026000F55B0208F55B0208F55B0208F55B020826
:10027000F55B0208F55B02085D470208000000001C
:10028000F55B0208F55B0208F55B02080000000060
:0802900000000000F55B02080C
:1002A00010B5054C237833B9044B13B10448AFF3B0
:1002B00000800123237010BDDC000024000000003A
:1002C000F01F040808B5034B1BB103490348AFF303
:1002D000008008BD00000000E0000024F01F0408BA
:1002E00010F8012B11F8013B012A28BF9A42F7D0E0
:1002F000D01A7047034613F8012B002AFBD1181AB5
:1003000001387047000000000000000000000000FD
:1003100001F0FF01102A2BDB10F0070F08D010F8B6
:10032000013B013A8B422DD010F0070F42B3F6D1BA
:10033000F0B441EA012141EA014122F007047FF0D3
:1003400000070023F0E80256083C85EA010586EA2A
:10035000010685FA47F5A3FA87F586FA47F6A5FA66
:1003600087F68EB9EED1F0BC01F0FF0102F0070272
:1003700032B110F8013B013A83EA010313B1F8D11D
:100380000020704701387047002D06BF35460338FE
:10039000073815F0010F07D1013015F4807F02BF37
:1003A000013015F4C03F0130F0BC0138704700BF88
:1003B00053B94AB9002908BF00281CBF4FF0FF31CC
:1003C0004FF0FF3000F074B9ADF1080C6DE904CEC8
:1003D00000F006F8DDF804E0DDE9022304B0704720
:1003E0002DE9F047089D04468E46002B4DD18A42E8
:1003F000944669D9B2FA82F252B101FA02F3C2F11B
:10040000200120FA01F10CFA02FC41EA030E9440AB
:100410004FEA1C48210CBEFBF8F61FFA8CF708FBCC
:1004200016E341EA034306FB07F199420AD91CEBA4
:10043000030306F1FF3080F01F81994240F21C81D6
:10044000023E63445B1AA4B2B3FBF8F008FB10331E
:1004500044EA034400FB07F7A7420AD91CEB040453
:1004600000F1FF3380F00A81A74240F20781644423
:10047000023840EA0640E41B00261DB1D4400023A8
:10048000C5E900433146BDE8F0878B4209D9002D0C
:1004900000F0EF800026C5E9000130463146BDE896
:1004A000F087B3FA83F6002E4AD18B4202D3824200
:1004B00000F2F980841A61EB030301209E46002DAF
:1004C000E0D0C5E9004EDDE702B9FFDEB2FA82F204
:1004D000002A40F09280A1EB0C014FEA1C471FFA62
:1004E0008CFE0126200CB1FBF7F307FB131140EA49
:1004F00001410EFB03F0884208D91CEB010103F116
:10050000FF3802D2884200F2CB804346091AA4B2D7
:10051000B1FBF7F007FB101144EA01440EFB00FEAB
:10052000A64508D91CEB040400F1FF3102D2A64510
:1005300000F2BB800846A4EB0E0440EA03409CE7AF
:10054000C6F12007B34022FA07FC4CEA030C20FA5C
:1005500007F401FA06F31C43F9404FEA1C4900FA7C
:1005600006F3B1FBF9F8200C1FFA8CFE09FB1811F9
:1005700040EA014108FB0EF0884202FA06F20BD96C
:100580001CEB010108F1FF3A80F08880884240F2BC
:100590008580A8F102086144091AA4B2B1FBF9F000
:1005A00009FB101144EA014100FB0EFE8E4508D9FB
:1005B0001CEB010100F1FF346CD28E456AD9023880
:1005C000614440EA0840A0FB0294A1EB0E01A14265
:1005D000C846A64656D353D05DB1B3EB080261EBD3
:1005E0000E0101FA07F722FA06F3F1401F43C5E9AD
:1005F000007100263146BDE8F087C2F12003D840E3
:100600000CFA02FC21FA03F3914001434FEA1C4724
:100610001FFA8CFEB3FBF7F007FB10360B0C43EA16
:10062000064300FB0EF69E4204FA02F408D91CEBC6
:10063000030300F1FF382FD29E422DD902386344C4
:100640009B1B89B2B3FBF7F607FB163341EA034164
:1006500006FB0EF38B4208D91CEB010106F1FF38B3
:1006600016D28B4214D9023E6144C91A46EA0046AA
:1006700038E72E46284605E70646E3E61846F8E63C
:100680004B45A9D2B9EB020864EB0C0E0138A3E785
:100690004646EAE7204694E74046D1E7D0467BE766
:1006A000023B614432E7304609E76444023842E7DE
:1006B000704700BF80B483B000AF786039607B685A
:1006C0001A6801213B6801FA03F31A437B681A6038
:1006D00000BF0C37BD465DF8047B704780B483B023
:1006E00000AF786039607B681A6801213B6801FAC5
:1006F00003F3DB431A407B681A6000BF0C37BD462A
:100700005DF8047B7047000080B500AF044B002209
:100710001A6004490A2000F0B5FD00BF80BD00BF8B
:10072000F80000242907020880B400AF044B1B68BE
:100730000133034A136000BFBD465DF8047B704778
:10074000F800002480B500AF064802F035F80648EE
:1007500002F01AF8054802F057F9054802F004F8CB
:1007600000BF80BD75070208990702082508020826
:10077000C107020880B582B000AF78600B46FB70FD
:10078000FB789BB21946786801F076FE02F046F8D5
:1007900000BF0837BD4680BD80B582B000AF78602D
:1007A0000B467B80054B1B6821337A881946786895
:1007B00020F09EF800BF0837BD4680BD7C020024B3
:1007C00080B588B004AFF860B9607A603B60134BC5
:1007D0001B78032B1ED930231A0630231B041A431F
:1007E00030231B021343302243EA020144231A063A
:1007F00046231B041A434C231B02134354221A435F
:100800003B8B02937B6801933B680093044B04206D
:1008100002F05EF800BF1037BD4680BDB49B0024D7
:100820000820040880B500AF05F0CCFB034618464D
:1008300080BD80B500AF00F005F800F04FF9034629
:10084000184680BD80B586B000AF1123BB60002381
:10085000FB6000233B614FF480537B603B1D1946D6
:1008600008480CF003FE4FF400537B603B1D194613
:1008700004480CF0FBFD00F02BF800BF1837BD4614
:1008800080BD00BF0010025880B500AF022000F00C
:1008900099FD00BF80BD000080B500AF0B4B4FF449
:1008A00000529A61094B4FF480529A61FFF7ECFFB6
:1008B000064B4FF000529A61FFF7E6FF034B4FF0F3
:1008C00080529A61FFF7E0FF00BF80BD0010025820
:1008D00080B500AF094B4FF000529A61FFF7D4FF8B
:1008E000064B4FF480529A61FFF7CEFF034B4FF453
:1008F00000529A61FFF7C8FF00BF80BD0010025888
:1009000080B584B000AF0346FB710023FB7329E080
:1009100097F90730002B04DA164B4FF400529A6116
:1009200003E0144B4FF000529A61FFF7ADFF114BFB
:100930004FF480529A61FFF7A7FF0E4B4FF08052A1
:100940009A610C4B4FF080529A61FB7B072B03D1CD
:10095000084B4FF400529A61FB795B00FB71FB7B03
:100960000133FB73FB7B072BD2D900BF00BF1037CD
:10097000BD4680BD0010025880B582B000AF002394
:10098000BB710023FB711AE0BB795B00BB71104B9C
:100990004FF480529A61FFF777FF0D4B1B6903F408
:1009A0000053002B02D0BB790133BB71084B4FF0D1
:1009B00080529A61FFF768FFFB790133FB71FB7985
:1009C000072BE1D9BB7918460837BD4680BD00BF6B
:1009D0000010025880B582B000AF114B4FF40052A6
:1009E0009A61FFF751FF0E4B4FF480529A61FFF767
:1009F0004BFF0B4B1B6903F40053002B02D0012368
:100A0000FB7101E00023FB71054B4FF080529A61AE
:100A1000FFF73AFFFB7918460837BD4680BD00BF97
:100A20000010025880B500AF0C4B4FF000529A6195
:100A3000FFF72AFF094B4FF480529A61FFF724FF1A
:100A4000064B4FF080529A61FFF71EFF034B4FF4A5
:100A500000529A61FFF718FF00BF80BD00100258D6
:100A600080B500AF094B4FF400529A61FFF70CFFBD
:100A7000064B4FF480529A61FFF706FF034B4FF08D
:100A800080529A61FFF700FF00BF80BD001002583E
:100A900080B584B000AF0346FB710F4B1B6903F4B4
:100AA0000053002B13D00C4B1B6903F48053002B15
:100AB0000DD0FFF7F1FEFB791846FFF721FFFFF796
:100AC00089FF0346FB73FFF703FFFB7B00E0012375
:100AD00018461037BD4680BD0010025880B500AFE3
:100AE000A020FFF7D5FF0346002B01D1012302E030
:100AF000FFF7EEFE0023184680BD90B585B000AF2D
:100B000078600B467B8013463B80FFF7C5FEA02034
:100B1000FFF7F6FEFFF75EFF0346002B3ED17B8812
:100B20001B0A9BB2DBB21846FFF7EAFEFFF752FF43
:100B30000346002B34D17B88DBB21846FFF7E0FE7A
:100B4000FFF748FF0346002B2CD1FFF7A5FEA1209D
:100B5000FFF7D6FEFFF73EFF0346002B24D100230C
:100B6000FB8113E0FB897A68D418FFF705FF034681
:100B70002370FA893B88013B9A4202D0FFF752FF6B
:100B800001E0FFF76DFFFB890133FB81FA893B88A8
:100B90009A42E7D3FFF79CFE012309E000BF04E07F
:100BA00000BF02E000BF00E000BFFFF791FE00239E
:100BB00018461437BD4690BDB0B58EB000AF786012
:100BC00007F108033022002118461FF0B9FE07F193
:100BD0000803302200211846FFF78FFF7B681D466F
:100BE00007F108040FCC0FC50FCC0FC594E80F0018
:100BF00085E80F0078683837BD46B0BD80B582B053
:100C000000AF0346FB8018201FF052FE03461A4631
:100C1000104B1A600F4B1B6800221A600D4B1B68AB
:100C200000225A600B4B1B680B4ADA60094B1B68A9
:100C30000A4A5A61074B1B68094A1A61054B1B682F
:100C4000FA885A8107490A2000F01CFB00BF0837C8
:100C5000BD4680BD80020024A51E02089D2002081A
:100C6000791F0208690C020880B500AF064B1B789B
:100C7000012B06D1054B1B681B69044A12681046FC
:100C8000984700BF80BD00BF000000248002002400
:100C900080B500AF0022012118480BF06BFE03461F
:100CA000002B01D003F042FB00224FF000711348EB
:100CB0000BF060FE0346002B01D003F037FB0F481A
:100CC0000BF064FC002201210D480BF053FE03469B
:100CD000002B01D003F02AFB00224FF000710848DE
:100CE0000BF048FE0346002B01D003F01FFB044825
:100CF0000BF04CFC0123184680BD00BF98AD0024CA
:100D000038AE002480B582B000AF786039607B686F
:100D10001B68084A934201D102F05EFC7B681B68A5
:100D2000054A934201D102F0BBFC00BF0837BD4623
:100D300080BD00BF00A0004000A4004080B582B08C
:100D400000AF786039607B681B68314A93422BD1D1
:100D5000304B314A402178680BF09EFC0346002B53
:100D600052D12D4B1B682D4AC2F830312B4BD3F892
:100D700030311A462A4B1A60274BDB681B0C274A76
:100D8000C2F82831254BDB69002B09D0234BDB69E6
:100D9000224AD2F83001214AD2F828211D49984729
:100DA000002000F0ADFA2FE07B681B681D4A9342DB
:100DB0002AD11D4B184A402178680BF06DFC034680
:100DC000002B21D1144B1B68184AC2F83031174B45
:100DD000D3F830311A46164B1A600F4BDB681B0CE8
:100DE000124AC2F82831114BDB69002B09D00F4B96
:100DF000DB690E4AD2F830010C4AD2F828210A49A0
:100E00009847012000F07CFA00BF0837BD4680BD3E
:100E100000A000401C050024F404002484020024E7
:100E20002C05002400A4004024050024BC03002459
:100E30003005002480B584B000AFF860B9607A60F6
:100E40003B60BB68FA680949094800F019F83B683B
:100E50007A680849084800F013F808490A2000F0A9
:100E600011FA00BF1037BD4680BD00BF98AD002409
:100E70008402002438AE0024BC030024250F02089D
:100E800080B584B000AFF860B9607A603B60FB6801
:100E9000BA681A6018201FF00BFD03461A46FB685B
:100EA0005A60FB685B6800221A60FB685B6800227E
:100EB0005A60FB685B680122DA81FB685B683A680C
:100EC00092B25A81FB685B6800229A81FB685B687A
:100ED00000221A81FB685B680D4A1A61FB685B6837
:100EE0000C4A5A61FB6802221A72FB6800221A61DE
:100EF000FB68094A9A617A68FB68DA60FB68074A0E
:100F00001A62FB68064A5A6200BF1037BD4680BDB0
:100F1000031E0208911D020825110208551002083F
:100F2000FD10020880B500AF154B5B68154A1360D1
:100F3000134B5B69002B03D0114800F027F80AE03F
:100F40000F4B5B680F4A13600E4B1B685B690D4AC1
:100F50001268104698470C4B5B69002B03D00A4877
:100F600000F014F80AE0084B5B68064A1360054B72
:100F70001B685B69034A12681046984700BF80BD32
:100F8000840200247C050024BC03002480B584B0C6
:100F900000AF78607B681B695A1C7B681A617B68AC
:100FA0001B7A1A467B681B6903FB02F27B68DB68CD
:100FB0009A424AD37B6800221A617B6801225A72E6
:100FC0007B685B69002B3DD07B685B691A687B6836
:100FD000C3F834217B6803F1A8007B685B6903F1E7
:100FE00009017B685B691B7A1A461FF081FC7B68EC
:100FF0005B695A687B68DA607B685B691B7A1A46B2
:101000007B68C3F82C217B685B6A786898477B68AB
:101010005B699B69002B0CD07B685B699B69FB60FB
:101020007B685B6918461FF04BFC7B68FA685A6165
:101030000BE07B685B6918461FF042FC7B6800226E
:101040005A6102E07B6800225A7200BF1037BD4629
:1010500080BD000080B584B000AFF860B9603B602F
:101060001346FB71FB79082B3BD8FB681B681F4AB2
:10107000934218D11E4B00225A61FB791B041C4A73
:10108000D3601B4B00229A61194B00225A60184A08
:10109000BB681360164B00229A603A6814491348E3
:1010A0000BF09FFA1EE0FB681B68124A934219D1AD
:1010B000114B00225A61FB791B040F4AD3600E4B7F
:1010C00000229A610C4B00225A600B4ABB681360E5
:1010D000094B00229A603A68074906480BF081FAEA
:1010E00000E000BF1037BD4680BD00BF98AD0024B2
:1010F0003405002438AE00245805002480B582B0A1
:1011000000AF78607B68D3F834117B68D3F82C315A
:10111000DAB27B68A8337868FFF79CFF00BF083716
:10112000BD4680BD80B588B000AFF860B9603B6057
:101130001346FB7100237B611C201FF0B9FB0346A3
:101140007B617B690933FA79396818461FF0D0FB57
:101150007B6900229A617B69BA681A607B69FA79B7
:101160001A727B69BA6A5A60FB685B69002B03D10B
:10117000FB687A695A6114E00023FB770023BB61A6
:10118000FB685B69BB6105E0FB7F0133FB77BB69F3
:101190009B69BB61BB699B69002BF5D1BB697A690F
:1011A0009A6100BF2037BD4680BD000080B584B085
:1011B00000AF03460A46FB711346BB71BB79002B97
:1011C00002D10023FB7301E00123FB73FB79013B98
:1011D000072B4CD801A252F823F000BFFD110208E2
:1011E0000B1202081912020827120208351202080F
:1011F000431202085112020861120208FB7B1A46D0
:1012000010211D480CF0E2FA31E0FB7B1A46012167
:101210001A480CF0DBFA2AE0FB7B1A460821174833
:101220000CF0D4FA23E0FB7B1A46042113480CF09F
:10123000CDFA1CE0FB7B1A46202110480CF0C6FAC0
:1012400015E0FB7B1A4610210C480CF0BFFA0EE0AB
:10125000FB7B1A464FF4005109480CF0B7FA06E040
:10126000FB7B1A46402105480CF0B0FA00BF00BFD6
:101270001037BD4680BD00BF000402580010025860
:101280000008025880B483B000AF03463960FB7198
:10129000FB791A49542203FB02F20A441278013204
:1012A000D0B2164A542101FB03F3134402461A70CC
:1012B000FB79124A542101FB03F313441B78132BCF
:1012C00001D9002314E0FA79FB790C49542000FB82
:1012D00003F30B441B78591E084813465B00134464
:1012E000DA00D21A53189B0003443A685A6001236B
:1012F00018460C37BD465DF8047B70478005002416
:1013000080B584B000AF0346FB710023FB73FB790B
:10131000144A542101FB03F313441B78002B1CD007
:101320000023FB730FE0FA79F97B0E4813465B004C
:101330001344DA00D21A53189B0003445B689847A1
:10134000FB7B0133FB73FB79064A542101FB03F35A
:1013500013441B78FA7B9A42E5D300BF1037BD4691
:1013600080BD00BF8005002480B500AF044810F0A8
:1013700003FF044810F000FF0123184680BD00BFA2
:101380007CAF0024C8AF002480B582B000AF786085
:101390007B681B68094A934202D10920FFF7B0FF1E
:1013A0007B681B68064A934204D114F0A1F90A2015
:1013B000FFF7A6FF00BF0837BD4680BD0000014013
:1013C0000004014080B489B000AF78600023BB61A5
:1013D0001C4B5B687B611C4B1B681C4AA2FB0323F4
:1013E0009A0C7B6802FB03F33B610023BB61154B46
:1013F0009B68FB61134B9B68FB60FA68FB699A4230
:10140000F8D0FA68FB699A4206D2FA69FB68D31AE7
:10141000BA691344BB6107E07A69FB68D21AFB69B9
:101420001344BA691344BB61FB68FB61BA693B6949
:101430009A4200D2DEE700BF00BF2437BD465DF808
:10144000047B704710E000E04800002483DE1B436B
:1014500080B586B002AFF860B9607A603B60FB6A25
:1014600000930223FA684549454800F073FA3B6B44
:1014700000930223BA684349434800F06BFA7B6B40
:10148000009302237A684149414800F063FABB6B3C
:10149000009302233A683F493F4800F05BFAFB6B38
:1014A00000930223BA693D493D4800F053FA3B6C72
:1014B00000930223FA6939493A4800F04BFA7B6CF1
:1014C000009302233A6A3849384800F043FAFB6C2B
:1014D00000930223BA6A3649364800F03BFA334B90
:1014E000DB6901223449184611F0C8FB2D4BDB693A
:1014F00001223249184611F0C1FB214BDB69012260
:101500002F49184611F0BAFB1F4BDB6901222D4908
:10151000184611F0B3FB1E4BDB6901222A4918461D
:1015200011F0ACFB1C4BDB6901222849184611F075
:10153000A5FB1B4BDB6901222549184611F09EFBD8
:101540001C4BDB6901222349184611F097FBBB6C49
:10155000009302237A6A2049204800F0FBF91F4BD0
:10156000DB6901221E49184611F088FB1D490A203B
:10157000FFF788FE00BF1037BD4680BD54B200247F
:101580001C09002474B300245C19002404B4002452
:101590009C290024C4B10024DC390024A4B0002418
:1015A0009C6A00241C4A0024E4B200245C5A0024F3
:1015B00034B10024DC7A00245F5A00241F4A00243E
:1015C0001F0900245F1900249F290024DF3900240B
:1015D0009F6A0024DF7A002414B000241C8B0024AE
:1015E0001F8B0024E915020880B500AF0E4800F0FB
:1015F00025FA0E4800F022FA0D4800F01FFA0D48B7
:1016000000F01CFA0C4800F019FA0C4800F016FA29
:101610000B4800F013FA0B4800F010FA0A4800F0EB
:101620000DFA00BF80BD00BF1C0900245C19002416
:101630009C290024DC3900249C6A00241C4A0024D4
:101640005C5A0024DC7A00241C8B002480B588B00E
:1016500000AFF860B9603B601346FB8000237B61FC
:101660004FF401701FF024F903467B617B6904335A
:10167000FA88B96818461FF03BF97B690022C3F865
:1016800000223B689AB27B695A807B69FA881A808B
:101690007B69BA6AC3F8FC21FB6803F580535B6B76
:1016A000002B06D1FB6803F580531A467B69536310
:1016B00019E00023FB770023BB61FB6803F580532F
:1016C0005B6BBB6106E0FB7F0133FB77BB69D3F843
:1016D0000032BB61BB69D3F80032002BF3D1BB6988
:1016E0007A69C3F8002200BF2037BD4680BD0000E4
:1016F00080B58AB004AF78607B68DB69002B24D1A9
:10170000654B1B78012B40F2C38030231A0630232F
:101710001B041A4330231B021343302243EA020105
:1017200044231A0646231B041A434C231B0213436B
:1017300054221A43594B0293BA230193584B0093F6
:10174000584B022001F0C4F8A2E07B6803F58053F7
:1017500000229A847B68DB691B68534A934200F03D
:1017600098807B68DB691B68504A934258D07B683D
:10177000DB691B684E4A934206D101224FF4806117
:101780004C480CF023F84BE07B68DB691B684A4A45
:10179000934206D101224FF4006146480CF016F83E
:1017A0003EE07B68DB691B68444A934206D1012214
:1017B0004FF4807142480CF009F831E07B68DB6936
:1017C0001B68404A934206D101224FF400713C4805
:1017D0000BF0FCFF24E07B68DB691B683A4A93420C
:1017E0000CD17B68D8697B6803F621017B6803F51F
:1017F00080535A8C642311F0ABF911E07B68DB69EC
:101800001B68324A93420BD17B68D8697B6803F628
:1018100021017B6803F580535A8C642311F098F9F9
:101820007B6803F621037A6802F58052528C7B6153
:101830003A613B69002B1DDD7B6903F01F023B69A8
:101840001344FB607B69BB60BFF34F8F00BF204A2E
:10185000BB68C2F87032BB682033BB60FB68203BBA
:10186000FB60FB68002BF2DCBFF34F8F00BFBFF3C0
:101870006F8F00BF00BF7B68D8697B6803F62101CA
:101880007B6803F580535B8C1A4611F04DFA00E03B
:1018900000BF1837BD4680BDB49B0024AC4C040883
:1018A0008820040834200408000C0058004C004034
:1018B00000100140000C0258004800400014014094
:1018C00000080258007800400044004000500040EA
:1018D00000ED00E080B582B000AF78607B681B78D7
:1018E000002B07D17B6801221A707B6803F58053B7
:1018F00000229A847B6803F580539B8C19467B6891
:10190000DA787B680B4483F821207B6803F58053E9
:101910009B8C01339AB27B6803F580539A847B6871
:10192000D8697B6803330122194611F0A7F97B6857
:101930000022DA607B6803F580539B8CB3F5806FDF
:1019400004D37B6803F5805300229A8400BF0837D4
:10195000BD4680BD80B584B000AFF860B9607A60E4
:10196000FB70FB680022DA607A68FB689A60FB68AB
:10197000BA68DA61FB6803F580531A462A4BD362D2
:10198000FB6803F580531A46284B9362FB6803F506
:1019900080531A46264B936318201EF089FF034696
:1019A0001A46FB6803F58053DA63FB6803F580533E
:1019B000DB6B00221A60FB6803F58053DB6B0022AF
:1019C0005A60FB6803F58053DB6B0022DA81FB6809
:1019D00003F58053DB6BBA6992B25A81FB6803F559
:1019E0008053DB6B00229A81FB6803F58053DB6B2D
:1019F00000221A81FB6803F58053DB6B0D4A1A61E4
:101A0000FB6803F58053DB6B0B4A5A61FB680222CB
:101A100083F82020FB6800221A61FB6864225A6167
:101A200000BF1037BD4680BDD5180208F116020868
:101A30004D160208031E0208911D020880B582B0EF
:101A400000AF78607B6803F580531B6B002B03D1DC
:101A50007B6801229A7032E07B681B78012B2ED1C3
:101A60007B68DB685A1C7B68DA607B6893F82030FF
:101A70001A467B68DB6803FB02F27B689B689A422C
:101A80001DD37B680022DA607B6800221A707B68B5
:101A900003F580539B8C002B11D07B6803F580539A
:101AA0001B6B7A6802F121007A6802F58052928CF1
:101AB000114698477B6803F5805300229A847B681F
:101AC00003F580535B6B002B03D0786800F0DCF8E3
:101AD0000AE07B6803F58053DB6B5B697A6802F58B
:101AE0008052D26B1046984700BF0837BD4680BD74
:101AF00080B582B000AF78607B681B68284A93424B
:101B000003D12848FFF7E6FE46E07B681B68264ABB
:101B1000934203D12548FFF7DDFE3DE07B681B685B
:101B2000234A934203D12348FFF7D4FE34E07B6875
:101B30001B68214A934203D12048FFF7CBFE2BE0DC
:101B40007B681B681E4A934203D11E48FFF7C2FE02
:101B500022E07B681B68124A934203D11A48FFF7C0
:101B6000B9FE19E07B681B68184A934203D11848F4
:101B7000FFF7B0FE10E07B681B68164A934203D162
:101B80001548FFF7A7FE07E07B681B68134A9342DE
:101B900002D11348FFF79EFE00BF0837BD4680BD47
:101BA000004C00401C4A0024001001401C09002485
:101BB000004800405C190024001401409C290024C6
:101BC00000780040DC3900249C6A00240044004076
:101BD0005C5A002400500040DC7A0024000C0058BD
:101BE0001C8B002480B582B000AF78607B681B68D6
:101BF0001D4A934233D07B681B681C4A934206D12E
:101C000000224FF480611A480BF0E0FD27E07B686A
:101C10001B68184A934206D100224FF40061144811
:101C20000BF0D4FD1BE07B681B68134A934206D17E
:101C300000224FF4807111480BF0C8FD0FE07B6863
:101C40001B680F4A934206D100224FF400710B48E3
:101C50000BF0BCFD03E07B681B680A4A934200BF9F
:101C60000837BD4680BD00BF004C00400010014059
:101C7000000C0258004800400014014000080258BF
:101C8000007800400044004080B584B000AF786028
:101C90007B681B695A1C7B681A617B6893F820304B
:101CA0001A467B681B6903FB02F27B685B699A42F8
:101CB0006AD37B6800221A617B6801221A767B68EE
:101CC00003F580535B6B002B5BD07B6803F6210030
:101CD0007B6803F580535B6B191D7B6803F58053AC
:101CE0005B6B1B881A461EF003FE7B6803F580536E
:101CF0005B6B5B881A467B685A617B6803F580538F
:101D00005B6B1A887B6803F580535A847B6803F504
:101D100080539B6A786898477B6803F580535B6BB8
:101D2000D3F8FC317A6802F5805213637B6803F5BF
:101D300080535B6BD3F80032002B14D07B6803F523
:101D400080535B6BD3F80032FB607B6803F58053F4
:101D50005B6B18461EF0B4FD7B6803F580531A4692
:101D6000FB68536310E07B6803F580535B6B184698
:101D70001EF0A6FD7B6803F580531A4600235363CB
:101D800002E07B6800221A7600BF1037BD4680BD96
:101D900080B582B000AF78607B68DB89012B2CD1E5
:101DA0007B681B89002B28D07B689B8901339AB202
:101DB0007B689A817B689B891A467B685B895B0894
:101DC0009BB219467B681B8991FBF3F39A4214DBA3
:101DD0007B6800229A817B681B68002B0DD07B6892
:101DE0001B685B68002B08D07B681B681B689847E2
:101DF0007B681B685A687B681A6000BF0837BD465D
:101E000080BD80B584B000AF786039600023FB608E
:101E10007B681B68002B27D17B685B68002B23D174
:101E200008201EF045FD03461A467B685A607B6811
:101E30005A687B681A607B681B683A681A607B681E
:101E40005B683A681A607B681B687A6852685A60F7
:101E50007B685B687A6812685A607B681B8901330B
:101E60009AB27B681A8119E008201EF021FD034612
:101E7000FB60FB683A681A607B681A68FB685A6006
:101E80007B685B68FA685A607B68FA685A607B68AE
:101E90001B8901339AB27B681A8100BF00BF1037DB
:101EA000BD4680BD90B587B000AFF860B9603B60BB
:101EB0001346FB7100237B61FB681B68002B2FD14D
:101EC000FB685B68002B2BD13C201EF0F1FC034625
:101ED0001A46FB685A60FB685A68FB681A60FB6820
:101EE0001B683222002118461EF02AFDFB681B6881
:101EF0001C46B868FEF7FEF903461A46B968204644
:101F00001EF0F6FCFB681B68FA7983F83220FB6848
:101F10001B683A685A63FB681B6800229A6326E0D4
:101F20003C201EF0C5FC03467B617B693222002108
:101F300018461EF005FD7C69B868FEF7DBF903461C
:101F40001A46B96820461EF0D3FC7B693A685A638A
:101F50007B69FA7983F832207B6900229A63FB68F7
:101F60005B687A699A63FB687A695A6000BF00BF50
:101F70001C37BD4690BD000090B589B004AF7860B5
:101F80007B681B8901339AB27B681A817B681B8945
:101F90005B007A685289934270DB7B681B68FB6048
:101FA000FB68002B03D17B6800221A8166E00023C6
:101FB000FB724FE0FB6893F83230012B3FD03222A6
:101FC000002130481EF0BCFCFC68FB681846FEF798
:101FD00091F903461A4621462A481EF089FC2A4BED
:101FE0001B78012B20D930231A0630231B041A43F7
:101FF00030231B021343302243EA020144231A0612
:1020000046231B041A434C231B02134354221A4336
:10201000FB6803931D4B0293892301931C4B009390
:102020001C4B022000F054FC1B4B1A68FB685B6BD6
:1020300019461046FEF73EFB0123FB7207E0164BE4
:102040001A68FB685B6B19461046FEF747FBFB6896
:102050009B6BFB60FB68002BACD17B681B68FB6053
:1020600006E0FB68002283F83220FB689B6BFB6074
:10207000FB68002BF5D17B6800221A811437BD461E
:1020800090BD00BF5C9B0024B49B0024BC4C0408A2
:10209000DC200408A8200408FC00002480B586B0D9
:1020A00000AFF860B9601346FB71FB681B687B6189
:1020B0000023FB747B69002B14D1002316E07B699D
:1020C000B9681846FEF70CF90346002B07D17B6967
:1020D000FA7983F832200123FB74FB7C06E07B69EC
:1020E0009B6B7B617B69002BE9D1FB7C1846183721
:1020F000BD4680BD80B500AF02490920FFF7C2F898
:1021000000BF80BD0921020880B500AF00F00CF8C7
:102110000246034B1B68A2F5E1621A6000BF80BD56
:10212000949B00240000000080B584B000AF4848B4
:1021300004F06CFB6421464804F066FC0346002B67
:102140006CD1434804F054FD03461A46414B1A60D3
:102150003F4804F025FC3F4B1B6807EE903AB8EE71
:10216000E77ADFED3D6AC7EE267A9FED3C7A67EEAF
:10217000877AC7ED037AD7ED037A9FED397A67EE58
:10218000876A9FED367AD7ED037A37EE677AC6EE27
:10219000877AC7ED027A97ED027ADFED316AC7EEF2
:1021A000267AC7ED017AD7ED017AB7EEE77AB0EE7D
:1021B000470B1FF0F1FDB0EE407BF7EEC77BC7ED9C
:1021C000017A97ED017ADFED276AC7EE267AC7ED2F
:1021D000017AD7ED017AB7EEE77A9FED176B37EE0C
:1021E000067BF7EEC77BC7ED017AF7EE006A97ED45
:1021F000017AC6EE877AC7ED017AD7ED017AB7EE9C
:10220000E77A9FED0F6B37EE467B9FED0F6B27EE66
:10221000067BFDEEC77B17EE903A06E00D4B0022E1
:102220001A600B4804F0BCFB002318461037BD466B
:1022300080BD00BFAFF3008045A725E6E1796B3F85
:102240006666666666127140000000000000594034
:102250000CAD0024909B002400FF7F473333534094
:1022600000401C460040534580B584B000AF034693
:10227000FB802E2017F09AF803461E4A13601D4B70
:102280001B68002B2FD01B4B1B68FA881A49184675
:1022900015F0E8FF0346FB7397F90F30002B09D0C8
:1022A000144B1B681946012014F0B6FB114B002299
:1022B0001A601BE00F4B1B68FF21184616F08AF8C6
:1022C00003460C4A13600B4B1B68002B0DD0094BC7
:1022D0001B680A49184617F0DDF818220021084843
:1022E0001EF02EFB02E000BF00E000BF1037BD462D
:1022F00080BD00BFB09B0024004E040805230208E7
:10230000989B002480B586B000AFF860B960134692
:10231000FB714FF0FF337B6100233B610CE01D4AF2
:102320003B69DB0013441B79002B02D13B697B61C5
:1023300005E03B6901333B613B69022BEFDD7B69C3
:10234000B3F1FF3F05D1B86815F080FF6FF00C03C3
:102350001BE00121B86816F037FE0F49B86817F086
:1023600033F80E49B86817F073F80D49B86817F0DC
:102370004DF808497B69BA6841F83320054A7B6902
:10238000DB00134401221A71002318461837BD469A
:1023900080BD00BF989B0024A523020811240208D9
:1023A0005D24020880B586B000AFF860B9607A603D
:1023B000FB707B68002B1BD100237B6110E0134A6C
:1023C0007B6952F83330BA689A4206D10F4A7B696A
:1023D000DB00134400221A7105E07B6901337B6145
:1023E0007B69022BEBDDB86815F046FE002309E09F
:1023F0007B681B891946B86816F002F9786815F0F1
:102400009DF9002318461837BD4680BD989B0024CF
:1024100080B485B000AF78600B46FB700023FB6092
:1024200010E00D4AFB6852F833307A689A4206D1C0
:10243000094AFB68DB00134400221A7106E0FB68BE
:102440000133FB60FB68022BEBDD00BF00BF1437DC
:10245000BD465DF8047B7047989B002480B485B02E
:1024600000AFF860B9601346FB8000BF1437BD466B
:102470005DF8047B7047000080B584B000AF7860E1
:102480000B467B800023FB601FE0144AFB68DB00E7
:1024900013441B79002B15D0104AFB6852F8330007
:1024A0007A880123796819F08FFE0346FB7297F949
:1024B0000B30002B06D1094AFB6852F8333018461E
:1024C0001AF06CFCFB680133FB60FB68022BDCDD5F
:1024D00000BF00BF1037BD4680BD00BF989B0024E1
:1024E00080B485B000AFF860B9607A60FB681A8884
:1024F000FB685B889A4201D101232DE0FB685B8871
:102500001A46FB6813441B79002B24D0FB685B88B8
:102510001A46FB681344DA7CBB681A70FB685B8858
:102520001A4613461B029B1A0E4A1A447B681A600D
:10253000FB685B885A1C0C4B83FB02131344D910B5
:10254000D317C91A0B461B015B1AD11A8AB2FB6852
:102550005A80002300E0012318461437BD465DF879
:10256000047B7047109C00248988888880B485B0DB
:1025700000AF786039607B681B885A1C154B83FB61
:1025800002131344D910D317C91A0B461B015B1A47
:10259000D11A0B46FB73FB7B9AB27B685B889A422D
:1025A00001D101230FE0FB7B9AB27B681A807B6824
:1025B0001B881A467B68134400221A717B681A88AC
:1025C0003B681A80002318461437BD465DF8047B2B
:1025D000704700BF8988888880B586B000AFB96031
:1025E0007A601A460346FB731346BB8100237B6166
:1025F0005B4B1B68002B08D0594B1B689847024661
:1026000013469B0013445B007B61BB89DE2B02D920
:10261000BB89213BBB813B6A44221A703B6A013370
:102620004C221A703B6A023353221A703B6A0333FE
:1026300001221A703B6A043335221A70494B1B7809
:102640005A1CD1B2474A11703A6A053213703B6A7C
:10265000063300221A70BB89DAB23B6A07331C3298
:10266000D2B21A7075231A0643231B041A43492356
:102670001B021343442213433B613B6A0833FA7C39
:102680001A703B6A0933BA7C1A703B6A0A337A7C47
:102690001A7007F110023B6A0B3312781A703B6A0A
:1026A0000C33FA7D1A703B6A0D33BA7D1A703B6A9F
:1026B0000E337A7D1A7007F114023B6A0F331278D9
:1026C0001A70FB7B1B015BB243F001035AB23B6AF9
:1026D0001033D2B21A703B6A113301221A703B6A6E
:1026E0001233FA7A1A703B6A1333BA7A1A703B6A59
:1026F00014337A7A1A7007F108023B6A153312789C
:102700001A703B6A1633FA791A703B6A1733BA7932
:102710001A703B6A18337A791A703A1D3B6A19337A
:1027200012781A703B6A1A3301221A703B6A1B3303
:1027300082221A703B6A1C3300221A703B6A1D33D6
:1027400000221A703B6A1E33BA89D2B21A703B6AF1
:102750001F3300221A7000BF1837BD4680BD00BF6E
:10276000C49B00240D9C002480B483B000AF78602B
:10277000044A7B68136000BF0C37BD465DF8047BDC
:10278000704700BFC09B002480B582B000AF786066
:10279000074A7B681360064B1B68002B04D0044B70
:1027A0001B68FF210348984700BF0837BD4680BD1E
:1027B000BC9B002404AB002480B586B002AF7860D7
:1027C000114A7B681360114B00930F23104A104984
:1027D0000220FFF701FF0023FB600AE0FB682033C3
:1027E0000C49FA680A441178084AD154FB6801334D
:1027F000FB60FB680E2BF1D9074B2F221A7000BF2C
:102800001037BD4680BD00BFB89B0024D09B00247C
:1028100043544C44040000240C9C002480B584B034
:1028200000AF0023FB7200237B600023FB60204B82
:102830001B68002B03D01E4B1B689847F8601D4B8C
:102840001B78002B17D01C4B1B68FA68D31AC82BB7
:1028500011D9194AFB681360164B00221A70174BE6
:102860001B68002B20D0154B1B68154A12781146A7
:102870001448984719E03A1D07F10B03194612480E
:10288000FFF72EFE0346002B0AD10C4B1B68002BD2
:102890000BD00A4B1B687A68F97A1046984704E017
:1028A0000A4B01221A7000E000BF1037BD4680BD00
:1028B000C49B0024C89B0024CC9B0024B89B00240C
:1028C0000C9C0024D09B002414000024360000241B
:1028D00008B480B58BB002AF0346B9607A60FB7371
:1028E00000237B770023BB610023FB8207F11603E3
:1028F00019464048FFF73AFE0346002B03D03E4BF3
:1029000001221A704FE007F130033B61FB8A1A463F
:1029100013461B029B1A2033384A13443A69F96A5A
:1029200018461EF091F90346FB83FB8B2033FB8393
:10293000FB8B0133FB83FB8A1846FA8B2F49034636
:102940001B021B1A0B44134400221A70FB8B013329
:10295000FB83FB8A1846FA8B284903461B021B1A85
:102960000B44134400221A70FB8A1A4613461B02BA
:102970009B1A224A1344FA8BF87B009313467A6819
:10298000B968FFF729FEFB8B2033FB83FB8A1946CE
:10299000FB8BDAB2174B0B44DA74FB8A1A46154BE1
:1029A000134401221A71164B1B78DBB2012B1AD18A
:1029B00007F1180207F11D0319460E48FFF790FDB5
:1029C0000346002B0FD17B7F002B0CD00C4B002239
:1029D0001A700C4B1B68002B05D00A4B1B68BA6998
:1029E000797F1046984700BF2437BD46BDE8804038
:1029F00001B0704714000024C89B0024109C0024E0
:102A000036000024B89B002480B483B000AF786007
:102A1000044A7B68136000BF0C37BD465DF8047B39
:102A2000704700BFC49B002480B582B000AF7860BF
:102A30000B467B807B88192B19D17B681B780F2B69
:102A40000CD17B6818331B78002B07D17B680133CE
:102A5000094A12681146184600F016F8074B1B6821
:102A60005B69064A106801220549984700E000BFEB
:102A70000837BD4680BD00BF04AD0024800200249D
:102A8000042104080000000080B48DB000AF78601D
:102A900039604FF0FF33BB62BB6A01337A6813447D
:102AA0001B781AB2BB6A023379680B441B781B028D
:102AB0001BB213431BB2C3F30A031BB23B81BB6AB5
:102AC00002337A6813441B78DB08DBB21AB2BB6AA4
:102AD000033379680B441B785B011BB213431BB2B1
:102AE000C3F30A031BB27B81BB6A03337A681344C6
:102AF0001B789B09DBB21AB2BB6A043379680B44BA
:102B00001B789B001BB213431AB2BB6A053379686A
:102B10000B441B789B021BB213431BB2C3F30A0383
:102B20001BB2BB81BB6A05337A6813441B785B0810
:102B3000DBB21AB2BB6A063379680B441B78DB013F
:102B40001BB213431BB2C3F30A031BB2FB81BB6A64
:102B500006337A6813441B781B09DBB21AB2BB6ACE
:102B6000073379680B441B781B011BB213431BB25C
:102B7000C3F30A031BB23B82BB6A07337A68134470
:102B80001B78DB09DBB21AB2BB6A083379680B44E5
:102B90001B785B001BB213431AB2BB6A0933796816
:102BA0000B441B785B021BB213431BB2C3F30A0333
:102BB0001BB27B82BB6A09337A6813441B789B087B
:102BC000DBB21AB2BB6A0A3379680B441B789B01EB
:102BD0001BB213431BB2C3F30A031BB2BB82BB6A13
:102BE0000A337A6813441B785B09DBB21AB2BB6AFA
:102BF0000B3379680B441B78DB001BB213431BB209
:102C0000C3F30A031BB2FB82BB6A0C337A6813441A
:102C10001B781AB2BB6A0D3379680B441B781B0210
:102C20001BB213431BB2C3F30A031BB23B83BB6A41
:102C30000D337A6813441B78DB08DBB21AB2BB6A27
:102C40000E3379680B441B785B011BB213431BB234
:102C5000C3F30A031BB27B83BB6A0E337A68134447
:102C60001B789B09DBB21AB2BB6A0F3379680B443D
:102C70001B789B001BB213431AB2BB6A10337968EE
:102C80000B441B789B021BB213431BB2C3F30A0312
:102C90001BB2BB83BB6A10337A6813441B785B0892
:102CA000DBB21AB2BB6A113379680B441B78DB01C3
:102CB0001BB213431BB2C3F30A031BB2FB83BB6AF1
:102CC00011337A6813441B781B09DBB21AB2BB6A52
:102CD000123379680B441B781B011BB213431BB2E0
:102CE000C3F30A031BB23B84BB6A12337A681344F2
:102CF0001B78DB09DBB21AB2BB6A133379680B4469
:102D00001B785B001BB213431AB2BB6A1433796899
:102D10000B441B785B021BB213431BB2C3F30A03C1
:102D20001BB27B84BB6A14337A6813441B789B08FC
:102D3000DBB21AB2BB6A153379680B441B789B016E
:102D40001BB213431BB2C3F30A031BB2BB84BB6A9F
:102D500015337A6813441B785B09DBB21AB2BB6A7D
:102D6000163379680B441B78DB001BB213431BB28C
:102D7000C3F30A031BB2FB840023FB621CE0FB6A63
:102D80005B0030333B4433F9283CA3F5787307EEFE
:102D9000903AB8EEE77B9FED166B27EE067BFB6A59
:102DA00001339B003A681344FDEEC77B17EE902A6F
:102DB0001A60FB6A0133FB62FB6A0F2BDFDD7B6865
:102DC00016331B78002B04D13B68443301221A6070
:102DD00003E03B68443300221A603B681B685A1CBE
:102DE0003B681A6000BF3437BD465DF8047B70470E
:102DF000E5620CACE338F63F90B583B000AF786085
:102E00001F4A7B6813601E4B1B6803F580531A46EC
:102E10001C4B13631A4B1B6804229A60184B1B68E7
:102E200003F58053DB6B0022DA81174B1B68DC68EB
:102E3000154B1868002300221449A047144B1B7837
:102E4000032B18D930231A0630231B041A433023CE
:102E50001B021343302243EA020144231A0646238D
:102E60001B041A434C231B02134354221A43094BDD
:102E70000420FFF72DFD00BF0C37BD4690BD00BFFD
:102E800008AD0024292A0208800200240421040835
:102E9000B49B00241021040880B588B000AF3B1D0E
:102EA00000221A605A609A60DA601A615A619A6167
:102EB000294B2A4A1A60284B4FF480225A60264B2D
:102EC00000229A60244B0022DA60234B04221A610C
:102ED000214B00221A75204B01225A751E4B0122EC
:102EE0009A611D4B00221A771B4B00225A621A4B23
:102EF00000229A62184B0022DA62174B00221A63F2
:102F0000154B00225A63144B002283F838201248D4
:102F100003F0DAFA0346002B01D001F007FA104B58
:102F20007B600623BB600023FB6040F2FF733B61C4
:102F300004237B610023BB6100237B773B1D194683
:102F4000054803F063FE0346002B01D001F0EEF9C3
:102F500000BF2037BD4680BD0CAD002400210240DB
:102F60000000844B80B5B8B000AF786007F1CC03A7
:102F700000221A605A609A60DA601A6107F1100341
:102F8000BC22002118461DF0DBFC7B681B682A4A26
:102F900093424DD14FF400233B6119237B614FF4E1
:102FA0009073BB610423FB6102233B6202237B62BB
:102FB0000023BB620023FB6200233B630023C7F8AE
:102FC000B03007F1100318460CF0F2FE0346002B58
:102FD00001D001F0ABF9194BD3F8D830174A43F0C0
:102FE0002003C2F8D830154BD3F8D83003F02003B3
:102FF000FB60FB68114BD3F8E030104A43F001034B
:10300000C2F8E0300D4BD3F8E03003F00103BB60B1
:10301000BB681023C7F8CC300323C7F8D030002397
:10302000C7F8D43007F1CC03194605480AF01EFA58
:1030300000BFE037BD4680BD002102400044025879
:103040000000025880B582B000AF0D4BD3F8E030DD
:103050000B4A43F40013C2F8E030094BD3F8E030D8
:1030600003F400137B607B6800220021812004F0C0
:10307000A8FC812004F0BFFC00BF0837BD4680BD1E
:103080000044025880B582B000AF254BD3F8D83049
:10309000234A43F00103C2F8D830214BD3F8D8308B
:1030A00003F001037B607B68002200210B2004F009
:1030B00088FC0B2004F09FFC002200210C2004F06F
:1030C00080FC0C2004F097FC002200210D2004F06D
:1030D00078FC0D2004F08FFC002200210E2004F06B
:1030E00070FC0E2004F087FC002200210F2004F069
:1030F00068FC0F2004F07FFC00220021102004F067
:1031000060FC102004F077FC00220021112004F064
:1031100058FC112004F06FFC00BF0837BD4680BD8D
:103120000044025880B400AF414B424A1A60424BFF
:10313000424A1A60424B434A1A60434B434A1A6060
:10314000434B444A1A60444B444A1A60384B1B684C
:1031500003F580531A46424B1363354B1B680A2212
:103160009A60354B1B6803F580531A463D4B136339
:10317000314B1B680A229A60314B1B6803F5805360
:103180001A46394B13632E4B1B680A229A602E4B4A
:103190001B6803F580531A46344B13632A4B1B6894
:1031A0000A229A602A4B1B6803F580531A46304B5B
:1031B0001363274B1B680A229A60274B1B6803F591
:1031C00080531A462B4B1363234B1B680A229A60C9
:1031D000294B2A4A1A602A4B2A4A1A60264B1B6836
:1031E000294ADA61264B1B68284ADA61284B294AAA
:1031F0001A60274B1B6803F580531A46264B13634E
:10320000234B1B680A229A60244B254A1A60234BE1
:103210001B6803F580531A46224B13631F4B1B6830
:103220000A229A6000BFBD465DF8047B704700BF6C
:1032300070AD00241C09002474AD00245C19002426
:1032400078AD00249C2900247CAD0024DC390024C6
:1032500080AD00241C4A002484AD00249C6A002414
:10326000A9320208FD32020851330208A5330208D0
:10327000F93302089934020894AD00248402002432
:1032800090AD0024BC0300243935020889350208BA
:1032900088AD00241C8B0024ED3402088CAD002482
:1032A000DC7A00244D34020880B582B000AF78602B
:1032B0000B467B807B681B78012B18D10E4B1B685B
:1032C00003F621037A88796818461DF011FB0A4B32
:1032D0001B6803F580531A467B885384064B1B6892
:1032E00003F580539B6A044A12681046984700BF52
:1032F0000837BD4680BD00BF70AD002480B582B0E8
:1033000000AF78600B467B807B681B78022B18D15E
:103310000E4B1B6803F621037A88796818461DF066
:10332000E7FA0A4B1B6803F580531A467B885384DF
:10333000064B1B6803F580539B6A044A12681046CB
:10334000984700BF0837BD4680BD00BF74AD00245C
:1033500080B582B000AF78600B467B807B681B78BD
:10336000032B18D10E4B1B6803F621037A8879686A
:1033700018461DF0BDFA0A4B1B6803F580531A4628
:103380007B885384064B1B6803F580539B6A044A71
:1033900012681046984700BF0837BD4680BD00BF81
:1033A00078AD002480B582B000AF78600B467B809A
:1033B0007B681B78042B18D10E4B1B6803F6210386
:1033C0007A88796818461DF093FA0A4B1B6803F552
:1033D00080531A467B885384064B1B6803F5805341
:1033E0009B6A044A12681046984700BF0837BD46DA
:1033F00080BD00BF7CAD002480B582B000AF786096
:103400000B467B807B681B78052B18D10E4B1B6805
:1034100003F621037A88796818461DF069FA0A4B89
:103420001B6803F580531A467B885384064B1B6840
:1034300003F580539B6A044A12681046984700BF00
:103440000837BD4680BD00BF80AD002480B582B086
:1034500000AF78600B467B800E4B1B6803F62103A0
:103460007A88796818461DF043FA0A4B1B6803F501
:1034700080531A467B885384064B1B6803F58053A0
:103480009B6A044A12681046984700BF0837BD4639
:1034900080BD00BF8CAD002480B582B000AF7860E5
:1034A0000B467B807B681B78062B18D10E4B1B6864
:1034B00003F621037A88796818461DF019FA0A4B39
:1034C0001B6803F580531A467B885384064B1B68A0
:1034D00003F580539B6A044A12681046984700BF60
:1034E0000837BD4680BD00BF84AD002480B582B0E2
:1034F00000AF78600B467B800E4B1B6803F6210300
:103500007A88796818461DF0F3F90A4B1B6803F5B1
:1035100080531A467B885384064B1B6803F58053FF
:103520009B6A044A12681046984700BF0837BD4698
:1035300080BD00BF88AD002490B587B002AFF860B1
:10354000B9607A60FB68012B17D10E4B1B68A8335A
:103550007A68B96818461DF0CBF90A4B1B689C695C
:10356000084B18687B68DAB2064B1B68A833002149
:103570000191022100910121A04700BF1437BD46EF
:1035800090BD00BF94AD002490B587B002AFF86045
:10359000B9607A60FB68022B17D10E4B1B68A83309
:1035A0007A68B96818461DF0A3F90A4B1B689C6934
:1035B000084B18687B68DAB2064B1B68A8330021F9
:1035C0000191022100910221A04700BF1437BD469E
:1035D00090BD00BF90AD002480B500AF2E4B2F4AA8
:1035E0001A602D4B00229A602B4B0022DA602A4B86
:1035F00000221A74284B00225A74274B00229A7416
:10360000254B0A225A61244B01229A61224B052242
:10361000DA61214B02221A621F4B01225A621E4BB1
:1036200001229A621C4B0122DA621B4B01221A63AF
:10363000194B00225A63184B00229A63164B002242
:10364000DA63154B20221A64134B04225A64124B7E
:1036500000229A64104B0422DA640F4B00221A6590
:103660000D4B04225A650C4B00229A650A4B00222E
:10367000DA65094B20221A66074B00225A66064B70
:1036800004229A66044808F0A3FD0346002B01D0EB
:1036900000F04CFE00BF80BD98AD002400A00040AB
:1036A00080B500AF2E4B2F4A1A602D4B00229A6036
:1036B0002B4B0022DA602A4B00221A74284B00227E
:1036C0005A74274B00229A74254B0A225A61244BC4
:1036D00001229A61224B0522DA61214B02221A62F1
:1036E0001F4B01225A621E4B01229A621C4B01227F
:1036F000DA621B4B01221A63194B00225A63184BE2
:1037000000229A63164B0022DA63154B20221A64BA
:10371000134B04225A64124B00229A64104B042269
:10372000DA640F4B00221A650D4B04225A650C4BCC
:1037300000229A650A4B0022DA65094B20221A669C
:10374000074B00225A66064B04229A66044808F08A
:103750003FFD0346002B01D000F0E8FD00BF80BD17
:1037600038AE002400A4004080B5BAB000AF786045
:1037700007F1D40300221A605A609A60DA601A6175
:1037800007F11803BC22002118461DF0D9F87B6808
:103790001B685C4A934256D14FF40043BB614FF023
:1037A0008053C7F8843007F1180318460CF000FB6B
:1037B0000346002B01D000F0B9FD534B1B680133C9
:1037C000514A1360504B1B68012B0ED14F4BD3F85D
:1037D000EC304E4A43F48073C2F8EC304B4BD3F8D4
:1037E000EC3003F480737B617B69484BD3F8E030A5
:1037F000464A43F00203C2F8E030444BD3F8E030CD
:1038000003F002033B613B694FF44073C7F8D430C7
:103810000223C7F8D8300023C7F8DC300023C7F8EC
:10382000E0300923C7F8E43007F1D40319463848DB
:1038300009F01CFE00220021132004F0C2F813201E
:1038400004F0D9F859E07B681B68324A934254D19E
:103850004FF40043BB614FF08053C7F8843007F149
:10386000180318460CF0A4FA0346002B01D000F010
:103870005DFD254B1B680133234A1360224B1B68F7
:10388000012B0ED1214BD3F8EC30204A43F4807346
:10389000C2F8EC301D4BD3F8EC3003F48073FB60BE
:1038A000FB681A4BD3F8E030184A43F00203C2F821
:1038B000E030164BD3F8E03003F00203BB60BB6886
:1038C0006023C7F8D4300223C7F8D8300023C7F8E4
:1038D000DC300023C7F8E0300923C7F8E43007F1F3
:1038E000D40319460A4809F0C1FD00220021142022
:1038F00004F067F8142004F07EF800BFE837BD46F6
:1039000080BD00BF00A00040D8AE00240044025893
:103910000004025800A4004080B58CB000AF07F14D
:103920001C0300221A605A609A60DA601A617A4BAE
:10393000D3F8E030784A43F01003C2F8E030764B19
:10394000D3F8E03003F01003BB61BB69724BD3F8CE
:10395000E030714A43F00403C2F8E0306E4BD3F814
:10396000E03003F004037B617B696B4BD3F8E030FC
:10397000694A43F08003C2F8E030674BD3F8E03087
:1039800003F080033B613B69634BD3F8E030624A4C
:1039900043F00103C2F8E0305F4BD3F8E03003F0AE
:1039A0000103FB60FB685C4BD3F8E0305A4A43F0FC
:1039B0000203C2F8E030584BD3F8E03003F00203C2
:1039C000BB60BB68544BD3F8E030534A43F0080364
:1039D000C2F8E030504BD3F8E03003F008037B60CE
:1039E0007B6801227D214D4809F0F0FE012242F260
:1039F00004014B4809F0EAFE002240F201714848F8
:103A000009F0E4FE00224021464809F0DFFE0022D2
:103A10004FF4C051414809F0D9FE002240F60B4155
:103A2000414809F0D3FE01221021404809F0CEFEA2
:103A300041F67D03FB6101233B6200237B6200238F
:103A4000BB6207F11C031946344809F00FFD42F22E
:103A50000573FB6101233B6200237B620023BB6291
:103A600007F11C0319462E4809F000FD4023FB61B5
:103A700001233B6200237B620023BB6207F11C032E
:103A80001946284809F0F2FC42F20203FB610023C8
:103A90003B6200237B6207F11C0319461F4809F0B3
:103AA000E5FC40F60B43FB6101233B6200237B6294
:103AB0000023BB6207F11C0319461B4809F0D6FC22
:103AC00044F21003FB614FF488133B6200237B62D6
:103AD00007F11C031946144809F0C8FC1023FB61C8
:103AE00001233B6200237B620023BB6207F11C03BE
:103AF00019460E4809F0BAFC8023FB6100233B62A3
:103B000000237B6207F11C031946084809F0AEFC4C
:103B100000BF3037BD4680BD004402580010025837
:103B20000008025800000258000C02580004025815
:103B300080B500AF1B4B1C4A1A601A4B1B4A5A60D7
:103B4000184B00229A60174B0122DA60154B0022B5
:103B50001A61144B00225A61124B00229A61114BD8
:103B60000022DA610F4B00221A620E4809F062FE51
:103B70000346002B01D000F0D9FB002109480AF0D0
:103B80006EFD0346002B01D000F0D0FB002105485C
:103B90000AF0B0FD0346002B01D000F0C7FB00BFC8
:103BA00080BD00BFDCAE0024001C0058FFECC0103C
:103BB00080B5B8B000AF786007F1CC0300221A607E
:103BC0005A609A60DA601A6107F11003BC22002182
:103BD00018461CF0B5FE7B681B682D4A934252D1F3
:103BE00010233B610023C7F8A43007F110031846E7
:103BF0000CF0DEF80346002B01D000F097FB254BBC
:103C0000D3F8E030234A43F00803C2F8E030214BF8
:103C1000D3F8E03003F00803FB60FB684FF4405337
:103C2000C7F8CC301223C7F8D0300023C7F8D430FF
:103C30000023C7F8D8300423C7F8DC3007F1CC03E1
:103C40001946154809F012FC124BD3F8F430114A0A
:103C500043F08003C2F8F4300E4BD3F8F43003F095
:103C60008003BB60BB68002200215F2003F0A9FE37
:103C70005F2003F0C0FE00220021602003F0A1FEBF
:103C8000602003F0B8FE00BFE037BD4680BD00BF36
:103C9000001C005800440258000C0258B0B5ADF5A5
:103CA0000E7D0EAF00F0F4FA364B5B6903F400337F
:103CB000002B1BD1BFF34F8F00BFBFF36F8F00BF2F
:103CC000304B0022C3F85022BFF34F8F00BFBFF329
:103CD0006F8F00BF2B4B5B692A4A43F4003353615B
:103CE000BFF34F8F00BFBFF36F8F00E000BF254BC6
:103CF0005B6903F48033002B46D1224B0022C3F8CA
:103D00008420BFF34F8F00BF1E4BD3F88030C7F81D
:103D1000FC31D7F8FC315B0BC3F30E03C7F8F83165
:103D2000D7F8FC31DB08C3F30903C7F8F431D7F83F
:103D3000F8315A0143F6E0731340D7F8F4219207A3
:103D400010491343C1F86032D7F8F4315A1EC7F84E
:103D5000F421002BEBD1D7F8F8315A1EC7F8F8211F
:103D6000002BDDD1BFF34F8F00BF064B5B69054AC7
:103D700043F480335361BFF34F8F00BFBFF36F8FA6
:103D800003E000BF00ED00E000BF02F095F800F096
:103D9000D5F9FFF7C1FDFFF775F9FFF71DFCFFF738
:103DA0007FFCFFF7C5FE00F03BFE00F07DFF00F05A
:103DB000CFFF01F021F801F077F801F025F901F0CB
:103DC000CBF801F079F900F07FFE11F045FBFFF729
:103DD00063F8FFF737F900F0AFFA00F011FFFCF7D6
:103DE00093FC4FF47A70FCF709FFFCF722FD00F01A
:103DF00029FA64230D9364230C9364230B936423A7
:103E00000A93642309936423089364230793642328
:103E10000693642305931423049314230393062326
:103E200002931423019314230093142314221421C6
:103E30001420FDF70DFBB14B07221A70FCF782FC32
:103E4000AF48FEF7D9FFFFF76DF9FCF721FFAD4B47
:103E50001868AD4B1968AD4B1A68AD4B1B68FCF781
:103E6000E9FFFEF747F9FDF77FFAAA4BAA4A1A6065
:103E700041F28830FEF7F8F902F0A4F80346A74AA9
:103E800012689B1A40F6B732934221D902F09AF891
:103E900003461A46A14B1A600421A14809F0AFFC61
:103EA0001021A04809F0ABFC01219F4809F0A7FCB4
:103EB00008219D4809F0A3FC04219B4809F09FFCC0
:103EC0002021994809F09BFC1021974809F097FCA4
:103ED00001210720FDF76AF900210820FDF766F9A6
:103EE0004FF4FA6002F07AF801210720FDF75EF93D
:103EF00001210820FDF75AF94FF4FA6002F06EF83C
:103F000000210720FDF752F901210820FDF74EF9A5
:103F10004FF4FA6002F062F801210720FDF746F93C
:103F200001210820FDF742F94FF4FA6002F056F83B
:103F30003B464FF4FA72002118461CF001FD754B08
:103F40001B685968734B1B689C68724B1B68DB6865
:103F5000704A1268126938460192009323460A4655
:103F600072491CF03BFE654B1B78032B18D930239C
:103F70001A0630231B041A4330231B02134330223A
:103F800043EA020144231A0646231B041A434C2326
:103F90001B02134354221A433B460420FEF798FCAD
:103FA0003B464FF4FA72002118461CF0C9FC594BED
:103FB0001B685969574B1B689C69564B1B68DB692A
:103FC000544A1268126A38460192009323460A4600
:103FD00057491CF003FE494B1B78032B18D930239B
:103FE0001A0630231B041A4330231B0213433022CA
:103FF00043EA020144231A0646231B041A434C23B6
:104000001B02134354221A433B460420FEF760FC74
:104010003B464FF4FA72002118461CF091FC3D4BD0
:104020001B68596A3B4B1B689C6A3A4B1B68DB6AEE
:10403000384A1268126B38460192009323460A46AA
:104040003C491CF0CBFD2D4B1B78032B18D930239A
:104050001A0630231B041A4330231B021343302259
:1040600043EA020144231A0646231B041A434C2345
:104070001B02134354221A433B460420FEF728FC3C
:104080003B464FF4FA72002118461CF059FC214BB4
:104090001B685C6B1F4B1B689D6B1E4B1B68DB6BAF
:1040A0001C4A1268126C1B490968496C3846029117
:1040B000019200932B4622461F491CF08FFD0F4BA7
:1040C0001B78032B7FF6D8AE30231A0630231B044F
:1040D0001A4330231B021343302243EA02014423D4
:1040E0001A0646231B041A434C231B021343542273
:1040F0001A433B460420FEF7EBFBBDE6B49B0024CD
:104100005C5A0024380000243C00002440000024B5
:104110004400002404AD00244001002428AF002402
:104120000008025800040258001002582421040814
:1041300078210408C82104081C22040880B59CB01A
:1041400000AF07F124034C22002118461CF0F8FBB5
:104150003B1D2022002118461CF0F2FB02200AF031
:104160003DFB00233B60344BDB6A334A23F0010301
:10417000D362314BDB6A03F001033B602F4B9B6939
:104180002E4A43F4404393612C4B9B6903F4404314
:104190003B603B6800BF294B9B6903F40053B3F5B8
:1041A000005FF8D1264B9B6A23F00303244A43F0B7
:1041B0000203936201237B624FF48033BB620223CC
:1041C000BB640223FB6402233B6540237B6502231F
:1041D000BB651423FB6504233B660C237B6600232D
:1041E000BB660023FB6607F1240318460AF026FE8F
:1041F0000346002B01D000F099F83F237B60032396
:10420000BB600023FB6008233B6140237B614023AC
:10421000BB614FF48063FB6140233B623B1D022185
:1042200018460BF039FA0346002B01D000F07EF857
:1042300000BF7037BD4680BD0004005800480258DA
:1042400000440258B0B58CB000AF0C4C3B46184649
:10425000FCF7B2FC25463C460FCC0FC50FCC0FC572
:1042600094E80F0085E80F00054B064A1A60064BDC
:10427000064A1A6000BF3037BD46B0BD00010024B9
:10428000949B00243801002404AD00244001002444
:1042900080B584B000AF3B4600221A605A609A6035
:1042A000DA6003F0C3FB01233B7000237B701D4BDE
:1042B0007B600E233B7200237B720123BB720323BE
:1042C000FB7201233B7300237B730023BB7300232A
:1042D000FB733B46184603F0E1FB01237B70092387
:1042E0003B720023BB7201237B730123FB733B46AC
:1042F000184603F0D3FB02237B700B4B7B600E232D
:104300003B720123BB7200237B730023FB733B468C
:10431000184603F0C3FB042003F0A0FB00BF1037D6
:10432000BD4680BD000004300000033080B400AF03
:1043300072B600BFFEE7000080B500AF124B134A13
:104340001A60114B01225A600F4B20229A600E4BCB
:104350001022DA600C4B18221A610B4B4FF480626A
:104360005A61094B01229A61074B8022DA61064BA0
:1043700000221A6204480AF06BFA0346002B01D0AF
:10438000FFF7D4FF00BF80BD2CAF002400500052C7
:1043900080B5BAB000AF786007F1D40300221A608C
:1043A0005A609A60DA601A6107F11803BC22002192
:1043B00018461CF0C5FA7B681B684E4A934240F0D1
:1043C00094804FF00073BB6100233B6607F1180334
:1043D00018460BF0EDFC0346002B01D0FFF7A6FFBB
:1043E000454BD3F8D430444A43F48043C2F8D43028
:1043F000414BD3F8D43003F480437B617B693E4B5F
:10440000D3F8E0303C4A43F00203C2F8E0303A4BC4
:10441000D3F8E03003F002033B613B69364BD3F83D
:10442000E030354A43F01003C2F8E030324BD3F8A5
:10443000E03003F01003FB60FB682F4BD3F8E03053
:104440002D4A43F00403C2F8E0302B4BD3F8E030A0
:1044500003F00403BB60BB680423C7F8D430022315
:10446000C7F8D8300023C7F8DC300323C7F8E030A2
:104470000923C7F8E43007F1D40319461F4808F0B0
:10448000F5FF4FF4F063C7F8D4300223C7F8D830F3
:104490000023C7F8DC300323C7F8E0300A23C7F84D
:1044A000E43007F1D4031946154808F0DFFF4FF454
:1044B0000063C7F8D4300223C7F8D8300023C7F808
:1044C000DC300323C7F8E0300923C7F8E43007F1F4
:1044D000D40319460B4808F0C9FF002200215C20D4
:1044E00003F06FFA5C2003F086FA00BFE837BD46A0
:1044F00080BD00BF00500052004402580004025822
:10450000001002580008025880B483B000AF0A4B74
:10451000D3F8F430084A43F00203C2F8F430064BF3
:10452000D3F8F43003F002037B607B6800BF0C37E4
:10453000BD465DF8047B70470044025880B400AF6C
:10454000FEE780B400AFFEE780B400AFFEE780B4C2
:1045500000AFFEE780B400AFFEE780B400AF00BF5D
:10456000BD465DF8047B704780B400AF00BFBD4618
:104570005DF8047B704780B400AF00BFBD465DF8B6
:10458000047B704780B500AF01F008FD00BF80BD1F
:1045900080B500AF024804F0EFFD00BF80BD00BF52
:1045A0000CB5002480B500AF024804F0E5FD00BF63
:1045B00080BD00BF84B5002480B500AF024804F080
:1045C000DBFD00BF80BD00BF74B6002480B500AF26
:1045D000024804F0D1FD00BF80BD00BFFCB500243F
:1045E00080B500AF024804F0C7FD00BF80BD00BF2A
:1045F000ECB6002480B500AF024804F0BDFD00BF5A
:1046000080BD00BF64B7002480B500AF024804F04D
:10461000B3FD00BF80BD00BFDCB7002480B500AF94
:10462000024808F021FA00BF80BD00BF98AD002409
:1046300080B500AF024808F017FA00BF80BD00BF88
:1046400038AE002480B500AF02480DF00DFE00BF6B
:1046500080BD00BF7CAF002480B500AF02480EF0E3
:10466000F5FB00BF80BD00BF54B2002480B500AF91
:1046700002480EF0EBFB00BF80BD00BFE4B2002497
:1046800080B500AF02480EF0E1FB00BF80BD00BF67
:1046900074B3002480B500AF02480DF0E5FD00BF03
:1046A00080BD00BFC8AF002480B500AF02480EF047
:1046B000CDFB00BF80BD00BFA4B0002480B500AF1B
:1046C00002480EF0C3FB00BF80BD00BF34B1002420
:1046D00080B500AF024806F0CDFB00BF80BD00BF33
:1046E000B4B8002480B500AF02480EF0AFFB00BFA5
:1046F00080BD00BF04B4002480B500AF02480EF0B6
:10470000A5FB00BF80BD00BFC4B1002480B500AFD1
:1047100002480AF011F900BF80BD00BF2CAF002491
:1047200080B500AF024809F015F900BF80BD00BF99
:10473000DCAE002480B500AF024809F025F900BFC7
:1047400080BD00BFDCAE002480B500AF024804F09D
:1047500013FD00BF80BD00BF94B4002480B500AF3E
:1047600002480EF073FB00BF80BD00BF14B00024F0
:1047700080B400AF01231846BD465DF8047B704746
:1047800080B483B000AF78603960054B16221A60A0
:104790004FF0FF3318460C37BD465DF8047B704779
:1047A000BCEA002480B582B000AF78604FF0FF31E2
:1047B0007868FFF7E5FFFEE780B586B000AFF860E8
:1047C000B9607A6000237B610AE0AFF300800146A4
:1047D000BB685A1CBA60CAB21A707B6901337B612C
:1047E0007A697B689A42F0DB7B6818461837BD46C9
:1047F00080BD80B586B000AFF860B9607A600023F4
:104800007B6109E0BB685A1CBA601B781846AFF39D
:1048100000807B6901337B617A697B689A42F1DBB6
:104820007B6818461837BD4680BD80B483B000AFA2
:1048300078604FF0FF3318460C37BD465DF8047BB7
:10484000704780B483B000AF786039603B684FF444
:1048500000525A60002318460C37BD465DF8047BB1
:10486000704780B483B000AF7860012318460C37DE
:10487000BD465DF8047B704780B485B000AFF8603A
:10488000B9607A60002318461437BD465DF8047B92
:104890007047000080B487B000AF7860144A154BB1
:1048A000D31A7B617B693B61134B1B68002B02D1E0
:1048B000114B124A1A60104B1A687B6813443A690C
:1048C0009A4205D20E4B0C221A604FF0FF3309E0DA
:1048D000094B1B68FB60084B1A687B681344064A47
:1048E0001360FB6818461C37BD465DF8047B7047B3
:1048F000000008240010000078AF0024C8EA00245B
:10490000BCEA002480B400AF394BD3F88830384A71
:1049100043F47003C2F88830364B1B6803F00F0372
:10492000062B07D8334B1B6823F00F03314A43F0A3
:1049300007031360304B1B682F4A43F001031360D9
:104940002D4B00221A612C4B1A682B492B4B13401C
:104950000B60284B1B6803F00803002B07D0254B86
:104960001B6823F00F03234A43F007031360224B15
:1049700000229A61204B0022DA611F4B00221A624A
:104980001D4B1F4A9A621C4B1E4ADA621A4B1E4A82
:104990001A63194B00225A63174B1B4A9A63164B32
:1049A0000022DA63144B184A1A64134B00225A642B
:1049B000114B1B68104A23F4802313600E4B002216
:1049C0001A66124B1A68124B1340B3F1005F02D201
:1049D000104B01221A60104B43F2D2021A60044BB2
:1049E0000E4A9A6000BFBD465DF8047B704700BF69
:1049F00000ED00E000200052004402587FEDF6EA8E
:104A0000000202020000FF01800201010010005CB0
:104A10000000FFFF08810051004000520000020822
:104A200080B588B000AF07F1100300221A605A6009
:104A30009A60DA603B1D00221A605A609A60204B2F
:104A4000204A1A601E4B40F2CF725A601C4B002263
:104A50009A601B4B42F20F72DA60194B00221A6106
:104A6000174B00225A61164B80229A6114480DF0B0
:104A70002BFB0346002B01D0FFF758FC4FF480536B
:104A80003B6107F1100319460D480DF00DFD03467B
:104A9000002B01D0FFF74AFC00237B600023BB60A2
:104AA0000023FB603B1D194605480DF055FF0346EA
:104AB000002B01D0FFF73AFC00BF2037BD4680BD78
:104AC0007CAF00240000014080B588B000AF07F142
:104AD000100300221A605A609A60DA603B1D0022BF
:104AE0001A605A609A60204B204A1A601E4B40F2AE
:104AF000CF725A601C4B00229A601B4BC722DA60AF
:104B0000194B00221A61184B00225A61164B0022E1
:104B10009A6115480DF0D8FA0346002B01D0FFF733
:104B200005FC4FF480533B6107F1100319460E4812
:104B30000DF0BAFC0346002B01D0FFF7F7FB002372
:104B40007B600023BB600023FB603B1D19460648C9
:104B50000DF002FF0346002B01D0FFF7E7FB00BF7B
:104B60002037BD4680BD00BFC8AF0024000401400F
:104B700080B584B000AF78607B681B681D4A9342A3
:104B800017D11D4BD3F8F0301B4A43F00103C2F894
:104B9000F030194BD3F8F03003F00103FB60FB68F1
:104BA00000220021192002F00CFF192002F023FF3F
:104BB0001BE07B681B68114A934216D10E4BD3F859
:104BC000F0300D4A43F00203C2F8F0300A4BD3F83C
:104BD000F03003F00203BB60BB68002200212C20F0
:104BE00002F0EFFE2C2002F006FF00BF1037BD469A
:104BF00080BD00BF00000140004402580004014095
:104C000080B500AF264B274A1A60254B4FF461420E
:104C10005A60234B00229A60214B0022DA60204B1D
:104C200000221A611E4B0C225A611D4B00229A6110
:104C30001B4B00221A621A4B00225A62184B302278
:104C40009A62174B4FF48052DA63154B4FF40052BF
:104C50001A64134B00225A6611480DF029FF0346CF
:104C6000002B01D0FFF762FB00210D4810F029FB5B
:104C70000346002B01D0FFF759FB0021084810F034
:104C80005EFB0346002B01D0FFF750FB044810F0F9
:104C9000DFFA0346002B01D0FFF748FB00BF80BDC1
:104CA00014B00024000C005880B500AF264B274AF2
:104CB0001A60254B4FF4E1325A60234B00229A6070
:104CC000214B0022DA60204B00221A611E4B0C227D
:104CD0005A611D4B00229A611B4B0022DA611A4B6C
:104CE00000221A62184B00225A62174B30229A6235
:104CF000154B4FF48052DA63134B4FF400521A6491
:104D000011480DF0D5FE0346002B01D0FFF70EFB36
:104D100000210D4810F0D5FA0346002B01D0FFF713
:104D200005FB0021084810F00AFB0346002B01D0C8
:104D3000FFF7FCFA044810F08BFA0346002B01D071
:104D4000FFF7F4FA00BF80BDA4B00024004C00407F
:104D500080B500AF264B274A1A60254B4FF46142BD
:104D60005A60234B00229A60214B0022DA60204BCC
:104D700000221A611E4B0C225A611D4B00229A61BF
:104D80001B4B0022DA611A4B00221A62184B0022D8
:104D90005A62174B30229A62154B4FF48052DA63F5
:104DA000134B4FF400521A6411480DF081FE034674
:104DB000002B01D0FFF7BAFA00210D4810F081FA5C
:104DC0000346002B01D0FFF7B1FA0021084810F08C
:104DD000B6FA0346002B01D0FFF7A8FA044810F0FA
:104DE00037FA0346002B01D0FFF7A0FA00BF80BDC1
:104DF00034B100240050004080B500AF284B294A50
:104E00001A60274B4FF4E1325A60254B00229A601A
:104E1000234B0022DA60224B00221A61204B0C2225
:104E20005A611F4B00229A611D4B0022DA611C4B14
:104E300000221A621A4B00225A62194B38229A62D7
:104E4000174B4FF400429A63154B4FF48052DA63CC
:104E5000134B4FF400521A6411480DF029FE03461B
:104E6000002B01D0FFF762FA00210D4810F029FA5B
:104E70000346002B01D0FFF759FA0021084810F033
:104E80005EFA0346002B01D0FFF750FA044810F0F9
:104E9000DFF90346002B01D0FFF748FA00BF80BDC1
:104EA000C4B100240078004080B500AF284B294AE7
:104EB0001A60274B4FF4E1325A60254B00229A606A
:104EC000234B0022DA60224B00221A61204B0C2275
:104ED0005A611F4B00229A611D4B0022DA611C4B64
:104EE00000221A621A4B00225A62194B38229A6227
:104EF000174B4FF400429A63154B4FF48052DA631C
:104F0000134B4FF400521A6411480DF0D1FD0346C3
:104F1000002B01D0FFF70AFA00210D4810F0D1F95B
:104F20000346002B01D0FFF701FA0021084810F0DA
:104F300006FA0346002B01D0FFF7F8F9044810F0F9
:104F400087F90346002B01D0FFF7F0F900BF80BDC1
:104F500054B200240010014080B500AF274B284A0E
:104F60001A60264B274A5A60244B4FF480529A60AD
:104F7000224B0022DA60214B4FF480621A611F4BF2
:104F80000C225A611D4B00229A611C4B0022DA61EF
:104F90001A4B00221A62194B00225A62174B302218
:104FA0009A62164B4FF48052DA63144B4FF400525E
:104FB0001A6412480DF07CFD0346002B01D0FFF768
:104FC000B5F900210D4810F07CF90346002B01D003
:104FD000FFF7ACF90021094810F0B1F90346002BA6
:104FE00001D0FFF7A3F9054810F032F90346002B72
:104FF00001D0FFF79BF900BF80BD00BFE4B20024E1
:1050000000440040A086010080B500AF284B294A2B
:105010001A60274B4FF4E1325A60254B00229A6008
:10502000234B0022DA60224B00221A61204B0C2213
:105030005A611F4B00229A611D4B0022DA611C4B02
:1050400000221A621A4B00225A62194B38229A62C5
:10505000174B4FF400429A63154B4FF48052DA63BA
:10506000134B4FF400521A6411480DF021FD034612
:10507000002B01D0FFF75AF900210D4810F021F95B
:105080000346002B01D0FFF751F90021084810F02A
:1050900056F90346002B01D0FFF748F9044810F0F9
:1050A000D7F80346002B01D0FFF740F900BF80BDC1
:1050B00074B300240048004080B500AF284B294A53
:1050C0001A60274B4FF4E1325A60254B00229A6058
:1050D000234B0022DA60224B00221A61204B0C2263
:1050E0005A611F4B00229A611D4B0022DA611C4B52
:1050F00000221A621A4B00225A62194B38229A6215
:10510000174B4FF400429A63154B4FF48052DA6309
:10511000134B4FF400521A6411480DF0C9FC0346BA
:10512000002B01D0FFF702F900210D4810F0C9F85B
:105130000346002B01D0FFF7F9F80021084810F0D2
:10514000FEF80346002B01D0FFF7F0F8044810F0FA
:105150007FF80346002B01D0FFF7E8F800BF80BDC1
:1051600004B400240014014080B5C8B000AF07F5B6
:105170009073A3F58E73186007F5867300221A608A
:105180005A609A60DA601A6107F15003BC2200216C
:1051900018461BF0D5FB07F59073A3F58E731B68BB
:1051A0001B688B4A93427ED104233B650023C7F8DA
:1051B000E03007F1500318460AF0FAFD0346002BD1
:1051C00001D0FFF7B3F8834BD3F8F430814A43F0B2
:1051D0000803C2F8F4307F4BD3F8F43003F008032F
:1051E000FB64FB6C7B4BD3F8E0307A4A43F001035D
:1051F000C2F8E030774BD3F8E03003F00103BB6432
:10520000BB6C4FF4C063C7F80C310223C7F81031F0
:105210000023C7F814310023C7F818310323C7F857
:105220001C3107F5867319466B4808F01FF96B4B64
:105230006B4A1A60694B0A225A60684B40229A6096
:10524000664B0022DA60654B4FF480621A61634B53
:1052500000225A61614B00229A61604B0022DA61A0
:105260005E4B00221A625D4802F05CFC0346002B94
:1052700001D0FFF75BF807F59073A3F58E731B68F9
:10528000564A9A67554A07F59073A3F58E731B68C3
:105290009363002200218E2002F093FB8E2002F007
:1052A000AAFB00F067BC07F59073A3F58E731B682B
:1052B0001B684C4A934240F09B8002233B650023CD
:1052C000C7F8C43007F1500318460AF071FD0346D1
:1052D000002B01D0FFF72AF83E4BD3F8E8303D4AC7
:1052E00043F40023C2F8E8303A4BD3F8E83003F433
:1052F00000237B647B6C374BD3F8E030354A43F0B6
:105300000103C2F8E030334BD3F8E03003F001037F
:105310003B643B6C4FF4C053C7F80C310223C7F811
:1053200010310023C7F814310023C7F818310623C1
:10533000C7F81C3107F586731946274808F096F818
:10534000294B2A4A1A60284B40225A60264B402299
:105350009A60254B0022DA60234B4FF480621A6179
:10536000214B00225A61204B00229A611E4B0022E1
:10537000DA611D4B00221A621B4B04225A621A4B3F
:1053800003229A62184B0022DA62174B00221A633A
:10539000154802F0C7FB0346002B01D0FEF7C6FFFD
:1053A00007F59073A3F58E731B680F4A9A670E4A30
:1053B00007F59073A3F58E731B6893630022002199
:1053C000342002F0FEFA342002F015FBD2E300BFD5
:1053D000000C0058004402580000025894B4002405
:1053E00008540258004C00400CB500241000024044
:1053F00007F59073A3F58E731B681B68994A934257
:1054000040F0A58002233B650023C7F8C43007F1B4
:10541000500318460AF0CCFC0346002B01D0FEF7DF
:1054200085FF914BD3F8E8308F4A43F48013C2F8DC
:10543000E8308D4BD3F8E83003F48013FB63FB6B4B
:10544000894BD3F8E030884A43F00403C2F8E030D7
:10545000854BD3F8E03003F00403BB63BB6B824B96
:10546000D3F8E030804A43F00803C2F8E0307E4BC6
:10547000D3F8E03003F008037B637B6B4FF4805379
:10548000C7F80C310223C7F810310023C7F81431D4
:105490000023C7F818310823C7F81C3107F58673B5
:1054A0001946724807F0E2FF0423C7F80C310223C3
:1054B000C7F810310023C7F814310023C7F818319A
:1054C0000823C7F81C3107F586731946684807F0AA
:1054D000CDFF684B684A1A60664B42225A60654BA2
:1054E00040229A60634B0022DA60624B4FF4806284
:1054F0001A61604B00225A615E4B00229A615D4B3B
:105500000022DA615B4B00221A625A4B00225A6277
:10551000584802F007FB0346002B01D0FEF706FFB8
:1055200007F59073A3F58E731B68524A9A67514A28
:1055300007F59073A3F58E731B6893630022002117
:10554000352002F03EFA352002F055FA12E307F555
:105550009073A3F58E731B681B68484A934240F012
:10556000958002233B650023C7F8C43007F1500340
:1055700018460AF01DFC0346002B01D0FEF7D6FEAC
:10558000394BD3F8E830384A43F08043C2F8E8306A
:10559000354BD3F8E83003F080433B633B6B324B31
:1055A000D3F8E030304A43F00103C2F8E0302E4B2C
:1055B000D3F8E03003F00103FB62FB6A4FF40143D0
:1055C000C7F80C310223C7F810310023C7F8143193
:1055D0000023C7F818310B23C7F81C3107F5867371
:1055E0001946274807F042FF264B274A1A60254BE9
:1055F00050225A60234B40229A60224B0022DA60EC
:10560000204B4FF480621A611E4B00225A611D4BE1
:1056100000229A611B4B0022DA611A4B00221A62A7
:10562000184B00225A62174802F07CFA0346002BFE
:1056300001D0FEF77BFE07F59073A3F58E731B6810
:10564000104A9A670F4A07F59073A3F58E731B688B
:10565000936300220021522002F0B3F9522002F09D
:10566000CAF987E20050004000440258000802587E
:10567000000C025884B50024280002400078004045
:1056800000000258FCB500245800024007F5907352
:10569000A3F58E731B681B68934A934240F08A807F
:1056A00001233B650023C7F8C83007F150031846B3
:1056B0000AF07EFB0346002B01D0FEF737FE8B4B32
:1056C000D3F8F030894A43F01003C2F8F030874B2A
:1056D000D3F8F03003F01003BB62BB6A834BD3F8FE
:1056E000E030824A43F00203C2F8E0307F4BD3F847
:1056F000E03003F002037B627B6A4FF44043C7F85B
:105700000C310223C7F810310023C7F814310023ED
:10571000C7F818310423C7F81C3107F586731946FA
:10572000734807F0A3FE734B734A1A60714B2A2229
:105730005A60704B40229A606E4B0022DA606D4BCB
:105740004FF480621A616B4B00225A61694B002250
:105750009A61684B0022DA61664B00221A62654B3F
:1057600004225A62634B03229A62624B0022DA627D
:10577000604B00221A635F4802F0D4F90346002B05
:1057800001D0FEF7D3FD07F59073A3F58E731B6868
:10579000584A9A67574A07F59073A3F58E731B68AA
:1057A000936300220021252002F00BF9252002F04E
:1057B00022F9DFE107F59073A3F58E731B681B6870
:1057C0004E4A934240F0A28002233B650023C7F873
:1057D000C43007F1500318460AF0EAFA0346002BDA
:1057E00001D0FEF7A3FD414BD3F8E8303F4A43F424
:1057F0000033C2F8E8303D4BD3F8E83003F4003210
:1058000007F59073A3F580731A6007F59073A3F5FD
:1058100080731B68354BD3F8E030344A43F00803FB
:10582000C2F8E030314BD3F8E03003F0080207F55E
:105830009073A3F582731A6007F59073A3F58273D2
:105840001B686023C7F80C310223C7F8103100230E
:10585000C7F814310023C7F818310723C7F81C31E3
:1058600007F586731946264807F000FE254B264AA1
:105870001A60244B2C225A60224B40229A60214B02
:105880000022DA601F4B4FF480621A611D4B002228
:105890005A611C4B00229A611A4B0022DA61194BA3
:1058A00000221A62174B00225A62164802F03AF997
:1058B0000346002B01D0FEF739FD07F59073A3F5E1
:1058C0008E731B680F4A9A670E4A07F59073A3F50B
:1058D0008E731B68936300220021262002F071F86A
:1058E000262002F088F845E10010014000440258EB
:1058F0000004025874B600244000024000440040F6
:10590000000C0258ECB600247000024007F59073BA
:10591000A3F58E731B681B68994A934240F09180EF
:1059200002233B650023C7F8C43007F15003184633
:105930000AF03EFA0346002B01D0FEF7F7FC914B2C
:10594000D3F8E8308F4A43F48023C2F8E8308D4B17
:10595000D3F8E83003F4802207F59073A3F584733D
:105960001A6007F59073A3F584731B68854BD3F811
:10597000E030844A43F00803C2F8E030814BD3F8AA
:10598000E03003F0080207F59073A3F586731A6000
:1059900007F59073A3F586731B684FF44073C7F83F
:1059A0000C310223C7F810310023C7F8143100234B
:1059B000C7F818310723C7F81C3107F58673194655
:1059C000714807F053FD714B714A1A606F4B2E22DC
:1059D0005A606E4B40229A606C4B0022DA606B4B2F
:1059E0004FF480621A61694B00225A61674B0022B2
:1059F0009A61664B0022DA61644B00221A62634BA3
:105A000000225A62614802F08DF80346002B01D053
:105A1000FEF78CFC07F59073A3F58E731B685B4A49
:105A20009A675A4A07F59073A3F58E731B689363C0
:105A300000220021272001F0C4FF272001F0DBFF16
:105A400098E007F59073A3F58E731B681B68514AA5
:105A5000934240F08F8001233B650023C7F8C83094
:105A600007F1500318460AF0A3F90346002B01D0B2
:105A7000FEF75CFC434BD3F8F030424A43F020037E
:105A8000C2F8F0303F4BD3F8F03003F0200207F5B6
:105A90009073A3F588731A6007F59073A3F5887364
:105AA0001B68384BD3F8E030364A43F00403C2F8A1
:105AB000E030344BD3F8E03003F0040207F5907384
:105AC000A3F58A731A6007F59073A3F58A731B68B0
:105AD000C023C7F80C310223C7F810310023C7F8E0
:105AE00014310023C7F818310723C7F81C3107F514
:105AF00086731946284807F0B9FC284B284A1A60D3
:105B0000264B48225A60254B40229A60234B0022A4
:105B1000DA60224B4FF480621A61204B00225A61F6
:105B20001E4B00229A611D4B0022DA611B4B0022A2
:105B30001A621A4B00225A62184801F0F3FF03461A
:105B4000002B01D0FEF7F2FB07F59073A3F58E73DF
:105B50001B68124A9A67114A07F59073A3F58E7372
:105B60001B68936300220021472001F02AFF472091
:105B700001F041FF00BF07F59077BD4680BD00BF33
:105B80000048004000440258000C025864B700244A
:105B9000880002400014014000080258DCB70024CD
:105BA000A0000240DFF834D0FEF7ACFE0C480D49EF
:105BB0000D4A002302E0D458C4500433C4188C4268
:105BC000F9D30A4A0A4C002301E013600432A242CE
:105BD000FBD31AF049FEFEF761F870470000082475
:105BE00000000024DC00002400580408DC0000242D
:105BF000C4EA0024FEE780B483B000AF7860396067
:105C00007B68002B0BD03B68DB68002B07D03B6820
:105C10009B68002B03D03B681B69002B02D14FF01F
:105C2000FF3314E03B681A687B689A603B685A68E7
:105C30007B68DA603B68DA687B685A613B689A681F
:105C40007B681A613B681A697B689A610023184671
:105C50000C37BD465DF8047B704780B586B000AF59
:105C600078600023FB600023BB6000237B6100237E
:105C70003B617B685B68002B7CD17B689B68002B59
:105C800002D07B689B6898477B6820221A600023BB
:105C90007B611CE07B685B6907F10802122178696F
:105CA00098470346002B03DA6FF004033B610BE0D7
:105CB000BB6803F01F037A699A4205D17B687A6951
:105CC0001A6000233B6105E07B6901337B617B69DE
:105CD0001F2BDFD97B681B681F2B02D96FF00203D3
:105CE0003B613B69002B45D17B681B697A68106872
:105CF0004FF40042002198470346002B37DB7B68B6
:105D00005B697A68106807F108020021984703462A
:105D1000002B28DB7B689B6998470346FB601CE0EF
:105D20007B689B69984703461A46FB68D31AB3F50C
:105D3000FA7F0ED87B685B697A68106807F1080201
:105D4000002198470346002B07DA6FF004033B61FC
:105D500010E06FF001033B610CE0BB6803F400430B
:105D6000002BDDD106E06FF004033B6102E06FF031
:105D700003033B613B69002B12D17B689B69984709
:105D80000346FB6000BF7B689B69984703461A4641
:105D9000FB68D31AB3F5FA6FF5D97B6801225A6014
:105DA0003B6918461837BD4680BD80B584B000AF4A
:105DB00078600023FB607B685B697A68106807F194
:105DC0000C02012198470346002B02DA6FF004030E
:105DD0006EE07B685B697A68106807F10C0201214C
:105DE00098470346002B02DA6FF0040360E0FB687B
:105DF00003F00403002B01D1012359E07B685B69A8
:105E00007A68106807F10C02002198470346002BBE
:105E100002DA6FF004034BE0FB6803F48053002BBD
:105E20001BD1FB6803F40053002B06D0FB6803F47E
:105E30008073002B01D002233AE0FB6803F4005387
:105E4000002B01D0032333E0FB6803F48073002BA5
:105E500001D004232CE005232AE07B685B697A6883
:105E6000106807F10C021F2198470346002B02DA45
:105E70006FF004031CE0FB6803F48053002B01D196
:105E8000062315E0FB6803F01C03182B01D1022345
:105E90000EE0FB6803F01C03082B01D1032307E08D
:105EA000FB6803F01C03142B01D1042300E005233D
:105EB00018461037BD4680BD80B582B000AF0320C4
:105EC00001F074FD09F09EFD0246154B9B691B0A0B
:105ED00003F00F031349CB5C03F01F0322FA03F313
:105EE0007B600F4B9B6903F00F030E4AD35C03F0FA
:105EF0001F037A6822FA03F30B4A13600B4A7B688C
:105F000013600F2000F014F80346002B01D001238A
:105F100002E0FEF7F9FA002318460837BD4680BDB7
:105F200000440258D44C04084C00002448000024CB
:105F300080B582B000AF7860154B1B78002B01D183
:105F4000012321E0134B1A68114B1B7819464FF4BB
:105F50007A73B3FBF1F3B2FBF3F3184601F059FD8A
:105F60000346002B01D001230EE07B680F2B0AD8DB
:105F7000002279684FF0FF3001F023FD064A7B686C
:105F80001360002300E0012318460837BD4680BD9A
:105F900054000024480000245000002480B400AFC6
:105FA000064B1B781A46064B1B681344044A1360C1
:105FB00000BFBD465DF8047B704700BF540000245D
:105FC00054B8002480B400AF034B1B681846BD468C
:105FD0005DF8047B704700BF54B8002480B584B0DE
:105FE00000AF7860FFF7EEFFB8607B68FB60FB688E
:105FF000B3F1FF3F05D00A4B1B781A46FB681344E8
:10600000FB6000BFFFF7DEFF0246BB68D31AFA68E9
:106010009A42F7D800BF00BF1037BD4680BD00BF11
:106020005400002480B400AF034B1B681B0C1846BF
:10603000BD465DF8047B70470010005C80B483B0FF
:1060400000AF7860064B5B6823F4600204497B680C
:1060500013434B6000BF0C37BD465DF8047B7047AF
:106060000004005880B483B000AF786039607B686A
:106070009B6823F47C123B681A437B689A6000BFDC
:106080000C37BD465DF8047B704780B483B000AF29
:10609000786039607B689B6823F0E0723B681A4344
:1060A0007B689A6000BF0C37BD465DF8047B704783
:1060B00080B483B000AF78607B689B6803F0E073C6
:1060C00018460C37BD465DF8047B704780B487B036
:1060D00000AFF860B9607A603B60FB6860331A46D5
:1060E000BB689B0013447B617B691B6803F0004223
:1060F0007B6803F0F8413B680B431A437B691A60E5
:1061000000BF1C37BD465DF8047B704780B485B086
:1061100000AFF860B9607A60FB681B6923F4F04255
:10612000BB6803F01F03796801FA03F31A43FB68A5
:106130001A6100BF1437BD465DF8047B704780B418
:1061400087B000AFF860B9607A60FB6860331A46C8
:10615000BB689B0013447B617B691B6823F0004292
:106160007B681A437B691A6000BF1C37BD465DF827
:10617000047B704780B483B000AF78607B68DB68D5
:1061800003F44063002B01D1012300E000231846F3
:106190000C37BD465DF8047B704780B487B000AF14
:1061A000F860B9607A60FB6830331A46BB681B0A36
:1061B0009B0003F00C0313447B617B691A68BB6886
:1061C00003F01F031F2101FA03F3DB431A407B682E
:1061D0009B0E03F01F01BB6803F01F0301FA03F3DA
:1061E0001A437B691A6000BF1C37BD465DF8047B0B
:1061F000704780B487B000AFF860B9607A60FB6820
:1062000014331A46BB685B0E9B0003F0040313446F
:106210007B617B691A68BB681B0D03F01F030721B4
:1062200001FA03F3DB431A40BB681B0D03F01F03A5
:10623000796801FA03F31A437B691A6000BF1C37BF
:10624000BD465DF8047B704780B485B000AFF86050
:10625000B9607A60FB68D3F8C020BB68C3F313034E
:10626000DB431A407B6803F018030849D940BB6838
:106270000B40C3F313031A43FB68C3F8C02000BFED
:106280001437BD465DF8047B704700BFFFFF0F0069
:1062900080B483B000AF78607B689B6803F01F0315
:1062A00018460C37BD465DF8047B704780B483B058
:1062B00000AF78607B689B6803F4404318460C3756
:1062C000BD465DF8047B704780B483B000AF786052
:1062D0007B689A68044B13407A68936000BF0C3760
:1062E000BD465DF8047B7047C0FFFF5F80B483B09C
:1062F00000AF78607B689B6803F00053B3F1005FE8
:1063000001D1012300E0002318460C37BD465DF89B
:10631000047B704780B483B000AF78607B689A6874
:10632000054B134043F080527B689A6000BF0C37E6
:10633000BD465DF8047B7047C0FFFF6F80B483B03B
:1063400000AF78607B689B6803F08053B3F1805F97
:1063500001D1012300E0002318460C37BD465DF84B
:10636000047B704780B483B000AF78607B689A6824
:10637000054B134043F001027B689A6000BF0C3765
:10638000BD465DF8047B7047C0FFFF7F80B483B0DB
:1063900000AF78607B689A68054B134043F00202B7
:1063A0007B689A6000BF0C37BD465DF8047B704780
:1063B000C0FFFF7F80B483B000AF78607B689B68CC
:1063C00003F00103012B01D1012300E00023184653
:1063D0000C37BD465DF8047B704780B483B000AFD6
:1063E00078607B689B6803F00203022B01D10123D4
:1063F00000E0002318460C37BD465DF8047B70476B
:1064000080B483B000AF78607B689A68054B134016
:1064100043F004027B689A6000BF0C37BD465DF80C
:10642000047B7047C0FFFF7F80B483B000AF78600B
:106430007B689A68054B134043F010027B689A60B2
:1064400000BF0C37BD465DF8047B7047C0FFFF7F7F
:1064500080B483B000AF78607B689B6803F004036E
:10646000042B01D1012300E0002318460C37BD4660
:106470005DF8047B7047000080B483B000AF7860A3
:106480007B689A68054B134043F020027B689A6052
:1064900000BF0C37BD465DF8047B7047C0FFFF7F2F
:1064A00080B483B000AF78607B689B6803F008031A
:1064B000082B01D1012300E0002318460C37BD460C
:1064C0005DF8047B7047000090B589B000AF78603C
:1064D0000023FB770023BB607B68002B01D10123E5
:1064E0008FE17B68DB68002B7B685B6D002B09D13B
:1064F0007868FCF737FD7B6800229A657B6800228C
:1065000083F850207B681B681846FFF7EFFE0346B0
:10651000002B04D07B681B681846FFF7D5FE7B680C
:106520001B681846FFF70AFF0346002B14D17B684F
:106530001B681846FFF7EEFE874B1B689B09874ACE
:10654000A2FB03239B090133BB6002E0BB68013B54
:10655000BB60BB68002BF9D17B681B681846FFF74E
:10656000EDFE0346002B0DD17B685B6D43F01002FE
:106570007B685A657B689B6D43F001027B689A6576
:106580000123FB777B681B681846FFF761FF786182
:106590007B685B6D03F01003002B40F029817B6961
:1065A000002B40F025817B685B6D23F4817343F001
:1065B00002027B685A657B681B681846FFF7FAFE83
:1065C0000346002B36D17B681B68654A934204D092
:1065D0007B681B68634A93420ED16148FFF7EAFE6D
:1065E00004466048FFF7E6FE03462343002B0CBF3A
:1065F00001230023DBB208E05B48FFF7DBFE034624
:10660000002B0CBF01230023DBB2002B12D07B68D0
:106610001B68534A934204D07B681B68514A9342DB
:1066200001D1524A00E0524A7B685B681946104625
:10663000FFF718FDFFF7F6FC034641F20302934211
:1066400014D97B689B68102B10D17B685B7D5A0343
:106650007B681B6B1A437B689B681A437B681B7FB4
:106660001B04134343F00C03BB610DE07B685B7DAF
:106670005A037B681B6B1A437B689B681A437B68D1
:106680001B7F1B041343BB617B681B7F012B06D15F
:106690007B681B6A013B5B04BA691343BB617B687F
:1066A0005B6A002B09D07B685B6A03F478727B68B5
:1066B0009B6A1343BA691343BB617B681B68DA6842
:1066C0002C4B13407A681268B9690B43D3607B681E
:1066D0001B681846FFF7BCFE38617B681B681846CC
:1066E000FFF7DEFEF8603B69002B5FD1FB68002BF3
:1066F0005CD17B681B7D9A037B68DB6A1343BB61BB
:106700007B681B68DA681C4B13407A681268B969A9
:106710000B43D3607B6893F83830012B30D17B6812
:106720005B6A002B7B681B681A69144B13407A68FC
:10673000D26B013A11047A68126C11437A68526C78
:1067400011437A68926C0A431A437B681B6842F0D3
:1067500001021A611CE000BF48000024632D3E05C1
:106760000020024000210240006002580023024045
:106770000063025803C0F0FFFCBFFFFF1EF800FCDF
:106780007B681B681A697B681B6822F001021A612A
:106790007B681B681B6923F070417B685A6B7B68C0
:1067A0001B680A431A61786800F026FF7B68DB6883
:1067B000012B0CD17B681B681B6B23F00F017B68DE
:1067C0009B695A1E7B681B680A431A6307E07B6853
:1067D0001B681A6B7B681B6822F00F021A637B68C8
:1067E0005B6D23F0030343F001027B685A6507E009
:1067F0007B685B6D43F010027B685A650123FB7771
:10680000FB7F18462437BD4690BD00BF80B586B0DB
:1068100000AF78607B681B685C4A934204D07B6859
:106820001B685B4A934201D15A4B00E05A4B184611
:10683000FFF72EFD38617B681B681846FFF708FEDE
:106840000346002B40F09A807B6893F85030012B70
:1068500001D1022395E07B68012283F850207868FB
:1068600000F0E0FD0346FB75FB7D002B40F08180CE
:106870007B685A6D494B134043F480727B685A65BC
:106880007B681B68424A934202D07B681B6800E029
:106890003E4B7A681268934202D03B69002B05D1C7
:1068A0007B685B6D23F480127B685A657B685B6D47
:1068B00003F48053B3F5805F06D17B689B6D23F0B2
:1068C00006027B689A6502E07B6800229A657B6815
:1068D0001B681C221A607B68002283F850207B68AA
:1068E0001B682B4A934202D07B681B6800E0274B51
:1068F0007A681268934208D03B69002B05D03B6947
:10690000052B02D03B69092B14D17B681B68DB681F
:1069100003F00073002B07D07B685B6D23F44053BA
:1069200043F480527B685A657B681B681846FFF702
:1069300067FD25E07B685B6D43F480127B685A65D8
:106940007B681B68124A934202D07B681B6800E098
:106950000E4BFB60FB68DB6803F00073002B0FD06D
:106960007B685B6D23F4405343F480527B685A6527
:1069700006E07B68002283F8502001E00223FB75CB
:10698000FB7D18461837BD4680BD00BF0020024081
:10699000002102400023024000630258FEF0FFFF86
:1069A00080B584B000AF78607B6893F85030012BDD
:1069B00001D1022321E07B68012283F850200321CA
:1069C000786800F073FC0346FB73FB7B002B0FD150
:1069D000786800F0B1FD0346FB73FB7B002B07D109
:1069E0007B685A6D074B134043F001027B685A6580
:1069F0007B68002283F85020FB7B18461037BD4689
:106A000080BD00BFFEEEFFFF80B588B000AF7860AC
:106A100039607B681B68724A934204D07B681B68AC
:106A2000704A934201D1704B00E0704B1846FFF75B
:106A30002FFC78617B681B69082B02D10823FB615E
:106A400037E07B69002B05D07B69052B02D07B6981
:106A5000092B11D17B681B68DB6803F00103002B55
:106A600007D07B685B6D43F020027B685A65012389
:106A7000B1E00423FB611CE07B681B68584A934229
:106A800004D07B681B68574A934201D1564B00E003
:106A9000564B1846FFF70AFC0346002B07D07B68CD
:106AA0005B6D43F020027B685A65012393E0042369
:106AB000FB61FFF787FA386121E03B68B3F1FF3FE4
:106AC0001DD0FFF77FFA02463B69D31A3A689A4213
:106AD00002D33B68002B12D17B681B681A68FB69E4
:106AE0001340002B0BD17B685B6D43F004027B6885
:106AF0005A657B68002283F8502003236BE07B6893
:106B00001B681A68FB691340002BD6D07B685B6D4D
:106B100043F400727B685A657B681B681846FFF770
:106B200029FB0346002B1CD07B685B7D002B18D112
:106B30007B681B681B6803F00803082B11D17B6876
:106B40005B6D23F480727B685A657B685B6D03F430
:106B50008053002B05D17B685B6D43F001027B689D
:106B60005A657B681B681F4A934202D07B681B688A
:106B700000E01B4B7A681268934208D07B69002BB7
:106B800005D07B69052B02D07B69092B04D17B687A
:106B90001B68DB68BB610CE07B681B68114A934291
:106BA00002D07B681B6800E00D4BFB60FB68DB6874
:106BB000BB61FB69082B04D17B681B6808221A6043
:106BC00008E0BB6903F48043002B03D17B681B689A
:106BD0000C221A60002318462037BD4680BD00BF36
:106BE00000200240002102400023024000630258BE
:106BF00080B483B000AF78607B681B681B6C18465C
:106C00000C37BD465DF8047B7047000090B5A1B01D
:106C100000AF78603960002387F87F300023BB60C5
:106C20003B68DB689D4A93427B6893F85030012BA8
:106C300001D1022321E37B68012283F850207B6885
:106C40001B681846FFF704FC0346002B40F0068340
:106C50003B681B68C3F31303002B08D13B681B6818
:106C60009B0E03F01F03012202FA03F316E03B68B8
:106C70001B687B667B6E93FAA3F33B663B6EBB6639
:106C8000BB6E002B01D1202303E0BB6EB3FA83F36C
:106C9000DBB203F01F03012202FA03F37A681268E1
:106CA000D1697A6812680B43D3617B6818683B68C6
:106CB00059683B681B681A46FFF76FFA7B681B68C8
:106CC0001846FFF7C5FBB8677B681B681846FFF7D7
:106CD000E7FB7867BB6F002B40F0B3807B6F002B26
:106CE00040F0AF807B6818683B6819683B689B6818
:106CF0001A46FFF77EFA6A4B1B6803F07043B3F144
:106D0000805F0BD13B685A697B681B68DB689B0816
:106D100003F007035B0002FA03F31DE07B681B68C6
:106D2000DB6803F01003002B0BD13B685A697B68CA
:106D30001B68DB689B0803F007035B0002FA03F3A0
:106D40000AE03B685A697B681B68DB689B0803F0B4
:106D500004035B0002FA03F33B673B681B69042BE7
:106D600027D07B6818683B6819693B681A683B6FD5
:106D7000FFF7ACF97B6818683B6819693B685B7E74
:106D8000012B02D14FF0004300E000231A46FFF729
:106D9000D6F97B6818683B6819693B681B7E012B34
:106DA00002D14FF4006300E000231A46FFF7AEF96A
:106DB00047E07B681B681B6E03F0F8423B681B686A
:106DC0009B069A4207D17B681B681A6E7B681B681A
:106DD00022F000421A667B681B685B6E03F0F84283
:106DE0003B681B689B069A4207D17B681B685A6EFA
:106DF0007B681B6822F000425A667B681B689B6EAA
:106E000003F0F8423B681B689B069A4207D17B68F7
:106E10001B689A6E7B681B6822F000429A667B684A
:106E20001B68DB6E03F0F8423B681B689B069A42C6
:106E300007D17B681B68DA6E7B681B6822F0004212
:106E4000DA667B681B681846FFF7B4FA0346002B26
:106E500040F00D827B6818683B6819683B68DB6806
:106E60001A46FFF7F1F93B68DB680C4A934240F0A1
:106E700033817B6818683B681B68C3F31303002BDE
:106E800010D13B681B689B0E013303F01F03092BD5
:106E900094BF01230023DBB21EE000BF0000FF47C8
:106EA0000010005C3B681B68BB65BB6D93FAA3F3E5
:106EB0007B657B6DFB65FB6D002B01D1202303E01F
:106EC000FB6DB3FA83F3DBB2013303F01F03092B2D
:106ED00094BF01230023DBB2002B79D03B681B68F1
:106EE000C3F31303002B07D13B681B689B0E0133D0
:106EF0009B0603F0F84215E03B681B68FB64FB6CE3
:106F000093FAA3F3BB64BB6C3B653B6D002B01D1D3
:106F1000202303E03B6DB3FA83F3DBB201339B061E
:106F200003F0F8423B681B68C3F31303002B09D13D
:106F30003B681B689B0E013303F01F03012101FA1C
:106F400003F317E03B681B683B643B6C93FAA3F3C5
:106F5000FB63FB6B7B647B6C002B01D1202303E084
:106F60007B6CB3FA83F3DBB2013303F01F0301211F
:106F700001FA03F342EA03013B681B68C3F31303FE
:106F8000002B0AD13B681B689B0E013303F01F02E4
:106F900013465B0013441B0518E03B681B687B63CA
:106FA0007B6B93FAA3F33B633B6BBB63BB6B002B25
:106FB00001D1202303E0BB6BB3FA83F3DBB20133CF
:106FC00003F01F0213465B0013441B050B437EE0D6
:106FD0003B681B68C3F31303002B07D13B681B6896
:106FE0009B0E01339B0603F0F84215E03B681B68DB
:106FF000BB62BB6A93FAA3F37B627B6AFB62FB6AA8
:10700000002B01D1202303E0FB6AB3FA83F3DBB248
:1070100001339B0603F0F8423B681B68C3F313037C
:10702000002B09D13B681B689B0E013303F01F0343
:10703000012101FA03F317E03B681B68FB61FB6960
:1070400093FAA3F3BB61BB693B623B6A002B01D19E
:10705000202303E03B6AB3FA83F3DBB2013303F08E
:107060001F03012101FA03F342EA03013B681B6895
:10707000C3F31303002B0DD13B681B689B0E013338
:1070800003F01F0213465B0013441E3B1B0543F035
:1070900000731BE03B681B683B613B6993FAA3F3F9
:1070A000FB60FB687B617B69002B01D1202303E03F
:1070B0007B69B3FA83F3DBB2013303F01F0213469B
:1070C0005B0013441E3B1B0543F000730B433A68FF
:1070D00092681946FFF78DF83B681B68002B80F219
:1070E000C6807B681B68674A934204D07B681B6834
:1070F000654A934201D1654B00E0654B1846FEF7A7
:10710000D7FFF8667B681B685E4A934204D07B68B1
:107110001B685D4A93420ED15A48FFF74BF904466B
:107120005948FFF747F903462343002B0CBF0123BF
:107130000023DBB208E05748FFF73CF90346002B79
:107140000CBF01230023DBB2002B7DD03B681B6802
:10715000514A934230D1FB6E03F40003002B2BD134
:107160007B681B684B4A934240F081807B681B68B8
:10717000444A934204D07B681B68434A934201D13E
:10718000424A00E0424AFB6E43F4000319461046AF
:10719000FEF77BFF414B1B689B09414AA2FB03237F
:1071A0009B0901335B00BB6002E0BB68013BBB6035
:1071B000BB68002BF9D15AE03B681B68394A9342FF
:1071C0001ED1FB6E03F08073002B19D17B681B6806
:1071D000304A93424BD17B681B682A4A934204D0C1
:1071E0007B681B68284A934201D1284A00E0284A5C
:1071F000FB6E43F0807319461046FEF746FF36E0FB
:107200003B681B68284A934231D1FB6E03F480032C
:10721000002B2CD17B681B681E4A934227D17B68C8
:107220001B68184A934204D07B681B68164A934235
:1072300001D1164A00E0164AFB6E43F4800319465A
:107240001046FEF722FF12E07B685B6D43F02002E0
:107250007B685A65012387F87F3008E07B685B6DA7
:1072600043F020027B685A65012387F87F307B68F2
:10727000002283F8502097F87F3018468437BD46A7
:1072800090BD00BF002002400021024000230240C8
:107290000063025800600258000084CB48000024BC
:1072A000632D3E05000052C70000B8CF80B588B0FE
:1072B00000AF786039600023FB613B68BB617B688D
:1072C0001B681846FFF7C4F838617B681B681846CE
:1072D000FFF7E6F8F8603B69002B03D1FB68002B51
:1072E00000F098807B681B68DB6803F00073002B5C
:1072F0002AD07B685B7D012B26D17B681B7D012B0F
:1073000022D10123BB6114E0FB69454A93420DD9A8
:107310007B685B6D43F010027B685A657B689B6DF0
:1073200043F001027B689A65012374E0FB69013335
:10733000FB617B681B681B6803F04003402BE3D1B3
:107340007B681B6840221A60BB69022B14D07B68E3
:107350001B681846FFF77CF80346002B0CD07B68AF
:107360001B681846FFF739F80346002B04D17B68E9
:107370001B681846FFF758F8BB69012B14D07B68CF
:107380001B681846FFF78CF80346002B0CD07B686F
:107390001B681846FFF721F80346002B04D17B68D1
:1073A0001B681846FFF768F8BB69022B05D0BB695C
:1073B000032B05D10C237B6105E008237B6102E0F0
:1073C00004237B6100BFFEF7FDFDB8601BE0FEF704
:1073D000F9FD0246BB68D31A052B14D97B681B68DC
:1073E0009A687B691340002B0DD07B685B6D43F07E
:1073F00010027B685A657B689B6D43F001027B68D5
:107400009A65012307E07B681B689A687B691340D3
:10741000002BDCD1002318462037BD4680BD00BFBD
:10742000FFDB0C0080B584B000AF78607B681B6820
:107430001846FEF7BFFF0346002B6ED17B681B6822
:107440009A68384B1340002B0DD07B685B6D43F07E
:1074500010027B685A657B689B6D43F001027B6874
:107460009A6501235AE07B681B681846FEF77AFF8D
:10747000FEF7A8FDF8607B681B682B4A934204D096
:107480007B681B68294A934201D1294B00E0294BB4
:107490001846FEF7FDFEB8607B681B68234A9342DE
:1074A00002D07B681B6800E01F4B7A681268934229
:1074B0002CD0BB68002B30D128E07B681B681846B5
:1074C000FEF778FF0346002B04D17B681B68184643
:1074D000FEF748FFFEF776FD0246FB68D31A022B43
:1074E00014D97B681B681B6803F00103012B0DD0C6
:1074F0007B685B6D43F010027B685A657B689B6D0F
:1075000043F001027B689A65012307E07B681B68F2
:107510001B6803F00103012BCFD10023184610375D
:10752000BD4680BD3F000080002002400021024097
:10753000002302400063025880B584B000AF786039
:107540007B681B681846FEF748FFF8607B681B687D
:107550001846FEF72FFF0346002B47D0FB68002B91
:1075600044D17B681B689B6803F00D03012B0CD191
:107570007B681B681846FEF709FF7B681B680322BF
:107580001A60FEF71FFDB86029E07B685B6D43F071
:1075900010027B685A657B689B6D43F001027B6833
:1075A0009A65012323E0FEF70DFD0246BB68D31A5E
:1075B000022B14D97B681B689B6803F00103002B26
:1075C0000DD07B685B6D43F010027B685A657B6869
:1075D0009B6D43F001027B689A65012307E07B689D
:1075E0001B689B6803F00103002BDCD100231846C5
:1075F0001037BD4680BD000080B584B000AF786014
:107600007B681B68794A934204D07B681B68784A80
:10761000934209D1774B9B6803F44033002B14BF8E
:1076200001230023DBB208E0734B9B6803F4403373
:10763000002B14BF01230023DBB2002B1CD008F069
:107640005BFBF8607B685B68B3F5403F10D0B3F537
:10765000403F71D8B3F5803F02D0B3F5003F6BD106
:107660007B685B681B0CFA68B2FBF3F3FB6066E0B7
:10767000FB689B08FB6062E04FF4002009F0DEFA33
:10768000F8607B685B68B3F5301F51D0B3F5301FED
:1076900054D8B3F5201F47D0B3F5201F4ED8B3F50B
:1076A000101F3DD0B3F5101F48D8B3F5001F33D0DD
:1076B000B3F5001F42D8B3F5E01F29D0B3F5E01FA2
:1076C0003CD8B3F5C01F1AD0B3F5C01F36D8B3F5F8
:1076D000A01F14D0B3F5A01F30D8B3F5801F0ED073
:1076E000B3F5801F2AD8B3F5402F08D0B3F5402F4B
:1076F00024D8B3F5802F02D0B3F5002F1ED17B68BC
:107700005B689B0C5B00FA68B2FBF3F3FB6016E06E
:10771000FB681B09FB6012E0FB685B09FB600EE085
:10772000FB689B09FB600AE0FB68DB09FB6006E085
:10773000FB681B0AFB6002E000BF00E000BFFEF731
:1077400071FC034641F20302934215D8FB682B4AB1
:10775000934208D97B681B689A687B681B6842F46F
:1077600080729A603EE07B681B689A687B681B6841
:1077700022F480729A6035E0FB685B08FB60FB686E
:107780001F4A934208D87B681B689A687B681B680D
:1077900022F440729A6025E0FB681A4A93420AD8A4
:1077A0007B681B689B6823F440727B681B6842F40B
:1077B00080729A6016E0FB68134A93420AD87B688D
:1077C0001B689B6823F440727B681B6842F400725C
:1077D0009A6007E07B681B689A687B681B6842F4C4
:1077E00040729A6000BF1037BD4680BD0020024045
:1077F000002102400023024000630258002D3101A5
:10780000105E5F0020BCBE0040787D0180B485B072
:1078100000AF78607B6803F00703FB600B4BDB680D
:10782000BB60BA684FF6FF031340BB60FB681A02E7
:10783000BB681A43064B1343BB60044ABB68D36062
:1078400000BF1437BD465DF8047B704700ED00E0D3
:107850000000FA0580B400AF044BDB681B0A03F09C
:1078600007031846BD465DF8047B704700ED00E055
:1078700080B483B000AF0346FB80B7F90630002B1D
:107880000BDBFB8803F01F020749B7F906305B09E1
:10789000012000FA02F241F8232000BF0C37BD4658
:1078A0005DF8047B704700BF00E100E080B483B066
:1078B00000AF03463960FB80B7F90630002B0ADBC6
:1078C0003B68DAB20C49B7F906301201D2B20B4468
:1078D00083F800230AE03B68DAB20849FB8803F02A
:1078E0000F03043B1201D2B20B441A7600BF0C37CF
:1078F000BD465DF8047B704700E100E000ED00E06C
:1079000080B489B000AFF860B9607A60FB6803F0BA
:107910000703FB61FB69C3F10703042B28BF0423A2
:10792000BB61FB690433062B02D9FB69033B00E012
:1079300000237B614FF0FF32BB6902FA03F3DA43A5
:10794000BB681A407B699A404FF0FF317B6901FAAE
:1079500003F3D9437B680B40134318462437BD46D5
:107960005DF8047B7047000080B582B000AF78609E
:107970007B68013BB3F1807F01D301230FE00A4A0A
:107980007B68013B53600F214FF0FF30FFF78EFF04
:10799000054B00229A60044B07221A600023184608
:1079A0000837BD4680BD00BF10E000E080B582B062
:1079B00000AF78607868FFF729FF00BF0837BD4641
:1079C00080BD80B586B000AF0346B9607A60FB81A8
:1079D000FFF740FF78617A68B9687869FFF790FF30
:1079E0000246B7F90E3011461846FFF75FFF00BF99
:1079F0001837BD4680BD80B582B000AF0346FB801E
:107A0000B7F906301846FFF733FF00BF0837BD4609
:107A100080BD80B582B000AF78607868FFF7A4FFC2
:107A2000034618460837BD4680BD000080B400AF4D
:107A3000BFF35F8F00BF074B5B6A064A23F48033B6
:107A40005362054B00225A6000BFBD465DF8047BBF
:107A5000704700BF00ED00E090ED00E080B483B01F
:107A600000AF78600B4A7B6843F0010353600A4B18
:107A70005B6A094A43F480335362BFF34F8F00BF00
:107A8000BFF36F8F00BF00BF0C37BD465DF8047BAE
:107A9000704700BF90ED00E000ED00E080B483B0DF
:107AA00000AF78607B685A781D4B9A607B681B78C2
:107AB000002B29D01A4A7B685B68D3607B681B7BEC
:107AC0001A077B68DB7A1B061A437B689B7ADB0408
:107AD0001A437B685B7B9B041A437B689B7B5B043C
:107AE0001A437B68DB7B1B041A437B685B7A1B02AF
:107AF0001A437B681B7A5B0013437A68127811463D
:107B0000074A0B43136105E0054B0022DA60044B82
:107B100000221A6100BF0C37BD465DF8047B704738
:107B200090ED00E080B586B000AF7860FEF74AFACD
:107B300038617B68002B01D1012316E37B681B6849
:107B4000664A93424AD07B681B68654A934245D097
:107B50007B681B68634A934240D07B681B68624A1B
:107B600093423BD07B681B68604A934236D07B6867
:107B70001B685F4A934231D07B681B685D4A934221
:107B80002CD07B681B685C4A934227D07B681B68BB
:107B90005A4A934222D07B681B68594A93421DD0AF
:107BA0007B681B68574A934218D07B681B68564A0B
:107BB000934213D07B681B68544A93420ED07B6873
:107BC0001B68534A934209D07B681B68514A934211
:107BD00004D07B681B68504A934201D1012300E026
:107BE0000023002B00F03B817B68022283F83520C4
:107BF0007B68002283F834207B681B68374A9342F5
:107C00004AD07B681B68364A934245D07B681B6824
:107C1000344A934240D07B681B68334A93423BD03E
:107C20007B681B68314A934236D07B681B68304AB8
:107C3000934231D07B681B682E4A93422CD07B68DC
:107C40001B682D4A934227D07B681B682B4A9342BE
:107C500022D07B681B682A4A93421DD07B681B6830
:107C6000284A934218D07B681B68274A934213D056
:107C70007B681B68254A93420ED07B681B68244AA8
:107C8000934209D07B681B68224A934204D07B68E8
:107C90001B68214A934208D17B681B681A687B687D
:107CA0001B6822F001021A6007E07B681B681A68F3
:107CB0007B681B6822F001021A602FE0FEF782F950
:107CC00002463B69D31A052B28D97B6820225A65C6
:107CD0007B68032283F83520012346E2100002402E
:107CE000280002404000024058000240700002405C
:107CF00088000240A0000240B80002401004024088
:107D0000280402404004024058040240700402402B
:107D100088040240A0040240B80402407B681B684B
:107D20001B6803F00103002BC8D17B681B681B682C
:107D30007B617A69834B13407B617B689A687B68BF
:107D4000DB681A437B681B691A437B685B691A43CB
:107D50007B689B691A437B68DB691A437B681B6AF3
:107D600013437A6913437B617B685B6A042B07D1F9
:107D70007B68DA6A7B681B6B13437A6913437B6108
:107D8000714B1A68714B1340B3F1005F28D37B68C5
:107D90005B68282B03D97B685B682E2B17D97B681F
:107DA0005B683E2B03D97B685B68422B0FD97B68ED
:107DB0005B68462B03D97B685B68482B07D97B68D7
:107DC0005B684E2B05D97B685B68522B01D8012379
:107DD00000E00023002B03D07B6943F480137B6118
:107DE0007B681B687A691A607B681B685B697B61CA
:107DF0007B6923F007037B617B685B6A7A691343C5
:107E00007B617B685B6A042B17D17B689B6A7A690C
:107E100013437B617B68DB6A002B0ED0786802F02D
:107E200041FB0346002B08D07B6840225A657B68E3
:107E3000012283F83520012397E17B681B687A696A
:107E40005A61786802F07CFA0346BB607B68DB6DA0
:107E500003F01F033F229A40BB689A60CDE07B6825
:107E60001B683B4A934222D07B681B68394A934285
:107E70001DD07B681B68384A934218D07B681B680A
:107E8000364A934213D07B681B68354A93420ED022
:107E90007B681B68334A934209D07B681B68324A6F
:107EA000934204D07B681B68304A934201D101237E
:107EB00000E00023002B00F097807B681B68244AB9
:107EC000934221D07B681B68224A93421CD07B6876
:107ED0001B68214A934217D07B681B681F4A934254
:107EE00012D07B681B681E4A93420DD07B681B68CA
:107EF0001C4A934208D07B681B681B4A934203D0FC
:107F00007B681B68194A934200BF7B68022283F892
:107F100035207B68002283F834207B681B681B684F
:107F20007B617A69124B13407B617B689B68402BB5
:107F300020D07B689B68802B02D14FF480431AE0ED
:107F4000002318E03F8010FE0010005C0000FFFFDF
:107F5000085402581C5402583054025844540258D1
:107F6000585402586C540258805402589454025881
:107F70000F00FEFF10237A68D268D2081A437B688C
:107F80001B69DB081A437B685B69DB081A437B6863
:107F90009B69DB081A437B68DB69DB081A437B6853
:107FA0001B6A1B0913437A6913437B617B681B6857
:107FB0007A691A607B681B681A466E4B13446E4AD6
:107FC000A2FB03231B099A007B68DA65786802F03C
:107FD000B7F90346FB607B68DB6D03F01F030122EA
:107FE0009A40FB685A6008E07B6840225A657B68CB
:107FF000032283F835200123B7E07B681B685F4AC2
:10800000934272D07B681B685D4A93426DD07B6857
:108010001B685C4A934268D07B681B685A4A93424B
:1080200063D07B681B68594A93425ED07B681B68AB
:10803000574A934259D07B681B68564A934254D0A2
:108040007B681B68544A93424FD07B681B68534A35
:1080500093424AD07B681B68514A934245D07B6863
:108060001B68504A934240D07B681B684E4A93423B
:108070003BD07B681B684D4A934236D07B681B68B7
:108080004B4A934231D07B681B684A4A93422CD0BA
:108090007B681B68484A934227D07B681B68474A25
:1080A000934222D07B681B68454A93421DD07B686F
:1080B0001B68444A934218D07B681B68424A93422B
:1080C00013D07B681B68414A93420ED07B681B68C3
:1080D0003F4A934209D07B681B683E4A934204D0D2
:1080E0007B681B683C4A934201D1012300E00023D6
:1080F000002B32D0786802F051FA7B689B68802BA5
:1081000002D17B6800225A607B685A687B681B6ECC
:10811000D2B21A607B685B6E7A68926E5A607B6836
:108120005B68002B10D07B685B68082B0CD87868E4
:1081300002F0CEFA7B68DB6E00221A607B681B6F50
:108140007A68526F5A6008E07B680022DA667B68C2
:1081500000221A677B6800225A677B6800225A65F2
:108160007B68012283F83520002318461837BD4666
:1081700080BD00BFF8ABFDA7CDCCCCCC1000024039
:1081800028000240400002405800024070000240B7
:1081900088000240A0000240B800024010040240E3
:1081A0002804024040040240580402407004024087
:1081B00088040240A0040240B80402400854025857
:1081C0001C5402583054025844540258585402580F
:1081D0006C540258805402589454025880B586B0AA
:1081E00000AFF860B9607A603B600023FB75FB6804
:1081F000002B01D1012326E2FB6893F83430012BD8
:1082000001D102231FE2FB68012283F83420FB68BE
:1082100093F83530DBB2012B40F00A82FB68022272
:1082200083F83520FB6800225A65FB681B68684AA2
:1082300093424AD0FB681B68664A934245D0FB686C
:108240001B68654A934240D0FB681B68634A9342AF
:108250003BD0FB681B68624A934236D0FB681B68C0
:10826000604A934231D0FB681B685F4A93422CD02E
:10827000FB681B685D4A934227D0FB681B685C4A19
:10828000934222D0FB681B685A4A93421DD0FB6878
:108290001B68594A934218D0FB681B68574A93429F
:1082A00013D0FB681B68564A93420ED0FB681B68CC
:1082B000544A934209D0FB681B68534A934204D046
:1082C000FB681B68514A934208D1FB681B681A6817
:1082D000FB681B6822F001021A6007E0FB681B685C
:1082E0001A68FB681B6822F001021A603B687A6812
:1082F000B968F86801F078FEFB681B68344A93425D
:108300004AD0FB681B68334A934245D0FB681B6820
:10831000314A934240D0FB681B68304A93423BD0BD
:10832000FB681B682E4A934236D0FB681B682D4AB7
:10833000934231D0FB681B682B4A93422CD0FB68D8
:108340001B682A4A934227D0FB681B68284A93423D
:1083500022D0FB681B68274A93421DD0FB681B682C
:10836000254A934218D0FB681B68244A934213D0D5
:10837000FB681B68224A93420ED0FB681B68214AA7
:10838000934209D0FB681B681F4A934204D0FB68E4
:108390001B681E4A934201D1012300E00023002BF9
:1083A00036D0FB681B681B6823F01E02FB681B6845
:1083B00042F016021A60FB681B6C002B3ED0FB6873
:1083C0001B681A68FB681B6842F008021A6035E0F7
:1083D00010000240280002404000024058000240C5
:1083E0007000024088000240A0000240B800024035
:1083F0001004024028040240400402405804024095
:108400007004024088040240A0040240B804024004
:10841000FB681B681B6823F00E02FB681B6842F0B8
:108420000A021A60FB681B6C002B07D0FB681B68F4
:108430001A68FB681B6842F004021A60FB681B683C
:10844000834A934272D0FB681B68824A93426DD084
:10845000FB681B68804A934268D0FB681B687F4AB0
:10846000934263D0FB681B687D4A93425ED0FB68F1
:108470001B687C4A934259D0FB681B687A4A934236
:1084800054D0FB681B68794A93424FD0FB681B6845
:10849000774A93424AD0FB681B68764A934245D09C
:1084A000FB681B68744A934240D0FB681B68734AA0
:1084B00093423BD0FB681B68714A934236D0FB68FD
:1084C0001B68704A934231D0FB681B686E4A934226
:1084D0002CD0FB681B686D4A934227D0FB681B6851
:1084E0006B4A934222D0FB681B686A4A93421DD0B4
:1084F000FB681B68684A934218D0FB681B68674A90
:10850000934213D0FB681B68654A93420ED0FB6808
:108510001B68644A934209D0FB681B68624A934215
:1085200004D0FB681B68614A934201D1012300E03B
:108530000023002B1AD0FB681B6E1B6803F48033EA
:10854000002B07D0FB681B6E1A68FB681B6E42F499
:1085500080721A60FB68DB6E002B07D0FB68DB6E55
:108560001A68FB68DB6E42F480721A60FB681B6855
:10857000374A93424AD0FB681B68364A934245D03B
:10858000FB681B68344A934240D0FB681B68334A3F
:1085900093423BD0FB681B68314A934236D0FB685C
:1085A0001B68304A934231D0FB681B682E4A9342C5
:1085B0002CD0FB681B682D4A934227D0FB681B68B0
:1085C0002B4A934222D0FB681B682A4A93421DD053
:1085D000FB681B68284A934218D0FB681B68274A2F
:1085E000934213D0FB681B68254A93420ED0FB6868
:1085F0001B68244A934209D0FB681B68224A9342B5
:1086000004D0FB681B68214A934208D1FB681B68B1
:108610001A68FB681B6842F001021A6012E0FB68EE
:108620001B681A68FB681B6842F001021A6009E0C7
:10863000FB684FF400625A65FB68002283F834201F
:108640000123FB75FB7D18461837BD4680BD00BF72
:108650001000024028000240400002405800024042
:108660007000024088000240A0000240B8000240B2
:108670001004024028040240400402405804024012
:108680007004024088040240A0040240B804024082
:10869000085402581C54025830540258445402588A
:1086A000585402586C54025880540258945402583A
:1086B00080B586B000AF7860FDF784FC38617B68D8
:1086C000002B01D10123DCE27B6893F83530DBB26B
:1086D000022B08D07B6880225A657B68002283F8D1
:1086E00034200123CDE27B681B68764A93424AD04E
:1086F0007B681B68744A934245D07B681B68734A49
:10870000934240D07B681B68714A93423BD07B68A0
:108710001B68704A934236D07B681B686E4A93424E
:1087200031D07B681B686D4A93422CD07B681B68F4
:108730006B4A934227D07B681B686A4A934222D0D7
:108740007B681B68684A93421DD07B681B68674A38
:10875000934218D07B681B68654A934213D07B68AC
:108760001B68644A93420ED07B681B68624A93423E
:1087700009D07B681B68614A934204D07B681B6800
:108780005F4A934201D1012300E00023002B13D064
:108790007B681B681A687B681B6822F01E021A60DF
:1087A0007B681B685A697B681B6822F080025A61EB
:1087B0007B681B687B610AE07B681B681A687B68C2
:1087C0001B6822F00E021A607B681B687B617B6865
:1087D0001B683C4A934272D07B681B683A4A9342BA
:1087E0006DD07B681B68394A934268D07B681B68F0
:1087F000374A934263D07B681B68364A93425ED007
:108800007B681B68344A934259D07B681B68334AA3
:10881000934254D07B681B68314A93424FD07B68A7
:108820001B68304A93424AD07B681B682E4A9342A9
:1088300045D07B681B682D4A934240D07B681B68FB
:108840002B4A93423BD07B681B682A4A934236D01E
:108850007B681B68284A934231D07B681B68274A93
:1088600093422CD07B681B68254A934227D07B68B3
:108870001B68244A934222D07B681B68224A934299
:108880001DD07B681B68214A934218D07B681B6807
:108890001F4A934213D07B681B681E4A93420ED036
:1088A0007B681B681C4A934209D07B681B681B4A83
:1088B000934204D07B681B68194A934232D101234A
:1088C00031E000BF1000024028000240400002409A
:1088D000580002407000024088000240A0000240A0
:1088E000B800024010040240280402404004024044
:1088F000580402407004024088040240A004024070
:10890000B8040240085402581C540258305402580B
:1089100044540258585402586C5402588054025817
:10892000945402580023002B07D07B681B6E1A68F2
:108930007B681B6E22F480721A607B681B686D4A2C
:1089400093424AD07B681B686B4A934245D07B6850
:108950001B686A4A934240D07B681B68684A93420E
:108960003BD07B681B68674A934236D07B681B68A4
:10897000654A934231D07B681B68644A93422CD08D
:108980007B681B68624A934227D07B681B68614AF8
:10899000934222D07B681B685F4A93421DD07B685C
:1089A0001B685E4A934218D07B681B685C4A9342FE
:1089B00013D07B681B685B4A93420ED07B681B68B0
:1089C000594A934209D07B681B68584A934204D0A5
:1089D0007B681B68564A934208D17B681B681A68FB
:1089E0007B681B6822F001021A6007E07B681B6845
:1089F0001A687B681B6822F001021A6013E0FDF719
:108A0000E1FA02463B69D31A052B0CD97B68202278
:108A10005A657B68032283F835207B68002283F83F
:108A2000342001232DE17B691B6803F00103002B37
:108A3000E5D17B681B682F4A93424AD07B681B684C
:108A40002D4A934245D07B681B682C4A934240D004
:108A50007B681B682A4A93423BD07B681B68294A83
:108A6000934236D07B681B68274A934231D07B689B
:108A70001B68264A93422CD07B681B68244A934289
:108A800027D07B681B68234A934222D07B681B68EF
:108A9000214A93421DD07B681B68204A934218D01C
:108AA0007B681B681E4A934213D07B681B681D4A73
:108AB00093420ED07B681B681B4A934209D07B68A7
:108AC0001B681A4A934204D07B681B68184A934279
:108AD00001D1012300E00023002B2BD07B689B6D8C
:108AE000BB607B68DB6D03F01F033F229A40BB68CD
:108AF0009A602AE010000240280002404000024034
:108B0000580002407000024088000240A00002406D
:108B1000B800024010040240280402404004024011
:108B2000580402407004024088040240A00402403D
:108B3000B80402407B689B6DFB607B68DB6D03F0D3
:108B40001F0301229A40FB685A607B681B684F4AEA
:108B5000934272D07B681B684D4A93426DD07B680C
:108B60001B684C4A934268D07B681B684A4A934210
:108B700063D07B681B68494A93425ED07B681B6860
:108B8000474A934259D07B681B68464A934254D067
:108B90007B681B68444A93424FD07B681B68434AFA
:108BA00093424AD07B681B68414A934245D07B6818
:108BB0001B68404A934240D07B681B683E4A934200
:108BC0003BD07B681B683D4A934236D07B681B686C
:108BD0003B4A934231D07B681B683A4A93422CD07F
:108BE0007B681B68384A934227D07B681B68374AEA
:108BF000934222D07B681B68354A93421DD07B6824
:108C00001B68344A934218D07B681B68324A9342EF
:108C100013D07B681B68314A93420ED07B681B6877
:108C20002F4A934209D07B681B682E4A934204D096
:108C30007B681B682C4A934201D1012300E000238A
:108C4000002B15D07B685B6E7A68926E5A607B68E9
:108C5000DB6E002B0CD07B68DB6E1A687B68DB6EEA
:108C600022F480721A607B681B6F7A68526F5A60B8
:108C70007B68012283F835207B68002283F834204A
:108C8000002318461837BD4680BD00BF10000240C3
:108C9000280002404000024058000240700002409C
:108CA00088000240A0000240B800024010040240C8
:108CB000280402404004024058040240700402406C
:108CC00088040240A0040240B8040240085402583C
:108CD0001C540258305402584454025858540258F4
:108CE0006C540258805402589454025880B584B091
:108CF00000AF78607B68002B01D1012337E27B68ED
:108D000093F83530DBB2022B04D07B6880225A65A1
:108D100001232CE27B681B685C4A93424AD07B6843
:108D20001B685B4A934245D07B681B68594A934253
:108D300040D07B681B68584A93423BD07B681B68D5
:108D4000564A934236D07B681B68554A934231D0CD
:108D50007B681B68534A93422CD07B681B68524A3D
:108D6000934227D07B681B68504A934222D07B688D
:108D70001B684F4A93421DD07B681B684D4A934243
:108D800018D07B681B684C4A934213D07B681B68E1
:108D90004A4A93420ED07B681B68494A934209D0E5
:108DA0007B681B68474A934204D07B681B68464A2D
:108DB000934201D1012300E00023002B00F08680C4
:108DC0007B68042283F835207B681B682F4A934216
:108DD0004AD07B681B682E4A934245D07B681B684B
:108DE0002C4A934240D07B681B682B4A93423BD06D
:108DF0007B681B68294A934236D07B681B68284AE7
:108E0000934231D07B681B68264A93422CD07B6802
:108E10001B68254A934227D07B681B68234A9342EC
:108E200022D07B681B68224A93421DD07B681B6856
:108E3000204A934218D07B681B681F4A934213D084
:108E40007B681B681D4A93420ED07B681B681C4AD6
:108E5000934209D07B681B681A4A934204D07B680E
:108E60001B68194A934208D17B681B681A687B68A3
:108E70001B6822F001021A6078E17B681B681A689F
:108E80007B681B6822F001021A606FE1100002404B
:108E9000280002404000024058000240700002409A
:108EA00088000240A0000240B800024010040240C6
:108EB000280402404004024058040240700402406A
:108EC00088040240A0040240B80402407B681B688A
:108ED0001A687B681B6822F00E021A607B681B68A8
:108EE0006C4A93424AD07B681B686B4A934245D0D8
:108EF0007B681B68694A934240D07B681B68684A5C
:108F000093423BD07B681B68664A934236D07B68AD
:108F10001B68654A934231D07B681B68634A934261
:108F20002CD07B681B68624A934227D07B681B6801
:108F3000604A934222D07B681B685F4A93421DD0EF
:108F40007B681B685D4A934218D07B681B685C4A4B
:108F5000934213D07B681B685A4A93420ED07B68B9
:108F60001B68594A934209D07B681B68574A934251
:108F700004D07B681B68564A934208D17B681B6803
:108F80001A687B681B6822F001021A6007E07B68A0
:108F90001B681A687B681B6822F001021A607B68F4
:108FA0001B683C4A934272D07B681B683A4A9342E2
:108FB0006DD07B681B68394A934268D07B681B6818
:108FC000374A934263D07B681B68364A93425ED02F
:108FD0007B681B68344A934259D07B681B68334ACC
:108FE000934254D07B681B68314A93424FD07B68D0
:108FF0001B68304A93424AD07B681B682E4A9342D2
:1090000045D07B681B682D4A934240D07B681B6823
:109010002B4A93423BD07B681B682A4A934236D046
:109020007B681B68284A934231D07B681B68274ABB
:1090300093422CD07B681B68254A934227D07B68DB
:109040001B68244A934222D07B681B68224A9342C1
:109050001DD07B681B68214A934218D07B681B682F
:109060001F4A934213D07B681B681E4A93420ED05E
:109070007B681B681C4A934209D07B681B681B4AAB
:10908000934204D07B681B68194A934232D1012372
:1090900031E000BF100002402800024040000240C2
:1090A000580002407000024088000240A0000240C8
:1090B000B80002401004024028040240400402406C
:1090C000580402407004024088040240A004024098
:1090D000B8040240085402581C5402583054025834
:1090E00044540258585402586C5402588054025840
:1090F000945402580023002B28D07B681B6E1A68FA
:109100007B681B6E22F480721A607B689B6DFB602B
:109110007B68DB6D03F01F0301229A40FB685A60F5
:109120007B685B6E7A68926E5A607B68DB6E002BA0
:109130000CD07B68DB6E1A687B68DB6E22F4807271
:109140001A607B681B6F7A68526F5A607B680122D5
:1091500083F835207B68002283F834207B681B6D00
:10916000002B03D07B681B6D786898470023184656
:109170001037BD4680BD00BF80B58AB000AF7860B3
:109180000023FB60674B1B68674AA2FB03239B0A13
:109190007B627B689B6D3B627B689B6DFB613B6A7E
:1091A0001B68BB61FB691B687B617B681B685F4A4E
:1091B00093424AD07B681B685D4A934245D07B68E6
:1091C0001B685C4A934240D07B681B685A4A9342B2
:1091D0003BD07B681B68594A934236D07B681B683A
:1091E000574A934231D07B681B68564A93422CD031
:1091F0007B681B68544A934227D07B681B68534A9C
:10920000934222D07B681B68514A93421DD07B68F1
:109210001B68504A934218D07B681B684E4A9342A1
:1092200013D07B681B684D4A93420ED07B681B6845
:109230004B4A934209D07B681B684A4A934204D048
:109240007B681B68484A934201D1012300E0002358
:10925000002B00F02B847B68DB6D03F01F030822DA
:109260009A40BB691340002B00F0A2807B681B680A
:109270002E4A93424AD07B681B682D4A934245D0C0
:109280007B681B682B4A934240D07B681B682A4A44
:1092900093423BD07B681B68284A934236D07B6858
:1092A0001B68274A934231D07B681B68254A93424A
:1092B0002CD07B681B68244A934227D07B681B68AC
:1092C000224A934222D07B681B68214A93421DD0D8
:1092D0007B681B681F4A934218D07B681B681E4A34
:1092E000934213D07B681B681C4A93420ED07B6864
:1092F0001B681B4A934209D07B681B68194A93423A
:1093000004D07B681B68184A93422FD17B681B6886
:109310001B6803F00403002B14BF01230023DBB2FE
:109320002EE000BF48000024B5814E1B1000024013
:1093300028000240400002405800024070000240F5
:1093400088000240A0000240B80002401004024021
:1093500028040240400402405804024070040240C5
:1093600088040240A0040240B80402407B681B68E5
:109370001B6803F00803002B14BF01230023DBB29A
:10938000002B15D07B681B681A687B681B6822F06D
:1093900004021A607B68DB6D03F01F0308229A4009
:1093A0003B6A9A607B685B6D43F001027B685A659B
:1093B0007B68DB6D03F01F03BA6922FA03F303F045
:1093C0000103002B6ED07B681B68694A93424AD028
:1093D0007B681B68674A934245D07B681B68664A76
:1093E000934240D07B681B68644A93423BD07B68C1
:1093F0001B68634A934236D07B681B68614A93427C
:1094000031D07B681B68604A93422CD07B681B6814
:109410005E4A934227D07B681B685D4A934222D004
:109420007B681B685B4A93421DD07B681B685A4A65
:10943000934218D07B681B68584A934213D07B68CC
:109440001B68574A93420ED07B681B68554A93426B
:1094500009D07B681B68544A934204D07B681B6820
:10946000524A93420AD17B681B685B6903F0800310
:10947000002B14BF01230023DBB203E07B681B68D1
:109480001B680023002B0DD07B68DB6D03F01F03EE
:1094900001229A403B6A9A607B685B6D43F002024E
:1094A0007B685A657B68DB6D03F01F0304229A40DA
:1094B000BB691340002B00F08F807B681B682C4A2F
:1094C00093424AD07B681B682A4A934245D07B6806
:1094D0001B68294A934240D07B681B68274A934205
:1094E0003BD07B681B68264A934236D07B681B685A
:1094F000244A934231D07B681B68234A93422CD084
:109500007B681B68214A934227D07B681B68204AEE
:10951000934222D07B681B681E4A93421DD07B6811
:109520001B681D4A934218D07B681B681B4A9342F4
:1095300013D07B681B681A4A93420ED07B681B6865
:10954000184A934209D07B681B68174A934204D09B
:109550007B681B68154A93422AD17B681B681B688D
:1095600003F00203002B14BF01230023DBB223E02E
:109570001000024028000240400002405800024013
:109580007000024088000240A0000240B800024083
:1095900010040240280402404004024058040240E3
:1095A0007004024088040240A0040240B804024053
:1095B0007B681B681B680023002B0DD07B68DB6D6C
:1095C00003F01F0304229A403B6A9A607B685B6D3C
:1095D00043F004027B685A657B68DB6D03F01F0370
:1095E00010229A40BB691340002B00F0A6807B68D4
:1095F0001B68854A93424AD07B681B68834A934222
:1096000045D07B681B68824A934240D07B681B68C8
:10961000804A93423BD07B681B687F4A934236D096
:109620007B681B687D4A934231D07B681B687C4A0B
:1096300093422CD07B681B687A4A934227D07B6880
:109640001B68794A934222D07B681B68774A934211
:109650001DD07B681B68764A934218D07B681B68D4
:10966000744A934213D07B681B68734A93420ED0AE
:109670007B681B68714A934209D07B681B68704AFB
:10968000934204D07B681B686E4A93420AD17B6880
:109690001B681B6803F00803002B14BF0123002381
:1096A000DBB209E07B681B681B6803F00403002B36
:1096B00014BF01230023DBB2002B3ED07B68DB6D9F
:1096C00003F01F0310229A403B6A9A607B681B6874
:1096D0001B6803F48023002B18D07B681B681B6871
:1096E00003F40023002B08D17B681B6C002B24D0D3
:1096F0007B681B6C786898471FE07B689B6C002B2D
:109700001BD07B689B6C7868984716E07B681B6869
:109710001B6803F48073002B07D17B681B681A68F1
:109720007B681B6822F008021A607B681B6C002BA8
:1097300003D07B681B6C786898477B68DB6D03F00F
:109740001F0320229A40BB691340002B00F01081B8
:109750007B681B682C4A93424AD07B681B682B4A63
:10976000934245D07B681B68294A934240D07B686E
:109770001B68284A93423BD07B681B68264A934269
:1097800036D07B681B68254A934231D07B681B68C2
:10979000234A93422CD07B681B68224A934227D0ED
:1097A0007B681B68204A934222D07B681B681F4A53
:1097B00093421DD07B681B681D4A934218D07B687A
:1097C0001B681C4A934213D07B681B681A4A934259
:1097D0000ED07B681B68194A934209D07B681B68CE
:1097E000174A934204D07B681B68164A93422BD1D8
:1097F0007B681B681B6803F01003002B14BF012358
:109800000023DBB22AE000BF100002402800024023
:1098100040000240580002407000024088000240B0
:10982000A0000240B8000240100402402804024098
:109830004004024058040240700402408804024080
:10984000A0040240B80402407B681B681B6803F058
:109850000203002B14BF01230023DBB2002B00F016
:1098600087807B68DB6D03F01F0320229A403B6AF0
:109870009A607B6893F83530DBB2042B39D17B6872
:109880001B681A687B681B6822F016021A607B68E6
:109890001B685A697B681B6822F080025A617B68EA
:1098A0001B6C002B03D17B689B6C002B07D07B6863
:1098B0001B681A687B681B6822F008021A607B68C4
:1098C000DB6D03F01F033F229A403B6A9A607B687E
:1098D000012283F835207B68002283F834207B68DE
:1098E0001B6D002B00F04A837B681B6D78689847DE
:1098F00044E37B681B681B6803F48023002B18D0AB
:109900007B681B681B6803F40023002B08D17B686D
:109910005B6C002B2CD07B685B6C7868984727E0E9
:109920007B68DB6B002B23D07B68DB6B7868984708
:109930001EE07B681B681B6803F48073002B0FD14B
:109940007B681B681A687B681B6822F010021A602B
:109950007B68012283F835207B68002283F834205D
:109960007B68DB6B002B03D07B68DB6B78689847E8
:109970007B685B6D002B00F006837B685B6D03F0FA
:109980000103002B00F088807B68042283F83520D7
:109990007B681B687A4A93424AD07B681B68794A85
:1099A000934245D07B681B68774A934240D07B68DE
:1099B0001B68764A93423BD07B681B68744A93428B
:1099C00036D07B681B68734A934231D07B681B6832
:1099D000714A93422CD07B681B68704A934227D00F
:1099E0007B681B686E4A934222D07B681B686D4A75
:1099F00093421DD07B681B686B4A934218D07B68EA
:109A00001B686A4A934213D07B681B68684A93427A
:109A10000ED07B681B68674A934209D07B681B683D
:109A2000654A934204D07B681B68644A934208D11C
:109A30007B681B681A687B681B6822F001021A6049
:109A400007E07B681B681A687B681B6822F00102CC
:109A50001A60FB680133FB607A6A9A4207D37B681D
:109A60001B681B6803F00103002BF2D100E000BF6C
:109A70007B681B681B6803F00103002B04D07B6824
:109A8000032283F8352003E07B68012283F8352028
:109A90007B68002283F834207B68DB6C002B00F0AD
:109AA00072827B68DB6C786898476CE27B681B6825
:109AB000434A934222D07B681B68424A93421DD09E
:109AC0007B681B68404A934218D07B681B683F4AFA
:109AD000934213D07B681B683D4A93420ED07B684B
:109AE0001B683C4A934209D07B681B683A4A934200
:109AF00004D07B681B68394A934201D1012300E0FE
:109B00000023002B00F03F827B681B681B683B61D1
:109B10007B68DB6D03F01F0304229A407B691340CE
:109B2000002B00F0CD803B6903F00403002B00F014
:109B3000C7807B68DB6D03F01F0304229A40FB693A
:109B40005A603B6903F40043002B49D03B6903F49E
:109B50008033002B09D17B689B6C002B00F01082B6
:109B60007B689B6C786898470AE27B681B6C002BCB
:109B700000F006827B681B6C7868984700E200BFA3
:109B800010000240280002404000024058000240FD
:109B90007000024088000240A0000240B80002406D
:109BA00010040240280402404004024058040240CD
:109BB0007004024088040240A0040240B80402403D
:109BC000085402581C540258305402584454025845
:109BD000585402586C5402588054025894540258F5
:109BE0003B6903F02003002B60D17B681B687F4A30
:109BF00093424AD07B681B687D4A934245D07B687C
:109C00001B687C4A934240D07B681B687A4A934227
:109C10003BD07B681B68794A934236D07B681B68CF
:109C2000774A934231D07B681B68764A93422CD0A6
:109C30007B681B68744A934227D07B681B68734A11
:109C4000934222D07B681B68714A93421DD07B6887
:109C50001B68704A934218D07B681B686E4A934217
:109C600013D07B681B686D4A93420ED07B681B68DB
:109C70006B4A934209D07B681B686A4A934204D0BE
:109C80007B681B68684A934208D17B681B681A6826
:109C90007B681B6822F008021A6007E07B681B687B
:109CA0001A687B681B6822F004021A607B681B6CD0
:109CB000002B00F065817B681B6C786898475FE13A
:109CC0007B68DB6D03F01F0302229A407B6913401F
:109CD000002B00F0C5803B6903F00203002B00F06D
:109CE000BF807B68DB6D03F01F0302229A40FB6993
:109CF0005A603B6903F40043002B18D03B6903F41E
:109D00008033002B09D17B685B6C002B00F03A811B
:109D10007B685B6C7868984734E17B68DB6B002B71
:109D200000F030817B68DB6B786898472AE13B69FB
:109D300003F02003002B40F089807B681B682B4ACE
:109D400093424AD07B681B68294A934245D07B687E
:109D50001B68284A934240D07B681B68264A93427E
:109D60003BD07B681B68254A934236D07B681B68D2
:109D7000234A934231D07B681B68224A93422CD0FD
:109D80007B681B68204A934227D07B681B681F4A68
:109D9000934222D07B681B681D4A93421DD07B688A
:109DA0001B681C4A934218D07B681B681A4A93426E
:109DB00013D07B681B68194A93420ED07B681B68DE
:109DC000174A934209D07B681B68164A934204D015
:109DD0007B681B68144A934228D17B681B681A6809
:109DE0007B681B6822F014021A6027E01000024012
:109DF000280002404000024058000240700002402B
:109E000088000240A0000240B80002401004024056
:109E100028040240400402405804024070040240FA
:109E200088040240A0040240B80402407B681B681A
:109E30001A687B681B6822F00A021A607B6801229C
:109E400083F835207B68002283F834207B68DB6B45
:109E5000002B00F097807B68DB6B7868984791E077
:109E60007B68DB6D03F01F0308229A407B69134077
:109E7000002B00F088803B6903F00803002B00F002
:109E800082807B681B68414A93424AD07B681B688A
:109E90003F4A934245D07B681B683E4A934240D07C
:109EA0007B681B683C4A93423BD07B681B683B4AFB
:109EB000934236D07B681B68394A934231D07B6825
:109EC0001B68384A93422CD07B681B68364A934201
:109ED00027D07B681B68354A934222D07B681B6879
:109EE000334A93421DD07B681B68324A934218D094
:109EF0007B681B68304A934213D07B681B682F4AEB
:109F000093420ED07B681B682D4A934209D07B6830
:109F10001B682C4A934204D07B681B682A4A9342F0
:109F200008D17B681B681A687B681B6822F01C02DA
:109F30001A6007E07B681B681A687B681B6822F060
:109F40000E021A607B68DB6D03F01F0301229A404A
:109F5000FB695A607B6801225A657B68012283F89D
:109F600035207B68002283F834207B68DB6C002B73
:109F700009D07B68DB6C7868984704E000BF02E09A
:109F800000BF00E000BF2837BD4680BD1000024082
:109F90002800024040000240580002407000024089
:109FA00088000240A0000240B800024010040240B5
:109FB0002804024040040240580402407004024059
:109FC00088040240A0040240B804024080B483B078
:109FD00000AF78607B6893F83530DBB218460C37F9
:109FE000BD465DF8047B704780B487B000AFF86071
:109FF000B9607A603B60FB689B6D7B61FB689B6D21
:10A000003B61FB681B687F4A934272D0FB681B6808
:10A010007D4A93426DD0FB681B687C4A934268D0AE
:10A02000FB681B687A4A934263D0FB681B68794AD5
:10A0300093425ED0FB681B68774A934259D0FB6815
:10A040001B68764A934254D0FB681B68744A93425B
:10A050004FD0FB681B68734A93424AD0FB681B6869
:10A06000714A934245D0FB681B68704A934240D0C6
:10A07000FB681B686E4A93423BD0FB681B686D4AC5
:10A08000934236D0FB681B686B4A934231D0FB6821
:10A090001B686A4A93422CD0FB681B68684A93424B
:10A0A00027D0FB681B68674A934222D0FB681B6875
:10A0B000654A93421DD0FB681B68644A934218D0DE
:10A0C000FB681B68624A934213D0FB681B68614AB5
:10A0D00093420ED0FB681B685F4A934209D0FB682D
:10A0E0001B685E4A934204D0FB681B685C4A93423B
:10A0F00001D1012300E00023002B0DD0FB685B6E33
:10A10000FA68926E5A60FB68DB6E002B04D0FB6825
:10A110001B6FFA68526F5A60FB681B68394A93429A
:10A120004AD0FB681B68384A934245D0FB681B68DD
:10A13000364A934240D0FB681B68354A93423BD075
:10A14000FB681B68334A934236D0FB681B68324A6F
:10A15000934231D0FB681B68304A93422CD0FB6895
:10A160001B682F4A934227D0FB681B682D4A9342F5
:10A1700022D0FB681B682C4A93421DD0FB681B68E9
:10A180002A4A934218D0FB681B68294A934213D08D
:10A19000FB681B68274A93420ED0FB681B68264A5F
:10A1A000934209D0FB681B68244A934204D0FB68A1
:10A1B0001B68234A934201D1012300E00023002BB6
:10A1C00059D0FB68DB6D03F01F033F229A407B6987
:10A1D0009A60FB681B681A68FB681B6822F480227F
:10A1E0001A60FB681B683A685A60FB689B68402BE2
:10A1F00038D1FB681B687A689A60FB681B68BA688C
:10A20000DA6086E010000240280002404000024070
:10A21000580002407000024088000240A000024046
:10A22000B8000240100402402804024040040240EA
:10A23000580402407004024088040240A004024016
:10A24000B8040240085402581C54025830540258B2
:10A2500044540258585402586C54025880540258BE
:10A2600094540258FB681B68BA689A60FB681B68C4
:10A270007A68DA604DE0FB681B68294A934222D075
:10A28000FB681B68274A93421DD0FB681B68264A5F
:10A29000934218D0FB681B68244A934213D0FB6892
:10A2A0001B68234A93420ED0FB681B68214A9342E5
:10A2B00009D0FB681B68204A934204D0FB681B68E6
:10A2C0001E4A934201D1012300E00023002B20D03D
:10A2D000FB68DB6D03F01F0301229A403B695A6063
:10A2E000FB681B683A685A60FB689B68402B08D182
:10A2F000FB681B687A689A60FB681B68BA68DA605A
:10A3000007E0FB681B68BA689A60FB681B687A689C
:10A31000DA6000BF1C37BD465DF8047B704700BFA4
:10A32000085402581C5402583054025844540258DD
:10A33000585402586C54025880540258945402588D
:10A3400080B485B000AF78607B681B68424A934256
:10A350004AD07B681B68414A934245D07B681B68A2
:10A360003F4A934240D07B681B683E4A93423BD0B1
:10A370007B681B683C4A934236D07B681B683B4A2B
:10A38000934231D07B681B68394A93422CD07B685A
:10A390001B68384A934227D07B681B68364A934231
:10A3A00022D07B681B68354A93421DD07B681B68AE
:10A3B000334A934218D07B681B68324A934213D0C9
:10A3C0007B681B68304A93420ED07B681B682F4A1B
:10A3D000934209D07B681B682D4A934204D07B6866
:10A3E0001B682C4A934201D1012300E00023002B7B
:10A3F00024D07B681B68DBB2103B274AA2FB0323F7
:10A400001B09FB60FB6803F00703244AD35C1A4670
:10A410007B68DA65FB68032B08D97B681B681A46E2
:10A420001F4B13401A1D7B689A650DE07B681B6803
:10A430001A461B4B13407A68936505E07B681B68DE
:10A4400023F0FF027B689A657B689B6D1846143782
:10A45000BD465DF8047B70471000024028000240B2
:10A460004000024058000240700002408800024054
:10A47000A0000240B800024010040240280402403C
:10A480004004024058040240700402408804024024
:10A49000A0040240B8040240ABAAAAAAE44C0408F3
:10A4A00000FCFFFF80B485B000AF78600023FB7331
:10A4B0007B689B69002B20D17B689B6A032B58D853
:10A4C00001A252F823F000BFD9A40208EBA40208AD
:10A4D000D9A4020873A502087B68DB6A03F08073C5
:10A4E000002B48D00123FB7345E07B68DB6AB3F1A6
:10A4F000C07F42D10123FB733FE07B689B69B3F5CA
:10A50000005F23D17B689B6A032B38D801A252F8E5
:10A5100023F000BF25A502082BA5020825A50208E7
:10A520003DA502080123FB7330E07B68DB6A03F082
:10A530008073002B25D00123FB7322E07B68DB6A4C
:10A54000B3F1C07F1FD10123FB731CE07B689B6AC2
:10A55000022B02D9032B03D018E00123FB7315E073
:10A560007B68DB6A03F08073002B0ED00123FB7342
:10A570000BE000BF0AE000BF08E000BF06E000BF3C
:10A5800004E000BF02E000BF00E000BFFB7B184614
:10A590001437BD465DF8047B704700BF80B485B0BA
:10A5A00000AF78607B681B68BB607B681B68384ABB
:10A5B000934222D07B681B68364A93421DD07B6849
:10A5C0001B68354A934218D07B681B68334A934214
:10A5D00013D07B681B68324A93420ED07B681B689D
:10A5E000304A934209D07B681B682F4A934204D0BB
:10A5F0007B681B682D4A934201D1012300E00023B0
:10A60000002B1AD07B681B68DBB2083B284AA2FBF0
:10A6100003231B09FB60FA68264B13449B001A4670
:10A620007B681A667B68244A5A66FB6803F01F033E
:10A6300001229A407B689A6624E07B681B68DBB243
:10A64000103B1E4AA2FB03231B09FB60BB681C4A8C
:10A65000934206D8BB681B4A934202D9FB68083371
:10A66000FB60FA68184B13449B001A467B681A6615
:10A670007B68164A5A66FB6803F01F0301229A4062
:10A680007B689A6600BF1437BD465DF8047B70474F
:10A69000085402581C54025830540258445402586A
:10A6A000585402586C54025880540258945402581A
:10A6B000CDCCCCCC0096001680580258ABAAAAAAE2
:10A6C000B80402400F0402400082001080080240DB
:10A6D00080B485B000AF78607B685B68DBB2FB60FC
:10A6E000FB68002B4AD0FB68082B47D87B681B68A7
:10A6F000254A934222D07B681B68244A93421DD08E
:10A700007B681B68224A934218D07B681B68214AE9
:10A71000934213D07B681B681F4A93420ED07B681C
:10A720001B681E4A934209D07B681B681C4A9342EF
:10A7300004D07B681B681B4A934201D1012300E0CF
:10A740000023002B0AD0FA68174B13449B001A46CB
:10A750007B68DA667B68154A1A6709E0FA68144B69
:10A7600013449B001A467B68DA667B68114A1A67B5
:10A77000FB68013B01229A407B685A6700BF14378F
:10A78000BD465DF8047B7047085402581C540258BB
:10A790003054025844540258585402586C540258C9
:10A7A00080540258945402583F960016405902585B
:10A7B0003F8200104009024080B584B000AF78604D
:10A7C0007B68002B01D10123CFE07B68D3F8843074
:10A7D000002B06D17B682322C3F8842078680BF015
:10A7E00055F9644BD3F8F430624A43F00203C2F8DF
:10A7F000F430604BD3F8F43003F00203BB60BB6865
:10A800007B681B7A002B03D10020FBF717FC03E0C9
:10A810004FF40000FBF712FC574B5B687B681B682A
:10A8200003F580531B687A68126843F0010302F550
:10A8300080521360FBF7C6FBF86011E0FBF7C2FB28
:10A840000246FB68D31AB3F5FA7F09D97B68042264
:10A85000C3F888207B68E022C3F88420012384E0C9
:10A860007B681B6803F580531B6803F00103002B12
:10A87000E4D1786800F0E0FE05F03EFA03463F4A76
:10A88000A2FB03239A0C7B681B68013AC3F8DC2007
:10A89000786801F0CBF87B681B6803F58053D3F828
:10A8A000003123F4E0137A68126843F4002302F5C0
:10A8B0008052C2F800317B685B6903F00303002B10
:10A8C00009D07B680122C3F888207B68E022C3F8A6
:10A8D0008420012349E07B681B6803F58053D3F88B
:10A8E0000821274B13407A68526951007A68126830
:10A8F0000B4302F58052C2F80831786801F033F951
:10A90000786801F079F97B685B6805331B781A0277
:10A910007B685B6804331B7819467B681B680A43B5
:10A92000C3F800237B685B6803331B781A067B68D7
:10A930005B6802331B781B041A437B685B68013336
:10A940001B781B021A437B685B681B7819467B687F
:10A950001B680A43C3F804237B680022C3F88820DD
:10A960007B681022C3F88420002318461037BD46A8
:10A9700080BD00BF004402580004005883DE1B4322
:10A980000180FFFF80B582B000AF78607B68D3F8AC
:10A990008430102B53D17B682322C3F884207B683A
:10A9A0000422DA66786800F0F6F97B681B681A689A
:10A9B0007B681B6842F002021A607B681B681A6899
:10A9C0007B681B6842F001021A607B681B68D3F841
:10A9D000002D7B681B6842F00102C3F8002D7B68E4
:10A9E0001B6803F58053D3F804317A68126843F08A
:10A9F000010302F58052C2F804317B681B6803F53D
:10AA00008053D3F808317A68126843F0010302F5E5
:10AA10008052C2F808317B681B6803F58053D3F875
:10AA200060317A68126843F4817302F58052C2F88B
:10AA300060317B682322C3F88420002300E00123D7
:10AA400018460837BD4680BD80B483B000AF78603B
:10AA50007B68D3F88430232B3FD17B682322C3F853
:10AA600084207B681B6803F58053D3F804317A682F
:10AA7000126823F0010302F58052C2F804317B68AA
:10AA80001B6803F58053D3F808317A68126823F005
:10AA9000010302F58052C2F808317B681B681A680E
:10AAA0007B681B6822F001021A607B681B68D3F880
:10AAB000002D7B681B6842F00102C3F8002D7B6803
:10AAC0001B681A687B681B6822F002021A607B68A8
:10AAD0001022C3F88420002300E0012318460C371D
:10AAE000BD465DF8047B704780B586B000AFF86066
:10AAF000B9607A60BB68002B09D1FB68D3F8883055
:10AB000043F00102FB68C3F8882001237FE0FB6863
:10AB1000D3F88430232B79D10022B968F86801F08A
:10AB2000C9F80346002B09D0FB68D3F8883043F0FE
:10AB30000202FB68C3F88820012368E0BFF34F8F4F
:10AB400000BFFB689A6AFB68063253F822307B61CB
:10AB5000FB689B6A5A1CFB689A62FB689B6A032B22
:10AB600004D9FB689B6A1A1FFB689A62FB68996AA2
:10AB7000FB681A68FB68063153F8213002F58052F1
:10AB8000C2F82031FBF71EFA386139E0FB681B6818
:10AB900003F58053D3F8603103F48053002B12D0B7
:10ABA000FB68D3F8883043F00802FB68C3F88820BC
:10ABB000FB681B6803F58053D3F86021FB68C3F87A
:10ABC0008C20012323E07B68B3F1FF3F18D0FBF713
:10ABD000F9F902463B69D31A7A689A4202D37B6834
:10ABE000002B0DD1FB68D3F8883043F00402FB68DA
:10ABF000C3F888207B694FF04052DA60012306E0F9
:10AC00007B69DB68002BC1DB002300E001231846D1
:10AC10001837BD4680BD80B588B000AF7860396018
:10AC200000237B610023FB733B68002B09D17B6809
:10AC3000D3F8883043F001027B68C3F888200123F1
:10AC4000A5E07B68D3F88430232B01D001239EE05C
:10AC50007B68DB6DFB617B68FA69123253F8223046
:10AC6000BB617B68DB6EC3F10403BB6067E0BB695B
:10AC7000DB6803F08043002B07D0BB695A687B6810
:10AC80009A67BB691A687B685A67BB69DB6803F01F
:10AC90000053002B03D17B68DB6F002B3DD0BB69D9
:10ACA000DB6803F00053002B05D07B6800221A6696
:10ACB0007B6800225A667B685B693B61BB69DB6825
:10ACC00003F08053002B0DD0BB69DB68C3F30E0289
:10ACD0007B685B6ED31A3B61BB69DA687B681A6775
:10ACE0000123FB737B6803F17C007B6803F1800127
:10ACF000BB691B691A463B699BB20BF085F87B6800
:10AD00001B6E5A1C7B681A667B685A6E3B691A4434
:10AD10007B685A66BB6900221A61FB690133FB61DB
:10AD2000FB69032B02D9FB69043BFB617B68FA6971
:10AD3000123253F82230BB617B6901337B61BB69FE
:10AD4000DB68002B06DB7A69BB689A4202D2FB7B88
:10AD5000002B8CD07B68DA6E7B691A447B68DA66DC
:10AD60007B68DB6E002B02D0786800F014F87B68FB
:10AD7000FA69DA65FB7B012B08D17B68DA6F3B68E7
:10AD80001A607B680022DA67002300E0012318467E
:10AD90002037BD4680BD80B588B000AF7860002305
:10ADA000FB600123FB747B689B6EFB617B68FA6927
:10ADB000123253F822307B617B68DB6EBB613BE073
:10ADC0007B691B69002B12D107F10C0318460AF0AE
:10ADD000EBFFFB68002B02D10023FB7407E0FB684C
:10ADE0001A467B691A61FB681A467B691A60FB7C0C
:10ADF000002B21D0BFF35F8F00BF7B689B6D002BC2
:10AE000004D07B694FF04142DA6003E07B694FF088
:10AE10000142DA60FB690133FB61FB69032B02D954
:10AE2000FB69043BFB617B68FA69123253F82230FC
:10AE30007B61BB69013BBB61BB69002B02D0FB7C22
:10AE4000002BBDD17B68DB6EBA699A420DD07B685E
:10AE50001B6803F580531A460023C2F828317B682B
:10AE6000FA699A667B68BA69DA6600BF2037BD4620
:10AE700080BD000080B584B000AF78607B681B683F
:10AE800003F58053D3F8603103F04003402B15D114
:10AE90007B681B6803F58053D3F8343103F040031B
:10AEA000402B0BD17B681B6803F580531A4648F290
:10AEB0004003C2F86031786800F0F6F87B681B68E0
:10AEC00003F58053D3F8603103F00103012B15D152
:10AED0007B681B6803F58053D3F8343103F001031A
:10AEE000012B0BD17B681B6803F580531A4648F28F
:10AEF0000103C2F86031786800F0CCF87B681B6809
:10AF000003F58053D3F8603103F48043B3F5804FE9
:10AF100053D17B681B6803F58053D3F8343103F4B5
:10AF20008043B3F5804F48D17B68D3F8883043F035
:10AF300008027B68C3F888207B681B6803F5805390
:10AF4000D3F8603103F48053B3F5805F1ED17B6882
:10AF50001B6803F58053D3F8602141F202131340BC
:10AF60007A68C2F88C307B681B6803F58053D3F88D
:10AF700034317A68126823F4404302F58052C2F8F3
:10AF800034317B68E022C3F8842013E07B681B68BF
:10AF900003F58053D3F8603103F4CD427B68C3F8E6
:10AFA0008C207B681B6803F580531A464FF4CD4311
:10AFB000C2F86031786800F081F87B681B68D3F8CC
:10AFC000B430FB60FB6803F48043002B04D1FB68C2
:10AFD00003F40053002B19D07B68D3F8883043F07A
:10AFE00010027B68C3F888207B681B68D3F8B82000
:10AFF0007B68C3F890207B68E022C3F884207868DF
:10B0000000F05CF87B680022C3F890207B681B6826
:10B01000D3F8B03003F01003102B0FD17B681B68FE
:10B02000D3F8C03003F060027B68C3F894207868DE
:10B0300000F04EF87B680022C3F894207B681B6800
:10B04000D3F8B03003F02003202B0FD17B681B68AE
:10B05000D3F8C03003F00F027B68C3F898207868FB
:10B0600000F040F87B680022C3F89820084B9B6AE8
:10B0700003F48003002B06D0054B4FF480029A6244
:10B08000786800F039F800BF1037BD4680BD00BFBA
:10B090008000005880B483B000AF786000BF0C37E8
:10B0A000BD465DF8047B704780B483B000AF786024
:10B0B00000BF0C37BD465DF8047B704780B483B099
:10B0C00000AF786000BF0C37BD465DF8047B704769
:10B0D00080B483B000AF786000BF0C37BD465DF828
:10B0E000047B704780B483B000AF786000BF0C373A
:10B0F000BD465DF8047B704780B483B000AF7860D4
:10B1000000BF0C37BD465DF8047B704780B586B044
:10B1100000AFF860B9607A603B60FB681B68D3F8E9
:10B12000003203F00103002B01D001233EE0FB6855
:10B130001B68D3F800327B617B6923F07872BB68AF
:10B140005B0513437B617B6923F4F8127B681B0466
:10B1500013437B617B6943F00C037B617B6943F0A4
:10B1600001037B61FB681B687A69C3F80022FAF768
:10B1700029FF386109E0FAF725FF02463B69D31A37
:10B18000B3F57A7F01D9012310E0FB681B68D3F87F
:10B19000003203F00103002BEDD1FB681B68D3F8EC
:10B1A00004329BB21A463B681A60002318461837CF
:10B1B000BD4680BD80B586B000AFF860B9607A60EA
:10B1C0003B60FB681B68D3F8003203F00103002BDF
:10B1D00001D001233CE0FB681B68D3F800327B619F
:10B1E0007B6923F07872BB685B0513437B617B69E5
:10B1F00023F4F8127B681B0413437B617B6923F003
:10B200000C0343F004037B617B6943F001037B6122
:10B210003B689AB2104BC3F804220F4A7B69C2F80C
:10B220000032FAF7CFFE386109E0FAF7CBFE0246AA
:10B230003B69D31AB3F57A7F01D9012308E0FB6893
:10B240001B68D3F8003203F00103002BEDD100237B
:10B2500018461837BD4680BD0080024080B483B0D8
:10B2600000AF786039603B68002B01D10123C3E156
:10B270007B681B681B6803F00C023B68DA627B6822
:10B280001B681B6803F01003002B14BF012300236D
:10B29000DBB21A463B6883F828207B681B681B6872
:10B2A00003F060023B685A627B681B681B6803F40A
:10B2B0008073002B0CBF01230023DBB21A463B68CE
:10B2C00083F820207B681B681B6803F40073002B45
:10B2D00014BF01230023DBB21A463B68DA777B6890
:10B2E0001B681B6803F48063002B0CBF0123002341
:10B2F000DBB21A463B689A777B681B681B6803F4CD
:10B300000063002B14BF01230023DBB21A463B6805
:10B310005A777B681B681B6803F48053002B14BFAB
:10B3200001230023DBB21A463B681A777B681B684F
:10B330001B6803F400523B689A617B681B681B68BA
:10B3400003F480423B685A617B681B681B6803F406
:10B350008033002B14BF01230023DBB21A463B6865
:10B360009A747B681B681B6803F40033002B0CBFC6
:10B3700001230023DBB21A463B685A747B681B68C2
:10B380001B6803F40023002B0CBF01230023DBB256
:10B390001A463B681A747B681B681B6803F48013A9
:10B3A000002B14BF01230023DBB21A463B68DA737B
:10B3B0007B681B681B6803F40013002B14BF012378
:10B3C0000023DBB21A463B689A737B681B681B68D4
:10B3D00003F48003002B14BF01230023DBB21A46C1
:10B3E0003B685A737B681B681B6803F40003002BDF
:10B3F00014BF01230023DBB21A463B681A737B6833
:10B400001B681B6803F0E0623B689A607B681B68FE
:10B410001B6803F00063002B14BF01230023DBB281
:10B420001A463B681A717B681B681B6803F0E04290
:10B430003B681A607B681B685B68C3F30D023B685E
:10B440005A637B681B685B6803F48033002B0CBF76
:10B4500001230023DBB21A463B6883F832207B6865
:10B460001B685B6803F40033002B14BF0123002327
:10B47000DBB21A463B6883F831207B681B685B6847
:10B4800003F48023002B14BF01230023DBB21A46F0
:10B490003B6883F830207B681B685B6803F080732F
:10B4A000002B14BF01230023DBB21A463B6883F84C
:10B4B00038207B681B685B685B0E03F01F023B68EB
:10B4C000DA637B681B68DB6803F48073002B14BFAE
:10B4D00001230023DBB21A463B6883F840207B68D7
:10B4E0001B68DB6803F00F023B685A647B681B68CB
:10B4F0001B6F03F00203002B14BF01230023DBB2F8
:10B500001A463B6883F854207B681B681B6F03F066
:10B510008003002B0CBF01230023DBB21A463B68DB
:10B5200083F84C207B681B681B6F03F070023B683C
:10B530001A657B681B681B6F1B0C9AB23B689A6488
:10B540007B681B68D3F8903003F00103002B14BF15
:10B5500001230023DBB21A463B6883F856207B6840
:10B560001B68D3F8903003F00203002B14BF0123B3
:10B570000023DBB21A463B6883F855207B681B68C2
:10B58000D3F8003D03F072023B689A657B681B6844
:10B59000D3F8303D03F023023B68DA657B681B6813
:10B5A000D3F8303D03F00803002B14BF0123002320
:10B5B000DBB21A463B6883F862207B681B68D3F8CD
:10B5C000303D03F01003002B14BF01230023DBB236
:10B5D0001A463B6883F861207B681B68D3F8303DCE
:10B5E00003F04003002B0CBF01230023DBB21A46FB
:10B5F0003B6883F86020002318460C37BD465DF891
:10B60000047B704780B582B000AF786039603B68DA
:10B61000002B01D101230BE07B68D3F88430102B81
:10B6200005D13968786800F05FF8002300E0012355
:10B6300018460837BD4680BD80B584B000AF78603D
:10B640007B681B68D3F80032FB60FB6823F47063EF
:10B65000FB6004F051FBB860BB681E4A934208D9F6
:10B66000BB681D4A934204D8FB6843F40073FB6037
:10B6700027E0BB68184A934208D9BB68174A93422F
:10B6800004D2FB6843F44073FB601AE0BB68134AC2
:10B69000934203D3BB68124A934211D9BB68104A44
:10B6A000934208D9BB680F4A934204D8FB6843F41D
:10B6B0008073FB6005E0FB6843F48063FB6000E09F
:10B6C00000BF7B681B68FA68C3F8002200BF103710
:10B6D000BD4680BDFF2C3101BF0E160200879303CB
:10B6E000FFE0F5057FD1F00880B485B000AF786049
:10B6F00039603B689A683B681B681A433B681B7952
:10B70000DB061A433B681B7BDB051A433B685B7B0C
:10B710009B051A433B689B7B5B051A433B68DB7BBD
:10B720001B0513433A68127C002A02D14FF4002211
:10B7300000E0002213433A68527C002A02D14FF401
:10B74000003200E000221A433B689B7C1B041A4332
:10B750003B685B691A433B689B691A433B681B7FE4
:10B760001B031A433B685B7FDB0213433A68927FFB
:10B77000002A02D14FF4806200E000221A433B68A5
:10B78000DB7F5B0213433A6892F82020002A02D143
:10B790004FF4807200E000221A433B685B6A1A4350
:10B7A0003B6893F828301B011A433B68DB6A13435C
:10B7B000FB607B681B681A68564B13407A681268F6
:10B7C000F9680B4313603B68DB6B5A063B6893F8E0
:10B7D00038301B061A433B6893F830309B041A43F9
:10B7E0003B6893F831305B0413433A6892F8322097
:10B7F000002A02D14FF4803200E000221A433B6855
:10B800005B6B1343FB607B681B685A68424B1340B9
:10B810007A681268F9680B4353603B6893F84030CC
:10B820001A023B685B6C1343FB607B681B68DA6839
:10B830003A4B13407A681268F9680B43D3603B684F
:10B8400093F854305A003B681B6D13433A6892F8E2
:10B850004C20002A01D1802200E000221A433B68DC
:10B860009B6C1B041343FB607B681B681A6F4FF6CD
:10B870000D7313407A681268F9680B4313673B68CD
:10B8800093F856301A463B6893F855305B001343E3
:10B89000FB607B681B68D3F8903023F003017B6862
:10B8A0001B68FA680A43C3F890207B681B68D3F8CA
:10B8B000003D23F072013B689A6D7B681B680A4368
:10B8C000C3F8002D3B68DB6D3A6892F86020002ACF
:10B8D00001D1402200E000221A433B6893F8613016
:10B8E0001B011A433B6893F86230DB001343FB6093
:10B8F0007B681B68D3F8303D23F07B017B681B68B5
:10B90000FA680A43C3F8302D00BF1437BD465DF80E
:10B91000047B7047838004000080F8C0F0FEFFFFC6
:10B9200080B485B000AF786039607B681B6803F530
:10B9300080531A68384B13403A6811687A68126865
:10B940000B4302F5805213603B681B791A033B6876
:10B950009B681A433B681B7BDB031343FB607B68DC
:10B960001B6803F580535A682C4B13407A681268A1
:10B97000F9680B4302F5805253603B685B7B1A0405
:10B980003B681B6A1343FB607B681B6803F58053AD
:10B99000D3F80021224B13407A681268F9680B43F0
:10B9A00002F58052C2F800313B681A693B681B7D82
:10B9B0001B011A433B685B7F1B031343FB607B68DF
:10B9C0001B6803F58053D3F80421164B13407A68A3
:10B9D0001268F9680B4302F58052C2F804313B68E3
:10B9E0001B7FDA073B689B691343FB607B681B681E
:10B9F00003F58053D3F808210B4B13407A68126883
:10BA0000F9680B4302F58052C2F8083100BF1437C1
:10BA1000BD465DF8047B7047FD87FFFFFE2FFFFFEB
:10BA200000C0FEFFEFEFC0FFFFFFC07F80B5A4B0F6
:10BA300000AF7860012387F83B3000233B6500238B
:10BA400087F84930002387F84B30012387F83030DE
:10BA5000012387F85E30012387F83A30002387F806
:10BA60005430012387F88C304FF400537B6400235B
:10BA700087F864300023BB66002387F88D300023ED
:10BA800087F88E304FF4C3633B66002387F8383065
:10BA900000237B63012387F83D30002387F83E3085
:10BAA000002387F848300023FB6700237B670023CF
:10BAB000BB65002387F86C30002387F882300123B0
:10BAC00087F84A302023C7F88830012387F84C30A4
:10BAD000002387F85D304FF04053FB624FF4804302
:10BAE0003B64002387F839300223C7F884300023F1
:10BAF00087F88030002387F88130002387F85C3096
:10BB0000012387F83C3000233B67012387F8783016
:10BB100007F12C0319467868FFF7E6FD01233B7314
:10BB200001233B610023BB60002387F824300023FE
:10BB30007B7500233B754FF400133B6200233B777A
:10BB40004FF40013BB61002387F825304FF40673D0
:10BB5000BB6207F1080319467868FFF7E1FE00BFF2
:10BB60009037BD4680BD80B485B000AF78600023BB
:10BB7000FB601DE07B68D968FA6813465B001344DC
:10BB8000DB000B44BB60BB6800221A60BB6800226C
:10BB90005A60BB6800229A60BB680022DA60B9680C
:10BBA0007B68FA68063243F82210FB680133FB60B9
:10BBB000FB68032BDED97B6800229A627B681B68D6
:10BBC00003F580531A460323C2F82C317B68DA68E8
:10BBD0007B681B6803F58053C3F814217B68DA681F
:10BBE0007B681B6803F58053C3F8202100BF14371E
:10BBF000BD465DF8047B704780B485B000AF7860C7
:10BC00000023FB6023E07B681969FA6813465B0038
:10BC10001344DB000B44BB60BB6800221A60BB68A6
:10BC200000225A60BB6800229A60BB680022DA607A
:10BC3000BB6800221A61BB6800225A61B9687B6840
:10BC4000FA68123243F82210FB680133FB60FB688C
:10BC5000032BD8D97B680022DA657B6800221A663C
:10BC60007B6800229A667B680022DA667B68002285
:10BC70009A657B681B6803F580531A460323C2F854
:10BC800030317B681A697B681B6803F58053C3F801
:10BC90001C217B681B6903F148027B681B6803F564
:10BCA0008053C3F8282100BF1437BD465DF8047BDC
:10BCB0007047000080B48DB000AFF860B9607A6062
:10BCC000FB6818337B617B691B69FB627B691B69BD
:10BCD0003B6100237B627B69FA6A53F822303B6246
:10BCE000BB689B68FB610023BB613B6ADB6803F0B8
:10BCF0000043B3F1004F07D07A69FB6A04339B001D
:10BD000013445B68002B01D0022359E2BB681B6817
:10BD100003F00403002B44D03B6ADA68754B1340F0
:10BD2000BA68526A1A433B6ADA603B6ADB6843F4DA
:10BD300080323B6ADA60FB681B681A6EFB681B681E
:10BD400042F480121A66BB681B6803F00803002BDC
:10BD500027D03B6A9B689AB2BB68DB6A1B041A4314
:10BD60003B6A9A603B6ADB6843F400323B6ADA6004
:10BD70003B6ADB6823F44022BB681B6B1A433B6AB7
:10BD8000DA60FB681B685A6EFB681B6842F480121D
:10BD90005A66FB681B681A6DFB681B6842F080627C
:10BDA0001A65BB681B6803F01003002B0ED03B6ABA
:10BDB0009A68514B1340BA6892691A433B6A9A6079
:10BDC0003B6ADB6843F080623B6ADA60BB681B68F1
:10BDD00003F00403002B05D1BB681B6803F01003BC
:10BDE000002B36D03B6ADB6843F080423B6ADA6066
:10BDF000BFF35F8F00BF3B6ADB6843F000423B6AE2
:10BE0000DA60FB6A0133FB62FB6A032B02D9FB6A2F
:10BE1000043BFB627B69FA6A53F822303B627B6A1F
:10BE200001337B623B6ADB6803F00043B3F1004FF0
:10BE30000FD17B693A6953F822303B62BFF35F8FC1
:10BE400000BF3B6ADB6823F000423B6ADA600223F2
:10BE5000B6E17B6A01337B62FB691B681A463B6A69
:10BE60001A603B6A9A68244B1340FA6952681A4375
:10BE70003B6A9A60FB699B68002B12D0FB699B6848
:10BE8000FB61FB691B681A463B6A5A603B6A9A6809
:10BE90001A4B1340FA69526812041A433B6A9A60BB
:10BEA00008E03B6A00225A603B6A9A68134B1340D1
:10BEB0003A6A9360BB681B6803F01003002B21D023
:10BEC0003B6ADB6823F4F002BB681B6ADB041A439D
:10BED0003B6ADA603B6ADA68094B1340BA68D26998
:10BEE0001A433B6ADA603B6ADB6843F480223B6AB0
:10BEF000DA602EE00000FFFF00C0FFFFFFFF00C080
:10BF00000000FCFF3B6ADA687B4B1340BA6852685A
:10BF10001A433B6ADA60BB681B6803F00103002B1D
:10BF200008D03B6ADB6823F44032BB685B691A4384
:10BF30003B6ADA60BB681B6803F02003002B08D063
:10BF40003B6ADB6823F04062BB681B691A433B6AAB
:10BF5000DA60BB681B6803F00403002B08D03B6A5F
:10BF60009B6823F44042BB689B6A1A433B6A9A6011
:10BF70003B6ADB6843F000523B6ADA603B6ADB688D
:10BF800023F080423B6ADA60BFF35F8F00BF3B6AF9
:10BF9000DB6843F000423B6ADA60BB681B6803F071
:10BFA0000203002B00F0DA803B6ADB6823F060724A
:10BFB000BB68DB681A433B6ADA60CFE03B6ADB6848
:10BFC00023F080523B6ADA60FB6A0133FB62FB6A52
:10BFD000032B02D9FB6A043BFB627B69FA6A53F8C4
:10BFE00022303B623B6ADB6823F000523B6ADA6036
:10BFF0003B6ADB6803F00043B3F1004F07D07A6976
:10C00000FB6A04339B0013445B68002B29D03B6917
:10C01000FB627B69FA6A53F822303B620023BB6201
:10C0200019E0BFF35F8F00BF3B6ADB6823F000427B
:10C030003B6ADA60FB6A0133FB62FB6A032B02D9BD
:10C04000FB6A043BFB627B69FA6A53F822303B626D
:10C05000BB6A0133BB62BA6A7B6A9A42E1D30223AC
:10C06000AEE07B6A01337B62FB699B68FB61FB6925
:10C070001B681A463B6A1A603B6A9A681F4B13405A
:10C08000FA6952681A433B6A9A60FB699B68002B05
:10C0900012D0FB699B68FB61FB691B681A463B6A0F
:10C0A0005A603B6A9A68164B1340FA695268120448
:10C0B0001A433B6A9A6008E03B6A00225A603B6A76
:10C0C0009A680F4B13403A6A9360BB681B6803F091
:10C0D0001003002B18D03B6ADA680A4B1340BA6889
:10C0E000D2691A433B6ADA603B6ADB6843F4802218
:10C0F0003B6ADA6020E000BF0080FFFF00C0FFFF66
:10C10000FFFF00C00000FCFF3B6ADA682F4B1340C2
:10C11000BA6852681A433B6ADA60BB681B6803F06E
:10C120000103002B08D03B6ADB6823F44032BB6874
:10C130005B691A433B6ADA60BB690133BB61BFF3D9
:10C140005F8F00BF3B6ADB6843F000423B6ADA6006
:10C150003B6ADB6823F080423B6ADA60FB699B68DC
:10C16000002B7FF42BAF7B68002B06D03B6A9B68CB
:10C1700043F000423B6A9A6005E03B6A9B6823F00B
:10C1800000423B6A9A603B6ADB6843F080523B6A3C
:10C19000DA607B695A6A7969FB6A04339B000B4455
:10C1A0005A607B69FA6A1A6172B600BF7B699A6A43
:10C1B000BB6913445A1C7B699A6262B600BF0023B4
:10C1C00018463437BD465DF8047B70470080FFFF9A
:10C1D00080B598B000AF7860844A07F10C0311462F
:10C1E0004C22184614F084FB7B68002B01D10123FC
:10C1F000C6E17B681B687E4A934206D17B681B6858
:10C2000003F580731A467B685A607B6893F8983010
:10C21000DBB2002B06D17B68002283F89920786876
:10C22000F7F7A2FA7B681B689A697B681B6822F0A3
:10C2300010029A61F9F7C6FEF86514E0F9F7C2FE3C
:10C240000246FB6DD31A0A2B0DD97B68D3F89C30BC
:10C2500043F001027B68C3F89C207B68032283F8CB
:10C26000982001238CE17B681B689B6903F008031D
:10C27000082BE3D07B681B689A697B681B6842F0D7
:10C2800001029A61F9F79EFEF86514E0F9F79AFE4B
:10C290000246FB6DD31A0A2B0DD97B68D3F89C306C
:10C2A00043F001027B68C3F89C207B68032283F87B
:10C2B0009820012364E17B681B689B6903F00103FC
:10C2C000002BE3D07B681B689A697B681B6842F08F
:10C2D00002029A617B681B7C012B08D17B681B687A
:10C2E0009A697B681B6822F040029A6107E07B68CC
:10C2F0001B689A697B681B6842F040029A617B6800
:10C300005B7C012B08D17B681B689A697B681B6882
:10C3100042F480429A6107E07B681B689A697B68F7
:10C320001B6822F480429A617B689B7C012B08D1B8
:10C330007B681B689A697B681B6822F480529A614B
:10C3400007E07B681B689A697B681B6842F480522F
:10C350009A617B681B689B6923F440717B689A68CB
:10C360007B681B680A439A617B681B689A697B68D3
:10C370001B6822F0A4029A617B681B681A697B68BB
:10C380001B6822F010021A617B68DB68012B08D160
:10C390007B681B689A697B681B6842F004029A619B
:10C3A00030E07B68DB68002B2CD07B68DB68022BDD
:10C3B00020D07B681B689A697B681B6842F080020A
:10C3C0009A617B681B681A697B681B6842F01002DF
:10C3D0001A617B68DB68032B14D17B681B689A6940
:10C3E0007B681B6842F020029A610BE080220408FF
:10C3F00000A000407B681B689A697B681B6842F05C
:10C4000020029A617B689B69013B5A067B68DB6965
:10C41000013B1B021A437B681B6A013B42EA030192
:10C420007B685B69013B1A047B681B680A43DA611D
:10C430007B689B68B3F5407F15D17B689B6A5A1E69
:10C440007B68DB6A013B1B021A437B681B6B013B69
:10C450001B0142EA03017B685B6A013B1A047B68AB
:10C460001B680A43DA607B681B6E002B0AD07B686E
:10C470001B68D3F8C0107B685A6E7B681B680A4340
:10C48000C3F8C0207B68DA6D7B681B6E1344002BF9
:10C4900011D07B681B68D3F8C83023F007017B6894
:10C4A0009B6E9B0060333B4453F8542C7B681B68A5
:10C4B0000A43C3F8C8207B681B6C002B11D07B6833
:10C4C0001B68D3F8BC3023F007017B685B6C9B00D2
:10C4D00060333B4453F8542C7B681B680A43C3F811
:10C4E000BC207B689B6C002B12D07B681B68D3F848
:10C4F000BC3023F070017B68DB6C9B0060333B44F5
:10C5000053F8543C1A017B681B680A43C3F8BC20EB
:10C510007B681B6D002B12D07B681B68D3F8BC3086
:10C5200023F4E0617B685B6D9B0060333B4453F810
:10C53000543C1A027B681B680A43C3F8BC207B6822
:10C540001B68114A934207D17B685B689A687B68D5
:10C550005B6822F003029A607B680022C3F8942093
:10C560007B680022C3F89C207B68012283F8982016
:10C57000786800F077FD034687F85B3097F85B300A
:10C5800018466037BD4680BD00A0004080B483B02F
:10C5900000AF78607B6893F89830DBB2012B11D143
:10C5A0007B68022283F898207B681B689A697B6805
:10C5B0001B6822F001029A617B680022C3F89C206C
:10C5C000002308E07B68D3F89C3043F004027B68CA
:10C5D000C3F89C20012318460C37BD465DF8047B48
:10C5E000704780B586B000AFF860B9607A60FB68CC
:10C5F00093F89830DBB2022B41D1FB681B68D3F86B
:10C60000C03003F07C53002B09D1FB68D3F89C3079
:10C6100043F02002FB68C3F89C20012338E0FB684C
:10C620001B68D3F8C43003F40013002B09D0FB6857
:10C63000D3F89C3043F40072FB68C3F89C200123BC
:10C6400026E0FB681B68D3F8C4301B0C03F01F0303
:10C650007B617B697A68B968F86800F089FEFB68DD
:10C660001B6801217A6901FA02F2C3F8D020012285
:10C670007B699A40FB68C3F89420002308E0FB68BC
:10C68000D3F89C3043F00802FB68C3F89C200123D8
:10C6900018461837BD4680BD80B48BB000AFF86037
:10C6A000B9607A603B600023FB61FB6893F89830C7
:10C6B000FB76FB7E022B40F04B81BB68402B4DD1BB
:10C6C000FB681B68D3F8A03003F4FE03002B09D1EC
:10C6D000FB68D3F89C3043F02002FB68C3F89C2031
:10C6E00001233EE1FB681B68D3F8A43003F07F030D
:10C6F000002B09D1FB68D3F89C3043F48072FB68AF
:10C70000C3F89C2001232CE1FB681B68D3F8A430FC
:10C710001B0E03F00103012B0BD1FB681B68D3F840
:10C72000A030DB0F03F00103B3F1004F01D101236F
:10C73000FB61FB681B68D3F8A4301B0A03F03F03BE
:10C74000FA691344FB61FB685A6FFB685B6CF9691B
:10C7500001FB03F39B0013447B6269E0BB68412B40
:10C760004DD1FB681B68D3F8B03003F4FE03002BF7
:10C7700009D1FB68D3F89C3043F02002FB68C3F872
:10C780009C200123EDE0FB681B68D3F8B43003F074
:10C790007F03002B09D1FB68D3F89C3043F48072EF
:10C7A000FB68C3F89C200123DBE0FB681B68D3F81F
:10C7B000B4301B0E03F00103012B0BD1FB681B6887
:10C7C000D3F8B030DB0F03F00103B3F1004F01D118
:10C7D0000123FB61FB681B68D3F8B4301B0A03F02C
:10C7E0003F03FA691344FB61FB689A6FFB68DB6CDB
:10C7F000F96901FB03F39B0013447B6218E0FB68BB
:10C800001B6DBA689A4209D3FB68D3F89C3043F099
:10C810002002FB68C3F89C200123A2E0FB68DA6FCA
:10C82000FB685B6DB96801FB03F39B0013447B62FB
:10C830007B6A1B6803F080427B685A607B685B6898
:10C84000002B07D17B6A1B689B0CC3F30A027B6831
:10C850001A6005E07B6A1B6823F060427B681A60FF
:10C860007B6A1B6803F000527B689A607B6A1B68D6
:10C8700003F000427B681A617B6A04337B627B6A47
:10C880001B689AB27B68DA617B6A1B6803F47022CA
:10C890007B68DA607B6A1B6803F480127B685A61EC
:10C8A0007B6A1B6803F400127B689A617B6A1B68D1
:10C8B0001B0E03F07F027B681A627B6A1B68DA0F2B
:10C8C0007B685A627B6A04337B627B6A7B610023EC
:10C8D0003B620AE07A693B6A1A4439683B6A0B4456
:10C8E00012781A703B6A01333B627B68DB681B0C71
:10C8F0001F4AD35C1A463B6A9342EBD3BB68402B7A
:10C9000005D1FB681B68FA69C3F8A8201EE0BB6864
:10C91000412B05D1FB681B68FA69C3F8B82015E004
:10C92000BB681F2B08D8FB681B680121BA6801FA95
:10C9300002F2C3F8982009E0BB6803F01F02FB680D
:10C940001B68012101FA02F2C3F89C20002308E0D1
:10C95000FB68D3F89C3043F00802FB68C3F89C20C6
:10C96000012318462C37BD465DF8047B704700BF95
:10C97000EC4C040880B487B000AFF860B9607A600E
:10C98000FB6893F89830FB75FB7D012B02D0FB7D93
:10C99000022B55D1FB681B689A6DBB681340002BB6
:10C9A00008D1FB681B68DA6DFB681B6842F0010266
:10C9B000DA6514E0FB681B689A6DBB681340BA68BF
:10C9C0009A4208D1FB681B68DA6DFB681B6842F06D
:10C9D0000202DA6503E0FB681B680322DA65BB68C4
:10C9E00003F40073002B09D0FB681B68D3F8E01038
:10C9F000FB681B687A680A43C3F8E020BB6803F44D
:10CA00008063002B09D0FB681B68D3F8E410FB6837
:10CA10001B687A680A43C3F8E420FB681B68596DF9
:10CA2000BA680F4B1340FA6812680B4353650D4BFD
:10CA30005A69BB689B0F0B4913434B61002308E005
:10CA4000FB68D3F89C3043F00202FB68C3F89C20DB
:10CA5000012318461C37BD465DF8047B704700BFB4
:10CA6000FFFFCF3F00A8004080B596B000AF7860D0
:10CA70009A4B1B699B077B65984B5B699B077A6D9B
:10CA800013407B657B681B681B6D03F470433B653B
:10CA90007B681B685B6D3A6D13403B657B681B6868
:10CAA0001B6D03F00F03FB647B681B685B6DFA6C06
:10CAB0001340FB647B681B681B6D03F0F003BB64D1
:10CAC0007B681B685B6DBA6C1340BB647B681B683A
:10CAD0001B6D03F071537B647B681B685B6D7A6C24
:10CAE00013407B647B681B681B6D03F060733B64C1
:10CAF0007B681B685B6D3A6C13403B647B681B680A
:10CB00005B6DFB637B681B681B6DBB63FB6B1B0A68
:10CB100003F00103002B10D0BB6B1B0A03F00103D1
:10CB2000002B0AD07B681B684FF480721A656B4B30
:10CB300000221A61786800F054FAFB6B9B0A03F03C
:10CB40000103002B1DD0BB6B9B0A03F00103002BDC
:10CB500017D07B681B68D3F8DC307B637B681B686D
:10CB6000D3F8E4307A6B13407B637B681B684FF427
:10CB700080621A65594B00221A61796B786800F05F
:10CB800007FA7B6D002B0DD07B681A68796D544BCA
:10CB90000B401365514A7B6D9B0F1361796D78686B
:10CBA00000F0C0F93B6D002B0DD07B681A68396D21
:10CBB0004B4B0B401365494A3B6D9B0F1361396D1D
:10CBC000786800F0BAF9FB6C002B0DD07B681A680E
:10CBD000F96C434B0B401365404AFB6C9B0F136190
:10CBE000F96C7868F4F7AAF8BB6C002B0DD07B6861
:10CBF0001A68B96C3A4B0B401365384ABB6C9B0FF3
:10CC00001361B96C786800F0A3F9FB6BDB0A03F0E1
:10CC10000103002B10D0BB6BDB0A03F00103002BD8
:10CC20000AD07B681B684FF400621A652B4B002208
:10CC30001A61786800F097F9FB6B5B0A03F0010357
:10CC4000002B1DD0BB6B5B0A03F00103002B17D038
:10CC50007B681B68D3F8D8303B637B681B68D3F8CC
:10CC6000E0303A6B13403B637B681B684FF4007203
:10CC70001A651A4B00221A61396B786800F07DF949
:10CC8000FB6BDB0C03F00103002B10D0BB6BDB0C48
:10CC900003F00103002B0AD07B681B684FF40022CD
:10CCA0001A650E4B00221A61786800F07CF9FB6B64
:10CCB0001B0C03F00103002B16D0BB6B1B0C03F005
:10CCC0000103002B10D07B681B684FF480321A657B
:10CCD000024B00221A61786804E000BF00A80040FF
:10CCE000FFFFCF3F00F069F9FB6B9B0C03F00103E2
:10CCF000002B10D0BB6B9B0C03F00103002B0AD060
:10CD00007B681B684FF480221A65834B00221A61EE
:10CD1000786800F05CF9FB6B5B0C03F00103002BFF
:10CD200015D0BB6B5B0C03F00103002B0FD07B68AD
:10CD30001B684FF400321A65774B00221A617B683A
:10CD4000D3F89C3043F080027B68C3F89C203B6C96
:10CD5000002B0DD07B681A68396C704B0B40136543
:10CD60006D4A3B6C9B0F1361396C7868F3F7CAFF0F
:10CD70007B6C002B11D07B681A68796C674B0B4079
:10CD80001365654A7B6C9B0F13617B68D3F89C200D
:10CD90007B6C1A437B68C3F89C207B681B68604AE5
:10CDA000934240F0AC807B685B689B6803F00303B0
:10CDB000002B00F0A4807B685B681B6A03F00F0304
:10CDC000FB627B685B685B6AFA6A1340FB627B68A4
:10CDD0005B681B6A03F03003BB627B685B685B6A5D
:10CDE000BA6A1340BB627B685B681B6A03F4C0735A
:10CDF0007B627B685B685B6A7A6A13407B627B68F4
:10CE00005B681B6A03F4FC433B627B685B685B6A9C
:10CE10003A6A13403B627B685B681B6A03F4F02349
:10CE2000FB617B685B685B6AFA691340FB617B6846
:10CE30005B685B6ABB617B685B681B6A7B61FB6AE2
:10CE4000002B07D07B685B68FA6A1A62F96A786817
:10CE500000F0DBF8BB6A002B07D07B685B68BA6A1E
:10CE60001A62B96A786800F0DBF8BB699B0903F0C5
:10CE70000103002B1AD07B699B0903F00103002BEF
:10CE800014D07B685B68DB6B1B0C9BB23B617B68DF
:10CE90005B68DB6B03F03F03FB607B685B684022F1
:10CEA0001A62FA683969786800F0C5F87B6A002B65
:10CEB00007D07B685B687A6A1A62796A786800F0E2
:10CEC000C6F83B6A002B0BD07B685B683A6A1A6233
:10CED0007B68D3F89C203B6A1A437B68C3F89C208C
:10CEE000FB69002B0BD07B685B68FA691A627B6870
:10CEF000D3F89C20FB691A437B68C3F89C207B68AD
:10CF0000D3F89C30002B02D0786800F074F800BF92
:10CF10005837BD4680BD00BF00A80040FFFFCF3F8F
:10CF200000A0004080B483B000AF7860396000BFDB
:10CF30000C37BD465DF8047B704780B483B000AF0A
:10CF40007860396000BF0C37BD465DF8047B7047E0
:10CF500080B483B000AF7860396000BF0C37BD4645
:10CF60005DF8047B704780B483B000AF786000BF89
:10CF70000C37BD465DF8047B704780B483B000AFCA
:10CF80007860396000BF0C37BD465DF8047B7047A0
:10CF900080B483B000AF7860396000BF0C37BD4605
:10CFA0005DF8047B704780B483B000AF786000BF49
:10CFB0000C37BD465DF8047B704780B483B000AF8A
:10CFC000786000BF0C37BD465DF8047B704780B4C5
:10CFD00083B000AF786000BF0C37BD465DF8047BBE
:10CFE000704780B483B000AF786000BF0C37BD4697
:10CFF0005DF8047B704780B483B000AF786000BFF9
:10D000000C37BD465DF8047B704780B483B000AF39
:10D010007860396000BF0C37BD465DF8047B70470F
:10D0200080B483B000AF7860396000BF0C37BD4674
:10D030005DF8047B704780B485B000AFF860B960DC
:10D040007A6000BF1437BD465DF8047B704780B43A
:10D0500083B000AF7860396000BF0C37BD465DF823
:10D06000047B704780B485B000AF78607B685B6BF1
:10D07000BB607B681B68D3F88420A74B1340BA6859
:10D0800091007A6812680B43C2F884307B681B6891
:10D09000D3F8843023F47F017B689B6B1A047B6890
:10D0A0001B680A43C3F884207B689B6BBA681344EF
:10D0B000BB607B681B68D3F88820974B1340BA6825
:10D0C00091007A6812680B43C2F888307B681B684D
:10D0D000D3F8883023F4FE017B68DB6B1A047B688D
:10D0E0001B680A43C3F888207B68DB6B5B00BA6867
:10D0F0001344BB607B681B68D3F8A020864B1340A9
:10D10000BA6891007A6812680B43C2F8A0307B6855
:10D110001B68D3F8A03023F4FE017B681B6C1A0453
:10D120007B681B680A43C3F8A0207B681B6C7A6885
:10D13000526C02FB03F3BA681344BB607B681B6844
:10D14000D3F8B020744B1340BA6891007A68126823
:10D150000B43C2F8B0307B681B68D3F8B03023F4BF
:10D16000FE017B689B6C1A047B681B680A43C3F84A
:10D17000B0207B689B6C7A68D26C02FB03F3BA68C0
:10D180001344BB607B681B68D3F8AC20624B134030
:10D19000BA6891007A6812680B43C2F8AC307B68B9
:10D1A0001B6D7A68526D02FB03F3BA681344BB60CF
:10D1B0007B681B68D3F8F020574B1340BA68910086
:10D1C0007A6812680B43C2F8F0307B681B68D3F8AA
:10D1D000F03023F47C117B689B6D1A047B681B681C
:10D1E0000A43C3F8F0207B689B6D5B00BA68134468
:10D1F000BB607B681B68D3F8C020474B1340BA68FC
:10D2000091007A6812680B43C2F8C0307B681B68D3
:10D21000D3F8C03023F47C117B68DB6D1A047B6883
:10D220001B680A43C3F8C0207B681B68D3F8C03072
:10D2300023F07C517B681B6E1A067B681B680A43CF
:10D24000C3F8C0207B685A6B344B13449A007B6848
:10D25000DA667B68DA6E7B689B6B9B001A447B689E
:10D260001A677B681A6F7B68DB6BDB001A447B688C
:10D270005A677B685A6F7B681B6C7968496C01FB45
:10D2800003F39B001A447B689A677B689A6F7B68FC
:10D290009B6C7968C96C01FB03F39B001A447B68A3
:10D2A000DA677B68DA6F7B681B6D7968496D01FB13
:10D2B00003F39B001A447B68C3F880207B68D3F893
:10D2C00080207B689B6DDB001A447B68C3F8842058
:10D2D0007B68D3F884207B68DB6D7968896E01FBFD
:10D2E00003F39B001A447B68C3F888207B68D3F85B
:10D2F00088207B681B6E7968896E01FB03F39B00B5
:10D300001A447B68C3F890207B68D3F89030044AB5
:10D31000934215D906E000BF0300FFFF002B001069
:10D32000FCD300407B68D3F89C3043F020027B683C
:10D33000C3F89C207B68032283F89820012310E027
:10D340007B68DB6EFB6005E0FB6800221A60FB680F
:10D350000433FB607B68D3F89030FA689A42F3D3C9
:10D36000002318461437BD465DF8047B704700BFA4
:10D3700080B489B000AFF860B9607A603B60BB6888
:10D380005B68002B0AD1BB681A69BB689B681A43AB
:10D39000BB681B689B041343FB610AE0BB681A6906
:10D3A000BB689B681A43BB681B68134343F0804308
:10D3B000FB61BB681B6A1A06BB68DB691A43BB6862
:10D3C0009B691A43BB685B691A43BB68DB681343FC
:10D3D0003B61FB68D3F88420FB689B6E396801FBD6
:10D3E00003F39B001344BB61BB69FA691A60BB6914
:10D3F0000433BB61BB693A691A60BB690433BB6122
:10D4000000237B6120E07B6903337A6813441B7837
:10D410001A067B69023379680B441B781B041A4394
:10D420007B69013379680B441B781B0213437968CD
:10D430007A690A4412781A43BB691A60BB690433DB
:10D44000BB617B6904337B61BB68DB681B0C064AEC
:10D45000D35C1A467B699342D5D300BF00BF243703
:10D46000BD465DF8047B7047EC4C040880B489B07D
:10D4700000AF786039600023FB61894B7B6194E1E8
:10D480003B681A680121FB6901FA03F313403B6111
:10D490003B69002B00F086813B685B6803F0030367
:10D4A000012B05D03B685B6803F00303022B30D1EE
:10D4B0007B689B68BB61FB695B00032202FA03F394
:10D4C000DB43BA691340BB613B68DA68FB695B0008
:10D4D00002FA03F3BA691343BB617B68BA699A60C5
:10D4E0007B685B68BB610122FB6902FA03F3DB43E3
:10D4F000BA691340BB613B685B681B0903F001021A
:10D50000FB6902FA03F3BA691343BB617B68BA692A
:10D510005A603B685B6803F00303032B17D07B68FA
:10D52000DB68BB61FB695B00032202FA03F3DB43A8
:10D53000BA691340BB613B689A68FB695B0002FAF9
:10D5400003F3BA691343BB617B68BA69DA603B686D
:10D550005B6803F00303022B23D1FB69DA087B68C5
:10D56000083253F82230BB61FB6903F007039B00CC
:10D570000F2202FA03F3DB43BA691340BB613B6835
:10D580001A69FB6903F007039B0002FA03F3BA6907
:10D590001343BB61FB69DA087B680832B96943F859
:10D5A00022107B681B68BB61FB695B00032202FAE7
:10D5B00003F3DB43BA691340BB613B685B6803F06C
:10D5C0000302FB695B0002FA03F3BA691343BB6110
:10D5D0007B68BA691A603B685B6803F44033002BD0
:10D5E00000F0E0802F4BD3F8F4302E4A43F00203D2
:10D5F000C2F8F4302B4BD3F8F43003F00203FB6095
:10D60000FB68294AFB699B08023352F82330BB614F
:10D61000FB6903F003039B000F2202FA03F3DB43D1
:10D62000BA691340BB617B68204A934252D07B6841
:10D630001F4A934231D07B681E4A93422BD07B68AD
:10D640001D4A934225D07B681C4A93421FD07B68B9
:10D650001B4A934219D07B681A4A934213D07B68C5
:10D66000194A93420DD07B68184A934207D07B68D1
:10D67000174A934201D109232DE00A232BE0082306
:10D6800029E0072327E0062325E0052323E00423E0
:10D6900021E003231FE002231DE001231BE000BF64
:10D6A000800000580044025800040058000002584E
:10D6B0000004025800080258000C025800100258DA
:10D6C0000014025800180258001C0258002002588A
:10D6D000002402580023FA6902F0030292009340EA
:10D6E000BA691343BB613849FB699B080233BA69C5
:10D6F00041F823204FF0B0431B68BB613B69DB431B
:10D70000BA691340BB613B685B6803F48013002B6C
:10D7100003D0BA693B691343BB614FF0B042BB69A8
:10D7200013604FF0B0435B68BB613B69DB43BA6990
:10D730001340BB613B685B6803F40013002B03D00C
:10D74000BA693B691343BB614FF0B042BB69536098
:10D750007B695B68BB613B69DB43BA691340BB61B2
:10D760003B685B6803F40033002B03D0BA693B6964
:10D770001343BB617B69BA695A607B691B68BB61F3
:10D780003B69DB43BA691340BB613B685B6803F4E8
:10D790008033002B03D0BA693B691343BB617B69BB
:10D7A000BA691A60FB690133FB613B681A68FB695F
:10D7B00022FA03F3002B7FF463AE00BF00BF2437CF
:10D7C000BD465DF8047B70470004005880B483B008
:10D7D00000AF78600B467B8013467B707B78002B14
:10D7E00003D07A887B689A6103E07B881A047B689F
:10D7F0009A6100BF0C37BD465DF8047B704780B46A
:10D8000085B000AF78600B467B807B685B69FB600E
:10D810007A88FB6813401A04FB68D9437B880B4065
:10D820001A437B689A6100BF1437BD465DF8047BDC
:10D830007047000080B582B000AF78607B68002B35
:10D8400001D101237FE07B6893F84130DBB2002BEC
:10D8500006D17B68002283F840207868F6F7A8F9A3
:10D860007B68242283F841207B681B681A687B68E8
:10D870001B6822F001021A607B685A687B681B688B
:10D8800022F070621A617B681B689A687B681B686B
:10D8900022F400429A607B68DB68012B07D17B6829
:10D8A0009A687B681B6842F400429A6006E07B68D5
:10D8B0009A687B681B6842F404429A607B68DB6864
:10D8C000022B04D17B681B684FF400625A607B68AE
:10D8D0001B6859687B681A681D4B0B4353607B6853
:10D8E0001B68DA687B681B6822F40042DA607B6898
:10D8F0001A697B685B6942EA03017B689B691A02CB
:10D900007B681B680A43DA607B68D9697B681A6A9E
:10D910007B681B680A431A607B681B681A687B680F
:10D920001B6842F001021A607B6800225A647B681F
:10D93000202283F841207B6800221A637B68002242
:10D9400083F84220002318460837BD4680BD00BF3B
:10D950000080000280B584B000AF78607B681B68EF
:10D960009B69FB607B681B681B68BB607B685B6BAB
:10D97000002B05D07B685B6BBA68F96878689847BC
:10D9800000BF1037BD4680BD80B586B000AF78605F
:10D990007B681B689B697B617B681B681B683B61BC
:10D9A0007B691B0A03F00103002B10D03B69DB09E4
:10D9B00003F00103002B0AD07B685B6C43F001028B
:10D9C0007B685A647B681B684FF48072DA617B69FC
:10D9D0009B0A03F00103002B10D03B69DB0903F025
:10D9E0000103002B0AD07B685B6C43F008027B6864
:10D9F0005A647B681B684FF48062DA617B695B0A5A
:10DA000003F00103002B10D03B69DB0903F0010395
:10DA1000002B0AD07B685B6C43F002027B685A647F
:10DA20007B681B684FF40072DA617B685B6CFB609B
:10DA3000FB6803F00B03002B03D0F968786800F053
:10DA400077FC00BF1837BD4680BD80B483B000AFFF
:10DA5000786000BF0C37BD465DF8047B704780B42A
:10DA600083B000AF786000BF0C37BD465DF8047B23
:10DA7000704780B483B000AF78600B46FB701346EC
:10DA80003B8000BF0C37BD465DF8047B704780B417
:10DA900083B000AF786000BF0C37BD465DF8047BF3
:10DAA000704780B483B000AF786000BF0C37BD46CC
:10DAB0005DF8047B704780B483B000AF786000BF2E
:10DAC0000C37BD465DF8047B704780B586B000AF6B
:10DAD000F860B9607A60FB68DB6A7B61BB683B61B8
:10DAE000FB6893F84030012B01D10223ECE0FB6886
:10DAF000012283F840203B695B0903F00103002BFE
:10DB000009D07B685B0903F00103002B03D039695E
:10DB1000F86800F0BFF93B691B0903F00103002B13
:10DB20004DD07B681B0903F00103002B47D0FB6835
:10DB30005B8D9BB2002B28D1FB6893F84130DBB2A0
:10DB4000282B08D17B69B3F1007F04D13969F868CB
:10DB500000F098FB32E0FB6893F84130DBB2292BF0
:10DB60000ED17B6913F5803F0AD0FB681B68102239
:10DB7000DA61F86800F0D3FCF86800F02DF91DE0D8
:10DB8000FB681B681022DA6196E0FB681B681022B4
:10DB9000DA61FB685B6C43F00402FB685A647B69E2
:10DBA000002B04D07B69B3F1807F40F08580FB6857
:10DBB0005B6C1946F86800F0BBFB7DE07CE03B69DC
:10DBC0009B0803F00103002B30D07B689B0803F017
:10DBD0000103002B2AD0FB685B8D9BB2002B18D071
:10DBE000FB681B685A6AFB685B6AD2B21A70FB68F2
:10DBF0005B6A5A1CFB685A62FB681B8D013B9AB238
:10DC0000FB681A85FB685B8D9BB2013B9AB2FB688F
:10DC10005A85FB685B8D9BB2002B4FD17B6913F556
:10DC2000803F4BD0F86800F0D7F847E03B69DB084D
:10DC300003F00103002B0AD07B68DB0803F001032B
:10DC4000002B04D03969F86800F042F837E03B69EE
:10DC50005B0803F00103002B31D07B685B0803F005
:10DC60000103002B2BD0FB685B8D9BB2002B18D0DF
:10DC7000FB685B6A1A78FB681B689A62FB685B6AE0
:10DC80005A1CFB685A62FB685B8D9BB2013B9AB2DF
:10DC9000FB685A85FB681B8D013B9AB2FB681A85AD
:10DCA0000DE07B69B3F1807F02D07B69002B06D148
:10DCB000F86800F091F802E000BF00E000BFFB68E8
:10DCC000002283F84020002318461837BD4680BD47
:10DCD00080B584B000AF786039607B6893F84130DC
:10DCE000DBB203F02803282B6AD17B681B689B6991
:10DCF0001B0CDBB203F00103FB737B681B689B69A1
:10DD00001B0C9BB203F0FE03BB817B681B689B6806
:10DD10009BB2C3F309037B817B681B68DB689BB202
:10DD200003F0FE033B817B68DB68022B38D17B89E3
:10DD3000DB099AB2BB8953409BB203F00603002B68
:10DD40001CD17B89BB817B689B6C5A1C7B689A6465
:10DD50007B689B6C022B3BD17B6800229A647B68BA
:10DD60001B680822DA617B68002283F84020BA89A8
:10DD7000FB7B19467868FFF77CFE29E03B89BB8175
:10DD80004FF40041786800F00CFC7B68002283F8B7
:10DD90004020BA89FB7B19467868FFF76AFE17E0D6
:10DDA0004FF40041786800F0FCFB7B68002283F8A8
:10DDB0004020BA89FB7B19467868FFF75AFE07E0D6
:10DDC0007B681B680822DA617B68002283F84020A8
:10DDD00000BF1037BD4680BD80B584B000AF78600D
:10DDE0007B681B681B68FB607B68002283F842200D
:10DDF000FB689B0B03F00103002B08D07B681B68BA
:10DE00001A687B681B6822F480421A600DE0FB6888
:10DE1000DB0B03F00103002B07D07B681B681A683B
:10DE20007B681B6822F400421A607B6893F84130DB
:10DE3000DBB2292B12D17B68282283F841207B6832
:10DE400021221A630121786800F0ABFB7B68002275
:10DE500083F840207868FFF7F8FD17E07B6893F8B7
:10DE60004130DBB22A2B11D17B68282283F8412074
:10DE70007B6822221A630221786800F092FB7B689B
:10DE8000002283F840207868FFF7E9FD00BF1037D3
:10DE9000BD4680BD80B586B000AF786039607B68D4
:10DEA0001B681B683B613B687B617B6893F8413072
:10DEB000FB737B681B682022DA61FB7B212B02D07D
:10DEC000FB7B292B08D148F20101786800F069FB3F
:10DED0007B6821221A630DE0FB7B222B02D0FB7BA7
:10DEE0002A2B07D148F20201786800F05AFB7B68C0
:10DEF00022221A637B681B685A687B681B6842F49D
:10DF000000425A607B681B6859687B681A68804BBE
:10DF10000B405360786800F002FB3B699B0B03F0F9
:10DF20000103002B7AD07B681B681A687B681B682A
:10DF300022F480421A607B689B6B002B00F01181F9
:10DF40007B689B6B1B68734A934259D07B689B6BC1
:10DF50001B68714A934253D07B689B6B1B686F4A66
:10DF600093424DD07B689B6B1B686D4A934247D0B0
:10DF70007B689B6B1B686B4A934241D07B689B6BB1
:10DF80001B68694A93423BD07B689B6B1B68674A5E
:10DF9000934235D07B689B6B1B68654A93422FD0B8
:10DFA0007B689B6B1B68634A934229D07B689B6BA1
:10DFB0001B68614A934223D07B689B6B1B685F4A56
:10DFC00093421DD07B689B6B1B685D4A934217D0C0
:10DFD0007B689B6B1B685B4A934211D07B689B6B91
:10DFE0001B68594A93420BD07B689B6B1B68574A4E
:10DFF000934205D07B689B6B1B68554A934205D1C1
:10E000007B689B6B1B685B689BB204E07B689B6BC7
:10E010001B685B689BB27A685385A2E03B69DB0BA7
:10E0200003F00103002B00F09C807B681B681A68DA
:10E030007B681B6822F400421A607B68DB6B002B54
:10E0400000F08F807B68DB6B1B68324A934259D0AB
:10E050007B68DB6B1B68304A934253D07B68DB6B79
:10E060001B682E4A93424DD07B68DB6B1B682C4AA1
:10E07000934247D07B68DB6B1B682A4A934241D0AE
:10E080007B68DB6B1B68284A93423BD07B68DB6B69
:10E090001B68264A934235D07B68DB6B1B68244A99
:10E0A00093422FD07B68DB6B1B68224A934229D0B6
:10E0B0007B68DB6B1B68204A934223D07B68DB6B59
:10E0C0001B681E4A93421DD07B68DB6B1B681C4A91
:10E0D000934217D07B68DB6B1B681A4A934211D0BE
:10E0E0007B68DB6B1B68184A93420BD07B68DB6B49
:10E0F0001B68164A934205D07B68DB6B1B68144A89
:10E10000934227D17B68DB6B1B685B689BB226E080
:10E1100000E800FE100002402800024040000240DB
:10E12000580002407000024088000240A0000240F7
:10E13000B80002401004024028040240400402409B
:10E14000580402407004024088040240A0040240C7
:10E15000B80402407B68DB6B1B685B689BB27A6823
:10E1600053857B699B0803F00103002B20D07B695A
:10E1700023F004037B617B681B685A6A7B685B6AD7
:10E18000D2B21A707B685B6A5A1C7B685A627B68E1
:10E190001B8D002B0CD07B681B8D013B9AB27B68DA
:10E1A0001A857B685B8D9BB2013B9AB27B685A856E
:10E1B0007B685B8D9BB2002B05D07B685B6C43F06A
:10E1C00004027B685A647B68002283F842207B68E3
:10E1D00000225A637B685B6C002B10D07B685B6C01
:10E1E0001946786800F0A4F87B6893F84130DBB2F8
:10E1F000282B41D17969786800F044F83CE07B68CD
:10E20000DB6A13F5803F14D07868FFF7E5FD7B6883
:10E210001B4ADA627B68202283F841207B68002257
:10E220001A637B68002283F840207868FFF72FFC90
:10E2300022E07B6893F84130DBB2222B0ED17B6861
:10E24000202283F841207B6800221A637B68002229
:10E2500083F840207868FFF702FC0DE07B682022FD
:10E2600083F841207B6800221A637B68002283F8D0
:10E2700040207868FFF7E9FB00BF1837BD4680BD36
:10E280000000FFFF80B582B000AF786039607B6826
:10E29000264ADA627B6800221A637B68202283F8B0
:10E2A00041207B68002283F842207B6800225A6369
:10E2B0003B689B0803F00103002B22D07B681B689E
:10E2C0005A6A7B685B6AD2B21A707B685B6A5A1CB6
:10E2D0007B685A627B681B8D002B12D07B681B8D7C
:10E2E000013B9AB27B681A857B685B8D9BB2013BD0
:10E2F0009AB27B685A857B685B6C43F004027B684A
:10E300005A6448F20301786800F04BF97B681B6897
:10E310001022DA617B68002283F840207868FFF7DA
:10E32000B6FB00BF0837BD4680BD00BF0000FFFF41
:10E3300080B584B000AF786039607B6893F8413075
:10E34000FB737B68002283F842207B685D4ADA62B7
:10E350007B6800225A857B685A6C3B681A437B684D
:10E360005A64FB7B282B05D0FB7B292B02D0FB7B3F
:10E370002A2B0BD10321786800F013F97B6828223F
:10E3800083F841207B68504A5A6311E048F2030148
:10E39000786800F006F97B6893F84130DBB2602BB7
:10E3A00003D07B68202283F841207B6800225A63D7
:10E3B0007B681B6BBB607B689B6B002B39D0BB6899
:10E3C000112B02D0BB68212B33D17B681B681B68E3
:10E3D00003F48043B3F5804F07D17B681B681A684C
:10E3E0007B681B6822F480421A607B689B6B18462E
:10E3F000FBF7ECFD0346012B17D07B689B6B334A80
:10E400001A657B68002283F840207B689B6B184666
:10E41000FAF76CFC0346002B4DD07B689B6B1B6DA1
:10E420007A68926B1046984745E0786800F050F89B
:10E4300041E07B68DB6B002B39D0BB68122B02D02C
:10E44000BB68222B33D17B681B681B6803F4004335
:10E45000B3F5004F07D17B681B681A687B681B689F
:10E4600022F400421A607B68DB6B1846FBF7AEFDB6
:10E470000346012B17D07B68DB6B144A1A657B6857
:10E48000002283F840207B68DB6B1846FAF72EFCED
:10E490000346002B11D07B68DB6B1B6D7A68D26B57
:10E4A0001046984709E0786800F012F805E07868AF
:10E4B00000F00EF802E000BF00E000BF00BF103720
:10E4C000BD4680BD0000FFFFCBDA020867E5020809
:10E4D00080B582B000AF78607B6893F84130DBB2E2
:10E4E000602B0ED17B68202283F841207B680022BC
:10E4F0001A637B68002283F840207868FFF7DBFA14
:10E5000009E07B6800221A637B68002283F84020C0
:10E510007868FFF7C6FA00BF0837BD4680BD80B4F3
:10E5200083B000AF78607B681B689B6903F00203CF
:10E53000022B03D17B681B6800229A627B681B68F0
:10E540009B6903F00103012B07D07B681B689A6964
:10E550007B681B6842F001029A6100BF0C37BD4620
:10E560005DF8047B704780B584B000AF78607B684D
:10E570009B6BFB60FB689B6B002B03D0FB689B6B6A
:10E5800000221A65FB68DB6B002B03D0FB68DB6B9A
:10E5900000221A65F868FFF79BFF00BF1037BD46E1
:10E5A00080BD80B485B000AF78600B467B800023CF
:10E5B000FB607B8803F00103002B0FD0FB6843F066
:10E5C0004203FB607B6893F84130DBB203F0280321
:10E5D000282B03D0FB6843F0B003FB607B8803F07B
:10E5E0000203002B0FD0FB6843F04403FB607B6801
:10E5F00093F84130DBB203F02803282B03D0FB68EB
:10E6000043F0B003FB60B7F90230002B03DAFB687C
:10E6100043F0B803FB607B88102B03D1FB6843F009
:10E620009003FB607B88202B03D1FB6843F0200321
:10E63000FB607B88402B03D1FB6843F04003FB6009
:10E640007B681B681968FB68DA437B681B680A40B3
:10E650001A6000BF1437BD465DF8047B704780B474
:10E6600083B000AF786039607B6893F84130DBB2EB
:10E67000202B38D17B6893F84030012B01D1022345
:10E6800032E07B68012283F840207B68242283F8F3
:10E6900041207B681B681A687B681B6822F00102B6
:10E6A0001A607B681B681A687B681B6822F48052BA
:10E6B0001A607B681B6819687B681B683A680A43A4
:10E6C0001A607B681B681A687B681B6842F001024D
:10E6D0001A607B68202283F841207B68002283F83F
:10E6E0004020002300E0022318460C37BD465DF8A9
:10E6F000047B704780B485B000AF786039607B6878
:10E7000093F84130DBB2202B39D17B6893F840304D
:10E71000012B01D1022333E07B68012283F84020E2
:10E720007B68242283F841207B681B681A687B6819
:10E730001B6822F001021A607B681B681B68FB6083
:10E74000FB6823F47063FB603B681B02FA681343A9
:10E75000FB607B681B68FA681A607B681B681A6834
:10E760007B681B6842F001021A607B68202283F8F4
:10E7700041207B68002283F84020002300E0022330
:10E7800018461437BD465DF8047B704780B483B0EB
:10E7900000AF78607B68002B01D1012317E07B6814
:10E7A00093F83D30DBB2022B04D07B6880229A665E
:10E7B00001230CE07B68042283F83D207B681B6802
:10E7C000DA687B681B6822F00102DA6000231846D1
:10E7D0000C37BD465DF8047B7047000080B584B0FF
:10E7E00000AF7860194BDB6803F00403042B0AD0F8
:10E7F000164BDB6803F007037A689A4201D00123C5
:10E800001FE000231DE0114BDB6823F007020F49D6
:10E810007B681343CB60F7F7D5FBF86009E0F7F7A7
:10E82000D1FB0246FB68D31AB3F57A7F01D90123E5
:10E8300007E0064B5B6803F40053B3F5005FEED1CD
:10E84000002318461037BD4680BD00BF004802585F
:10E8500080B586B002AF7860F7F7B4FBF8607B68EC
:10E86000002B01D101235FE07B6893F84130DBB2DC
:10E87000002B07D17868F5F78BFD41F28831786875
:10E8800000F064FA7B681B681B6823F470617B6886
:10E890009B68013B1A027B681B680A431A607B680D
:10E8A0009B6C0093FB6800222021786800F08FFAAF
:10E8B0000346FB72FB7A002B35D17B681B681A6814
:10E8C0001B4B13407A68526811067A68D26811436C
:10E8D0007A68D26911437A68126A11437A681268B9
:10E8E0000B4313607B681B685A68124B13407A68AD
:10E8F000126911047A68526911437A689269114366
:10E900007A6812680B4353607B681B681A687B68DF
:10E910001B6842F001021A607B6800225A647B681F
:10E92000012283F84120FB7A18461037BD4680BD8E
:10E930002FFFFF00FEF8E0FF80B586B000AF7860E3
:10E940007B681B689B687B617B681B681B683B61FD
:10E950007B6903F00403002B64D03B6903F480233C
:10E96000002B5FD07B681B682033FB607B6893F8CB
:10E970004130DBB2122B25D11CE07B68DB6A002B17
:10E980000FD07B685B6A1A78FB681A707B685B6AD9
:10E990005A1C7B685A627B68DB6A5A1E7B68DA62A3
:10E9A00008E07B681B681A687B681B6822F4802279
:10E9B0001A6033E07B681B689B6803F00403002B3C
:10E9C000DBD12BE07B6893F84130DBB2222B25D1E1
:10E9D0001DE07B689B6B002B10D07B681B6BFA687B
:10E9E0001278D2B21A707B681B6B5A1C7B681A6350
:10E9F0007B689B6B5A1E7B689A6308E07B681B6888
:10EA00001A687B681B6822F480221A6006E07B6823
:10EA10001B689B6803F00403002BDAD1786800F0D0
:10EA200077F93CE17B6903F00203002B00F0B08032
:10EA30003B6903F40033002B00F0AA807B681B685D
:10EA40000222DA607B681B681A687B681B6822F404
:10EA5000E0221A607B6893F84130DBB2122B20D1A0
:10EA60007B681B681B6803F00403002B11D07B68D4
:10EA70001B681A687B681B6822F004021A607B68B6
:10EA8000DB6B1B68DA687B68DB6B1B6822F00102BA
:10EA9000DA607B68012283F84120786800F02EF963
:10EAA000FAE07B6893F84130DBB2222B43D17B68DC
:10EAB0001B681B6803F00403002B12D07B681B68E3
:10EAC0001A687B681B6822F004021A607B68DB6BA3
:10EAD0001B68DA687B68DB6B1B6822F00102DA6076
:10EAE00021E07B681B682033FB6013E07B689B6B35
:10EAF000002B17D07B681B6BFA681278D2B21A70A1
:10EB00007B681B6B5A1C7B681A637B689B6B5A1E65
:10EB10007B689A637B681B689B6803F47C53002BBB
:10EB2000E4D100E000BF7B68012283F841207868CF
:10EB300000F0DAF8B0E07B6893F84130DBB2022BEA
:10EB400007D17B68012283F84120786800F0C2F881
:10EB5000A2E07B6893F84130DBB2082B40F09C8048
:10EB60007B681B685A697B681B6822F040625A61A7
:10EB70007B68012283F841207B685B6C002B03D10A
:10EB8000786800F09DF887E0786800F08FF883E0FF
:10EB90007B6903F00803002B1FD03B6903F40023BB
:10EBA000002B1AD07B681B680822DA607B681B6820
:10EBB0001B6803F48003002B0BD07B681B681A686A
:10EBC0007B681B6822F410221A607B68012283F89C
:10EBD0004120786800F0A6F861E07B6903F001034A
:10EBE000002B47D03B6903F48033002B42D07B6875
:10EBF0001B680122DA607B681B681A687B681B68E7
:10EC000022F470221A607B685B6C43F002027B681E
:10EC10005A647B681B681B6803F00403002B21D037
:10EC20007B681B681A687B681B6822F004021A6004
:10EC30007B68DB6B1C4A9A657B68DB6B1846FFF7C9
:10EC4000A5FD0346002B29D07B685B6C43F00402D2
:10EC50007B685A647B68012283F84120786800F061
:10EC600025F81BE07B68012283F84120786800F0DA
:10EC70001DF813E07B6903F01003002B0FD03B69F4
:10EC800003F48013002B0AD07B681B681022DA6023
:10EC9000786800F051F802E000BF00E000BF00BF5C
:10ECA0001837BD4680BD00BF69ED020880B483B04F
:10ECB00000AF786000BF0C37BD465DF8047B70473D
:10ECC00080B483B000AF786000BF0C37BD465DF8FC
:10ECD000047B704780B483B000AF786000BF0C370E
:10ECE000BD465DF8047B704780B483B000AF7860A8
:10ECF00000BF0C37BD465DF8047B704780B483B01D
:10ED000000AF786000BF0C37BD465DF8047B7047EC
:10ED100080B483B000AF786000BF0C37BD465DF8AB
:10ED2000047B704780B483B000AF786000BF0C37BD
:10ED3000BD465DF8047B704780B483B000AF786057
:10ED400000BF0C37BD465DF8047B704780B483B0CC
:10ED500000AF786039607B683A689A6400BF0C370E
:10ED6000BD465DF8047B704780B584B000AF786025
:10ED70007B681B6CFB60FB6800229A63FB680022C7
:10ED8000DA62FB6893F84130DBB2082B14D1FB68E0
:10ED90001B680222DA60FB681B681A68FB681B6844
:10EDA00042F400321A60FB681B681A68FB681B6833
:10EDB00042F002021A6006E0FB68012283F841205B
:10EDC000F868FFF773FF00BF1037BD4680BD80B500
:10EDD00084B000AFF860B9603B601346FB711AE085
:10EDE000BB69B3F1FF3F16D0F7F7ECF802463B687A
:10EDF000D31ABA699A4202D3BB69002B0BD1FB68C4
:10EE0000042283F84120FB685B6C43F00102FB683D
:10EE10005A6401230EE0FB681B689A68BB681340C4
:10EE2000002B14BF01230023DBB21A46FB799A4260
:10EE3000D6D1002318461037BD4680BD80B58CB0B2
:10EE400000AF78607B68002B02D1012300F01DBC6D
:10EE50007B681B6803F00103002B00F08780994B4F
:10EE60001B6903F03803FB62964B9B6ABB62FB6A2B
:10EE7000102B07D0FB6A182B10D1BB6A03F00303D9
:10EE8000022B0BD18F4B1B6803F40033002B6CD08B
:10EE90007B685B68002B68D10123F6E37B685B68C5
:10EEA000B3F5803F06D1874B1B68864A43F4803315
:10EEB00013602EE07B685B68002B0CD1814B1B68D4
:10EEC000804A23F4803313607E4B1B687D4A23F411
:10EED000802313601DE07B685B68B3F5A02F0CD125
:10EEE000784B1B68774A43F480231360754B1B688B
:10EEF000744A43F4803313600BE0724B1B68714A11
:10EF000023F4803313606F4B1B686E4A23F4802315
:10EF100013607B685B68002B13D0F7F753F87862B7
:10EF200008E0F7F74FF802467B6AD31A642B01D941
:10EF30000323AAE3634B1B6803F40033002BF0D0D8
:10EF400014E0F7F73FF8786208E0F7F73BF802467D
:10EF50007B6AD31A642B01D9032396E3594B1B68B0
:10EF600003F40033002BF0D100E000BF7B681B6886
:10EF700003F00203002B00F0CB80524B1B6903F01F
:10EF800038033B624F4B9B6AFB613B6A002B07D007
:10EF90003B6A182B56D1FB6903F00303002B51D1B8
:10EFA000484B1B6803F00403002B05D07B68DB682B
:10EFB000002B01D1012368E3424B1B6823F01902A7
:10EFC0007B68DB683F4913430B60F6F7FBFF786211
:10EFD00008E0F6F7F7FF02467B6AD31A022B01D945
:10EFE000032352E3374B1B6803F00403002BF0D0DC
:10EFF000F7F718F8034641F20302934217D87B68EB
:10F000001B69402B08D12F4B5B6823F47C332D4ABE
:10F0100043F4003353607BE02A4B5B6823F47C327B
:10F020007B681B691B03274913434B6070E0254B2A
:10F030005B6823F0FE427B681B691B062149134372
:10F040004B6065E07B68DB68002B48D01D4B1B687C
:10F0500023F019027B68DB681A4913430B60F6F74B
:10F06000B1FF786208E0F6F7ADFF02467B6AD31A7B
:10F07000022B01D9032308E3124B1B6803F004039E
:10F08000002BF0D0F6F7CEFF034641F20302934285
:10F090001AD87B681B69402B08D10A4B5B6823F4A4
:10F0A0007C33084A43F40033536031E0054B5B681E
:10F0B00023F47C327B681B691B03024913434B60BA
:10F0C00026E000BF004402589A4B5B6823F0FE42E2
:10F0D0007B681B691B06974913434B6018E0954BEF
:10F0E0001B68944A23F001031360F6F76BFF786204
:10F0F00008E0F6F767FF02467B6AD31A022B01D9B4
:10F100000323C2E28B4B1B6803F00403002BF0D1F6
:10F110007B681B6803F01003002B00F0A980854B6F
:10F120001B6903F03803BB61824B9B6A7B61BB693F
:10F13000082B07D0BB69182B3AD17B6903F0030376
:10F14000012B35D17B4B1B6803F48073002B05D05A
:10F150007B68DB69802B01D0012396E2F6F762FF22
:10F16000034641F20302934217D87B681B6A202BA7
:10F1700008D1704B5B6823F0F8436E4A43F080433C
:10F18000536075E06B4B5B6823F0F8427B681B6A49
:10F190009B06684913434B606AE0664BDB6823F0CB
:10F1A0007C527B681B6A1B0662491343CB605FE09D
:10F1B0007B68DB69002B42D05E4B1B685D4A43F0E5
:10F1C00080031360F6F7FEFE786208E0F6F7FAFEB9
:10F1D00002467B6AD31A022B01D9032355E2554B11
:10F1E0001B6803F48073002BF0D0F6F71BFF034677
:10F1F00041F20302934217D87B681B6A202B08D187
:10F200004C4B5B6823F0F8434A4A43F08043536019
:10F210002EE0484B5B6823F0F8427B681B6A9B0634
:10F22000444913434B6023E0424BDB6823F07C529C
:10F230007B681B6A1B063F491343CB6018E03D4BBC
:10F240001B683C4A23F080031360F6F7BBFE78622C
:10F2500008E0F6F7B7FE02467B6AD31A022B01D903
:10F26000032312E2334B1B6803F48073002BF0D1AD
:10F270007B681B6803F00803002B36D07B685B6952
:10F28000002B19D02B4B5B6F2A4A43F001035367C5
:10F29000F6F798FE786208E0F6F794FE02467B6A7D
:10F2A000D31A022B01D90323EFE1224B5B6F03F04A
:10F2B0000203002BF0D018E01E4B5B6F1D4A23F0B9
:10F2C00001035367F6F77EFE786208E0F6F77AFEF0
:10F2D00002467B6AD31A022B01D90323D5E1154BD1
:10F2E0005B6F03F00203002BF0D17B681B6803F017
:10F2F0002003002B39D07B689B69002B1CD00D4B61
:10F300001B680C4A43F480531360F6F75BFE786287
:10F3100008E0F6F757FE02467B6AD31A022B01D9A2
:10F320000323B2E1034B1B6803F40053002BF0D01E
:10F330001BE000BF004402589B4B1B689A4A23F411
:10F3400080531360F6F73EFE786208E0F6F73AFE67
:10F3500002467B6AD31A022B01D9032395E1924B13
:10F360001B6803F40053002BF0D17B681B6803F08B
:10F370000403002B00F081808C4B1B688B4A43F404
:10F3800080731360F6F71EFE786208E0F6F71AFE47
:10F3900002467B6AD31A642B01D9032375E1834BA0
:10F3A0001B6803F48073002BF0D07B689B68012BF3
:10F3B00006D17D4B1B6F7C4A43F0010313672DE0A0
:10F3C0007B689B68002B0CD1774B1B6F764A23F030
:10F3D00001031367744B1B6F734A23F00403136715
:10F3E0001CE07B689B68052B0CD16F4B1B6F6E4A32
:10F3F00043F0040313676C4B1B6F6B4A43F001032C
:10F4000013670BE0684B1B6F674A23F00103136718
:10F41000654B1B6F644A23F0040313677B689B688A
:10F42000002B15D0F6F7CEFD78620AE0F6F7CAFD9C
:10F4300002467B6AD31A41F28832934201D90323F0
:10F4400023E1594B1B6F03F00203002BEED014E0B5
:10F45000F6F7B8FD78620AE0F6F7B4FD02467B6A7B
:10F46000D31A41F28832934201D903230DE14E4B66
:10F470001B6F03F00203002BEED17B685B6A002B4D
:10F4800000F00281484B1B6903F03803182B00F091
:10F49000BD807B685B6A022B40F09E80424B1B68FC
:10F4A000414A23F080731360F6F78CFD786208E020
:10F4B000F6F788FD02467B6AD31A022B01D9032393
:10F4C000E3E0394B1B6803F00073002BF0D1364B9F
:10F4D0009A6A374B13407A68916A7A68D26A120145
:10F4E0000A43314913438B627B681B6B013BC3F3B7
:10F4F00008027B685B6B013B5B029BB21A437B6833
:10F500009B6B013B1B0403F4FE031A437B68DB6B1C
:10F51000013B1B0603F0FE43234913430B63224BBD
:10F52000DB6A214A23F00103D3621F4B5A6B214B44
:10F5300013407A68926CD2001B4913434B631A4BF9
:10F54000DB6A23F00C027B681B6C17491343CB6208
:10F55000154BDB6A23F002027B685B6C1249134394
:10F56000CB62114BDB6A104A43F48033D3620E4BFB
:10F57000DB6A0D4A43F40033D3620B4BDB6A0A4A61
:10F5800043F48023D362084BDB6A074A43F001034C
:10F59000D362054B1B68044A43F080731360F6F78F
:10F5A00011FD786211E000BF004402580048025883
:10F5B0000CFCFFFF0700FFFFF6F704FD02467B6A25
:10F5C000D31A022B01D903235FE0324B1B6803F0EF
:10F5D0000073002BF0D057E02E4B1B682D4A23F010
:10F5E00080731360F6F7EEFC786208E0F6F7EAFC49
:10F5F00002467B6AD31A022B01D9032345E0254B2F
:10F600001B6803F00073002BF0D13DE0214B9B6A97
:10F610003B61204B1B6BFB607B685B6A012B31D02D
:10F620003B6903F003027B689B6A9A422AD13B69DB
:10F630001B0903F03F027B68DB6A9A4222D1FB6818
:10F64000C3F308027B681B6B013B9A421AD1FB682B
:10F650005B0A03F07F027B685B6B013B9A4211D12E
:10F66000FB681B0C03F07F027B689B6B013B9A429B
:10F6700008D1FB681B0E03F07F027B68DB6B013B4C
:10F680009A4201D0012300E0002318463037BD46DE
:10F6900080BD00BF0044025880B586B000AF7860DE
:10F6A00039607B68002B01D101239CE18A4B1B68E8
:10F6B00003F00F033A689A4210D9874B1B6823F076
:10F6C0000F0285493B6813430B60834B1B6803F0B3
:10F6D0000F033A689A4201D0012384E17B681B68DA
:10F6E00003F00403002B10D07B681A697B4B9B69E5
:10F6F00003F070039A4208D9784B9B6923F070029B
:10F700007B681B69754913438B617B681B6803F039
:10F710000803002B10D07B685A69704BDB6903F03B
:10F7200070039A4208D96D4BDB6923F070027B6845
:10F730005B696A491343CB617B681B6803F0100364
:10F74000002B10D07B689A69644BDB6903F4E0639B
:10F750009A4208D9614BDB6923F4E0627B689B69BC
:10F760005E491343CB617B681B6803F02003002BC9
:10F7700010D07B68DA69594B1B6A03F070039A4218
:10F7800008D9564B1B6A23F070027B68DB6953492A
:10F7900013430B627B681B6803F00203002B10D03D
:10F7A0007B68DA684D4B9B6903F00F039A4208D9D6
:10F7B0004A4B9B6923F00F027B68DB684749134380
:10F7C0008B617B681B6803F00103002B55D0434B12
:10F7D0009B6923F470627B689B68404913438B618B
:10F7E0007B685B68022B07D13C4B1B6803F400333A
:10F7F000002B21D10123F6E07B685B68032B07D146
:10F80000364B1B6803F00073002B15D10123EAE08F
:10F810007B685B68012B07D1304B1B6803F4807356
:10F82000002B09D10123DEE02C4B1B6803F00403FD
:10F83000002B01D10123D6E0284B1B6923F00702DE
:10F840007B685B68254913430B61F6F7BBFB786166
:10F850000AE0F6F7B7FB02467B69D31A41F2883219
:10F86000934201D90323BEE01C4B1B6903F038020D
:10F870007B685B68DB009A42EBD17B681B6803F016
:10F880000203002B10D07B68DA68144B9B6903F0ED
:10F890000F039A4208D2114B9B6923F00F027B6839
:10F8A000DB680E4913438B610B4B1B6803F00F039E
:10F8B0003A689A4214D2084B1B6823F00F0206499B
:10F8C0003B6813430B60044B1B6803F00F033A685B
:10F8D0009A4205D0012386E00020005200440258DD
:10F8E0007B681B6803F00403002B10D07B681A6947
:10F8F0003F4B9B6903F070039A4208D23C4B9B69D3
:10F9000023F070027B681B69394913438B617B6864
:10F910001B6803F00803002B10D07B685A69344B36
:10F92000DB6903F070039A4208D2314BDB6923F0A4
:10F9300070027B685B692E491343CB617B681B684F
:10F9400003F01003002B10D07B689A69284BDB6909
:10F9500003F4E0639A4208D2254BDB6923F4E062AA
:10F960007B689B6922491343CB617B681B6803F06A
:10F970002003002B10D07B68DA691D4B1B6A03F053
:10F9800070039A4208D21A4B1B6A23F070027B68FC
:10F99000DB69174913430B6200F034F80246144B3D
:10F9A0009B691B0A03F00F031249CB5C03F01F0392
:10F9B00022FA03F33B610E4B9B6903F00F030D4AE0
:10F9C000D35C03F01F033A6922FA03F30A4A136077
:10F9D0000A4A3B6913600A4B1B681846F6F7A8FAF7
:10F9E0000346FB73FB7B18461837BD4680BD00BF3E
:10F9F00000440258D44C04084C0000244800002461
:10FA00005000002480B489B000AFB34B1B6903F0F1
:10FA10003803182B00F2558101A252F823F000BFE1
:10FA200085FA0208C3FC0208C3FC0208C3FC0208F2
:10FA3000C3FC0208C3FC0208C3FC0208C3FC0208A2
:10FA4000ABFA0208C3FC0208C3FC0208C3FC0208AC
:10FA5000C3FC0208C3FC0208C3FC0208C3FC020882
:10FA6000B1FA0208C3FC0208C3FC0208C3FC020886
:10FA7000C3FC0208C3FC0208C3FC0208C3FC020862
:10FA8000B7FA0208944B1B6803F02003002B09D03F
:10FA9000914B1B68DB0803F00303904A22FA03F33F
:10FAA000BB6111E18D4BBB610EE18D4BBB610BE185
:10FAB0008C4BBB6108E1884B9B6A03F003037B61BD
:10FAC000854B9B6A1B0903F03F033B61824BDB6A5A
:10FAD00003F00103FB60804B5B6BDB08C3F30C039B
:10FAE000FA6802FB03F307EE903AF8EE677AC7ED87
:10FAF000027A3B69002B00F0E1807B69022B00F069
:10FB000083807B69022B00F2A1807B69002B03D0EC
:10FB10007B69012B56D099E06F4B1B6803F02003E3
:10FB2000002B2DD06C4B1B68DB0803F003036B4AE2
:10FB300022FA03F37B607B6807EE903AF8EE676A7F
:10FB40003B6907EE903AF8EE677A86EEA77A624B49
:10FB50001B6BC3F3080307EE903AF8EE676A97ED64
:10FB6000026ADFED615AC6EE257A76EEA77AF7EEE5
:10FB7000006A77EEA67A67EE277AC7ED077A87E004
:10FB80003B6907EE903AF8EE677ADFED586A86EE49
:10FB9000A77A514B1B6BC3F3080307EE903AF8EEBC
:10FBA000676A97ED026ADFED505AC6EE257A76EE67
:10FBB000A77AF7EE006A77EEA67A67EE277AC7EDA6
:10FBC000077A65E03B6907EE903AF8EE677ADFED79
:10FBD000486A86EEA77A404B1B6BC3F3080307EE17
:10FBE000903AF8EE676A97ED026ADFED3F5AC6EE8B
:10FBF000257A76EEA77AF7EE006A77EEA67A67EEB8
:10FC0000277AC7ED077A43E03B6907EE903AF8EEB2
:10FC1000677ADFED386A86EEA77A2F4B1B6BC3F34A
:10FC2000080307EE903AF8EE676A97ED026ADFED97
:10FC30002E5AC6EE257A76EEA77AF7EE006A77EEB0
:10FC4000A67A67EE277AC7ED077A21E03B6907EECF
:10FC5000903AF8EE677ADFED266A86EEA77A1E4BB9
:10FC60001B6BC3F3080307EE903AF8EE676A97ED53
:10FC7000026ADFED1D5AC6EE257A76EEA77AF7EE18
:10FC8000006A77EEA67A67EE277AC7ED077A00BF9B
:10FC9000114B1B6B5B0A03F07F0301333B603B6836
:10FCA00007EE903AB8EE677AD7ED076AC6EE877A24
:10FCB000FCEEE77A17EE903ABB6105E00023BB61EA
:10FCC00002E0074BBB6100BFBB6918462437BD4645
:10FCD0005DF8047B704700BF004402580090D003D9
:10FCE00000093D0040787D01000000460024744C6E
:10FCF0000024744A20BCBE4B80B582B000AFFFF731
:10FD000081FE0246104B9B691B0A03F00F030F494B
:10FD1000CB5C03F01F0322FA03F37B600A4B9B6961
:10FD200003F00F03094AD35C03F01F037A6822FA39
:10FD300003F3074A1360074A7B681360044B1B6890
:10FD400018460837BD4680BD00440258D44C04080C
:10FD50004C0000244800002480B500AFFFF7CCFF22
:10FD60000246064BDB691B0903F007030449CB5C21
:10FD700003F01F0322FA03F3184680BD0044025823
:10FD8000D44C040880B500AFFFF7B6FF0246064B1F
:10FD9000DB691B0A03F007030449CB5C03F01F0374
:10FDA00022FA03F3184680BD00440258D44C0408DC
:10FDB00080B586B000AF78600023FB750023BB756B
:10FDC0007B681B6803F00063002B3FD07B685B6E91
:10FDD000B3F5401F2AD0B3F5401F24D8B3F5001F58
:10FDE00018D0B3F5001F1ED8002B03D0B3F5801F29
:10FDF00007D018E0A34BDB6AA24A43F40033D36276
:10FE000015E07B6804330221184601F0F9FF034630
:10FE1000FB750CE07B6824330221184602F0A2F83F
:10FE20000346FB7503E00123FB7500E000BFFB7D8B
:10FE3000002B09D1934B1B6D23F440127B685B6E42
:10FE4000904913430B6501E0FB7DBB757B681B6824
:10FE500003F48073002B3DD07B685B6D042B26D8A8
:10FE600001A252F823F000BF7DFE02088BFE0208BB
:10FE70009DFE0208B5FE0208B5FE0208814BDB6A52
:10FE8000804A43F40033D36215E07B6804330021D9
:10FE9000184601F0B5FF0346FB750CE07B68243380
:10FEA0000021184602F05EF80346FB7503E00123CB
:10FEB000FB7500E000BFFB7D002B09D1714B1B6D72
:10FEC00023F007027B685B6D6E4913430B6501E00D
:10FED000FB7DBB757B681B6803F40073002B42D06D
:10FEE0007B689B6DB3F5807F2BD0B3F5807F25D8E1
:10FEF000C02B28D0C02B21D8802B16D0802B1DD80A
:10FF0000002B02D0402B07D018E05E4BDB6A5D4A25
:10FF100043F40033D36217E07B68043300211846B2
:10FF200001F06EFF0346FB750EE07B682433002171
:10FF3000184602F017F80346FB7505E00123FB7530
:10FF400002E000BF00E000BFFB7D002B09D14D4B5C
:10FF50001B6D23F4E0727B689B6D4A4913430B656C
:10FF600001E0FB7DBB757B681B6803F48063002B9D
:10FF700049D07B68D3F8A430B3F5000F30D0B3F587
:10FF8000000F2AD8B3F5C00F2CD0B3F5C00F24D87A
:10FF9000B3F5800F18D0B3F5800F1ED8002B03D017
:10FFA000B3F5001F07D018E0364BDB6A354A43F43F
:10FFB0000033D36217E07B6804330021184601F058
:10FFC0001FFF0346FB750EE07B68243300211846B3
:10FFD00001F0C8FF0346FB7505E00123FB7502E055
:10FFE00000BF00E000BFFB7D002B0AD1254B9B6DBD
:10FFF00023F460027B68D3F8A430224913438B6555
:020000040803EF
:1000000001E0FB7DBB757B681B6803F40063002B7C
:100010004BD07B68D3F8A830B3F1806F30D0B3F108
:10002000806F2AD8B3F1407F2ED0B3F1407F24D81F
:10003000B3F1007F18D0B3F1007F1ED8002B03D09E
:10004000B3F1807F07D018E00E4BDB6A0D4A43F412
:100050000033D36219E07B6804330021184601F0B5
:10006000CFFE0346FB7510E07B6824330021184661
:1000700001F078FF0346FB7507E00123FB7504E000
:1000800000BF02E00044025800BFFB7D002B0AD1F4
:10009000994B9B6D23F0E0627B68D3F8A8309649BA
:1000A00013438B6501E0FB7DBB757B681B6803F028
:1000B0000073002B32D07B689B6C302B1CD0302B14
:1000C00017D8202B0CD0202B13D8002B16D0102B98
:1000D0000FD1894BDB6A884A43F40033D3620EE0C8
:1000E0007B6804330221184601F08AFE0346FB7543
:1000F00005E00123FB7502E000BF00E000BFFB7DCF
:10010000002B09D17C4BDB6C23F030027B689B6CAD
:1001100079491343CB6401E0FB7DBB757B681B68A9
:1001200003F48053002B47D07B68DB6DB3F5804F21
:1001300030D0B3F5804F2AD8B3F5405F2CD0B3F55B
:10014000405F24D8B3F5005F18D0B3F5005F1ED828
:10015000002B03D0B3F5805F07D018E0664BDB6A55
:10016000654A43F40033D36217E07B68043300210F
:10017000184601F045FE0346FB750EE07B6824330C
:100180000021184601F0EEFE0346FB7505E0012351
:10019000FB7502E000BF00E000BFFB7D002B09D132
:1001A000554B1B6D23F4E0427B68DB6D52491343D2
:1001B0000B6501E0FB7DBB757B681B6803F4005396
:1001C000002B49D07B681B6EB3F5A02F2ED0B3F562
:1001D000A02F28D8B3F5802F2AD0B3F5802F22D8AE
:1001E000B3F5403F26D0B3F5403F1CD8B3F5003FF0
:1001F00010D0B3F5003F16D8002B1DD0B3F5803FCB
:1002000011D17B6804330121184601F0F9FD034642
:10021000FB7512E07B6824330121184601F0A2FE31
:100220000346FB7509E00123FB7506E000BF04E00F
:1002300000BF02E000BF00E000BFFB7D002B09D142
:100240002D4B1B6D23F4E0227B681B6E2A49134360
:100250000B6501E0FB7DBB757B681B6803F4804385
:10026000002B4DD07B68D3F8AC30B3F1A04F2ED02B
:10027000B3F1A04F28D8B3F1804F2AD0B3F1804F0B
:1002800022D8B3F1405F26D0B3F1405F1CD8B3F160
:10029000005F10D0B3F1005F16D8002B1DD0B3F172
:1002A000805F11D17B6804330121184601F0A8FD5D
:1002B0000346FB7512E07B6824330121184601F0E8
:1002C00051FE0346FB7509E00123FB7506E000BF04
:1002D00004E000BF02E000BF00E000BFFB7D002B98
:1002E0000CD1054B9B6D23F0E0427B68D3F8AC301A
:1002F000014913438B6503E000440258FB7DBB7545
:100300007B681B6803F40043002B2FD07B68DB6EF7
:10031000B3F1005F0ED0B3F1005F14D8002B15D0FD
:10032000B3F1805F0FD1AF4BDB6AAE4A43F40033C9
:10033000D3620CE07B6804330121184601F060FDB4
:100340000346FB7503E00123FB7500E000BFFB7D66
:10035000002B09D1A34B1B6D23F040527B68DB6E51
:10036000A04913430B6501E0FB7DBB757B681B68EF
:1003700003F08073002B32D07B685B6C032B1BD89F
:1003800001A252F823F000BFBF030308990303083A
:10039000A7030308BF030308924BDB6A914A43F4A7
:1003A0000033D3620CE07B6804330221184601F06D
:1003B00027FD0346FB7503E00123FB7500E000BF4A
:1003C000FB7D002B09D1874BDB6C23F003027B689C
:1003D0005B6C84491343CB6401E0FB7DBB757B6898
:1003E0001B6803F48003002B00F086807E4B1B68A3
:1003F0007D4A43F480731360F5F7E4FD386109E04A
:10040000F5F7E0FD02463B69D31A642B02D90323BA
:10041000FB7505E0744B1B6803F48073002BEFD071
:10042000FB7D002B66D16F4B1A6F7B68D3F8B03021
:10043000534003F44073002B13D06A4B1B6F23F41B
:100440004073FB60674B1B6F664A43F4803313674E
:10045000644B1B6F634A23F480331367614AFB6864
:1004600013677B68D3F8B030B3F5807F15D1F5F70B
:10047000A9FD38610BE0F5F7A5FD02463B69D31AEB
:1004800041F28832934202D90323FB7505E0554BB4
:100490001B6F03F00203002BEDD0FB7D002B26D158
:1004A0007B68D3F8B03003F44073B3F5407F0DD1CF
:1004B0004C4B1B6923F47C527B68D3F8B03019098C
:1004C0004A4B0B40474913430B6105E0454B1B6901
:1004D000444A23F47C531361424B1A6F7B68D3F870
:1004E000B030C3F30B033F4913430B6704E0FB7DBC
:1004F000BB7501E0FB7DBB757B681B6803F00103E6
:10050000002B00F085807B689B6F282B66D801A2AA
:1005100052F823F0F1050308DD050308DD050308A3
:10052000DD050308DD050308DD050308DD05030817
:10053000DD050308B9050308DD050308DD0503082B
:10054000DD050308DD050308DD050308DD050308F7
:10055000DD050308CB050308DD050308DD050308F9
:10056000DD050308DD050308DD050308DD050308D7
:10057000DD050308F1050308DD050308DD050308B3
:10058000DD050308DD050308DD050308DD050308B7
:10059000DD050308F1050308DD050308DD05030893
:1005A000DD050308DD050308DD050308DD05030897
:1005B000DD050308F10503087B68043301211846B3
:1005C00001F01EFC0346FB7513E07B682433012118
:1005D000184601F0C7FC0346FB750AE00123FB75D2
:1005E00007E000BF0044025800480258CFFFFF0058
:1005F00000BFFB7D002B09D1964B5B6D23F03802C9
:100600007B689B6F934913434B6501E0FB7DBB7592
:100610007B681B6803F00203002B38D07B685B6F9C
:10062000052B21D801A252F823F000BF6F06030862
:1006300045060308570603086F0603086F060308FC
:100640006F0603087B6804330121184601F0D8FBCC
:100650000346FB750CE07B6824330121184601F04A
:1006600081FC0346FB7503E00123FB7500E000BF3E
:10067000FB7D002B09D1774B5B6D23F007027B6874
:100680005B6F744913434B6501E0FB7DBB757B6871
:100690001B6803F00403002B3AD07B68D3F890303A
:1006A000052B21D801A252F823F000BFEF06030862
:1006B000C5060308D7060308EF060308EF0603087C
:1006C000EF0603087B6804330121184601F098FB0C
:1006D0000346FB750CE07B6824330121184601F0CA
:1006E00041FC0346FB7503E00123FB7500E000BFFE
:1006F000FB7D002B0AD1574B9B6D23F007027B68D3
:10070000D3F89030534913438B6501E0FB7DBB75F3
:100710007B681B6803F02003002B4BD07B68D3F869
:100720008C30B3F1A04F2ED0B3F1A04F28D8B3F145
:10073000804F2AD0B3F1804F22D8B3F1405F26D04A
:10074000B3F1405F1CD8B3F1005F10D0B3F1005F8C
:1007500016D8002B1DD0B3F1805F11D17B68043314
:100760000021184601F04CFB0346FB7512E07B6844
:1007700024330221184601F0F5FB0346FB7509E01E
:100780000123FB7506E000BF04E000BF02E000BFEC
:1007900000E000BFFB7D002B0AD12E4B5B6D23F0E8
:1007A000E0427B68D3F88C302A4913434B6501E063
:1007B000FB7DBB757B681B6803F04003002B4DD0AD
:1007C0007B68D3F89830B3F5A05F2ED0B3F5A05F67
:1007D00028D8B3F5805F2AD0B3F5805F22D8B3F56F
:1007E000406F26D0B3F5406F1CD8B3F5006F10D022
:1007F000B3F5006F16D8002B1DD0B3F5806F11D163
:100800007B6804330021184601F0FAFA0346FB75B1
:1008100012E07B6824330221184601F0A3FB034653
:10082000FB7509E00123FB7506E000BF04E000BF93
:1008300002E000BF00E000BFFB7D002B0CD1054BA8
:100840009B6D23F4E0527B68D3F898300149134341
:100850008B6503E000440258FB7DBB757B681B6819
:1008600003F08003002B4BD07B68D3F89C30B3F5AA
:10087000204F2ED0B3F5204F28D8B3F5004F2AD003
:10088000B3F5004F22D8B3F5C04F26D0B3F5C04F13
:100890001CD8B3F5804F10D0B3F5804F16D8002B7D
:1008A0001DD0B3F5005F11D17B68043300211846D9
:1008B00001F0A6FA0346FB7512E07B68243302219F
:1008C000184601F04FFB0346FB7509E00123FB7559
:1008D00006E000BF04E000BF02E000BF00E000BF90
:1008E000FB7D002B0AD19D4B9B6D23F460427B68FE
:1008F000D3F89C30994913438B6501E0FB7DBB75B0
:100900007B681B6803F00803002B1AD07B68D3F8C0
:100910008030B3F5805F0AD17B682433022118460A
:1009200001F020FB0346002B01D00123BB758B4B4C
:100930005B6D23F440527B68D3F8803087491343C2
:100940004B657B681B6803F01003002B1AD07B6893
:10095000D3F89430B3F5807F0AD17B682433022129
:10096000184601F0FFFA0346002B01D00123BB75A6
:100970007A4B9B6D23F440727B68D3F894307749AF
:1009800013438B657B681B6803F40023002B34D072
:100990007B68D3F8A030B3F5003F1DD0B3F5003F1E
:1009A00017D8002B03D0B3F5803F09D011E07B6846
:1009B00004330021184601F023FA0346FB750CE0CE
:1009C0007B6824330221184601F0CCFA0346FB75FC
:1009D00003E00123FB7500E000BFFB7D002B0AD183
:1009E0005E4B9B6D23F440327B68D3F8A0305B49AB
:1009F00013438B6501E0FB7DBB757B681B6803F4CB
:100A00008023002B33D07B68D3F88430B3F5401FAC
:100A10001CD0B3F5401F16D8B3F5801F03D0B3F533
:100A2000001F07D00FE04D4BDB6A4C4A43F4003304
:100A3000D3620CE07B6824330121184601F092FA5E
:100A40000346FB7503E00123FB7500E000BFFB7D5F
:100A5000002B0AD1414B5B6D23F440127B68D3F825
:100A600084303E4913434B6501E0FB7DBB757B68D9
:100A70001B6803F48033002B29D07B68DB6C002BD0
:100A800003D0B3F5803F07D00FE0344BDB6A334A25
:100A900043F40033D3620BE07B6804330221184631
:100AA00001F0AEF90346FB7502E00123FB7500BFC0
:100AB000FB7D002B09D1294BDB6C23F480327B6852
:100AC000DB6C26491343CB6401E0FB7DBB757B687F
:100AD0001B6803F00053002B0AD07B6824330221EB
:100AE000184601F03FFA0346002B01D00123BB75E5
:100AF0007B681B6803F40033002B33D07B68DB6F0B
:100B0000B3F5407F17D0B3F5407F11D8B3F5007F20
:100B100013D0B3F5007F0BD8002B10D0B3F5807F36
:100B200006D10E4BDB6A0D4A43F40033D36207E073
:100B30000123FB7504E000BF02E000BF00E000BF3E
:100B4000FB7D002B0CD1054B5B6D23F440727B6861
:100B5000DB6F024913434B6504E000BF00440258B9
:100B6000FB7DBB757B681B6803F48013002B08D0EA
:100B7000314B1B6D23F000427B681B6F2E491343E2
:100B80000B657B681B6803F08053002B09D02A4B50
:100B90001B6923F480427B68D3F8B43026491343A1
:100BA0000B617B681B6803F40013002B08D0224BF9
:100BB0001B6D23F080727B689B6E1F4913430B658E
:100BC0007B681B6803F08043002B0DD01A4B1B6918
:100BD000194A23F400431361174B1A697B68D3F851
:100BE000B830154913430B617B681B68002B08DA8A
:100BF000114BDB6C23F040527B681B6D0E49134395
:100C0000CB647B681B6803F40003002B09D00A4BFC
:100C10005B6D23F440027B68D3F8883006491343A8
:100C20004B65BB7D002B01D1002300E0012318465A
:100C30001837BD4680BD00BF0044025880B590B053
:100C400000AF78607B68B3F5807F40F09580974B6C
:100C50001B6D03F007033B633B6B042B00F28880A2
:100C600001A252F823F000BF7D0C0308A50C030875
:100C7000CD0C0308690D0308F50C03088B4B1B68AA
:100C800003F00073B3F1007F08D107F12403184685
:100C900000F064FFBB6AFB6300F094BC0023FB63BD
:100CA00000F090BC814B1B6803F00063B3F1006F50
:100CB00008D107F11803184600F0A8FCBB69FB63D4
:100CC00000F080BC0023FB6300F07CBC774B1B680A
:100CD00003F00053B3F1005F08D107F10C0318468D
:100CE00000F0E8FDFB68FB6300F06CBC0023FB63D5
:100CF00000F068BC6D4BDB6C03F040537B636B4BC7
:100D00001B6803F00403042B0CD17B6B002B09D16F
:100D1000664B1B68DB0803F00303654A22FA03F302
:100D2000FB631FE0614B1B6803F48073B3F5807FA6
:100D300006D17B6BB3F1805F02D15E4BFB6311E0A8
:100D40005A4B1B6803F40033B3F5003F06D17B6BAD
:100D5000B3F1005F02D1584BFB6303E00023FB6358
:100D600000F030BC00F02EBC544BFB6300F02ABCFA
:100D70000023FB6300F026BC7B68B3F5007F40F0E6
:100D80009F804A4B1B6D03F4E0733B633B6BB3F5F1
:100D9000807F4DD03B6BB3F5807F00F284803B6B4E
:100DA000C02B7DD03B6BC02B7DD83B6B802B2DD0D7
:100DB0003B6B802B77D83B6B002B03D03B6B402BDE
:100DC00012D070E0394B1B6803F00073B3F1007F61
:100DD00007D107F12403184600F0C0FEBB6AFB638D
:100DE000F0E30023FB63EDE3304B1B6803F000638B
:100DF000B3F1006F07D107F11803184600F006FCA5
:100E0000BB69FB63DEE30023FB63DBE3274B1B686B
:100E100003F00053B3F1005F07D107F10C0318464C
:100E200000F048FDFB68FB63CCE30023FB63C9E3F0
:100E30001E4BDB6C03F040537B631C4B1B6803F0C1
:100E40000403042B0CD17B6B002B09D1174B1B68BF
:100E5000DB0803F00303164A22FA03F3FB631EE0E8
:100E6000124B1B6803F48073B3F5807F06D17B6B54
:100E7000B3F1805F02D10F4BFB6310E00B4B1B689B
:100E800003F40033B3F5003F06D17B6BB3F1005F91
:100E900002D1094BFB6302E00023FB6392E391E381
:100EA000064BFB638EE30023FB638BE30044025895
:100EB0000090D00300093D0040787D010080BB0018
:100EC0007B68B3F5806F40F09C809D4B9B6D03F475
:100ED00060033B633B6BB3F5000F54D03B6BB3F542
:100EE000000F00F28B803B6BB3F5C00F00F08380E6
:100EF0003B6BB3F5C00F00F281803B6BB3F5800F05
:100F00002FD03B6BB3F5800F78D83B6B002B04D010
:100F10003B6BB3F5001F12D070E0894B1B6803F0E8
:100F20000073B3F1007F07D107F12403184600F0E6
:100F300015FEBB6AFB6345E30023FB6342E3804B82
:100F40001B6803F00063B3F1006F07D107F11803CA
:100F5000184600F05BFBBB69FB6333E30023FB63D4
:100F600030E3774B1B6803F00053B3F1005F07D108
:100F700007F10C03184600F09DFCFB68FB6321E3BE
:100F80000023FB631EE36E4BDB6C03F040537B637B
:100F90006B4B1B6803F00403042B0CD17B6B002B01
:100FA00009D1674B1B68DB0803F00303654A22FA8B
:100FB00003F3FB631EE0624B1B6803F48073B3F51D
:100FC000807F06D17B6BB3F1805F02D15E4BFB6308
:100FD00010E05B4B1B6803F40033B3F5003F06D110
:100FE0007B6BB3F1005F02D1584BFB6302E000233F
:100FF000FB63E7E2E6E2564BFB63E3E20023FB63BD
:10100000E0E27B68B3F5006F40F0A7804C4B9B6D2E
:1010100003F0E0633B633B6BB3F1806F55D03B6BF8
:10102000B3F1806F00F296803B6BB3F1407F00F02C
:1010300084803B6BB3F1407F00F28C803B6BB3F15B
:10104000007F30D03B6BB3F1007F00F283803B6BBD
:10105000002B04D03B6BB3F1807F12D07AE0384B89
:101060001B6803F00073B3F1007F07D107F124037D
:10107000184600F073FDBB6AFB63A3E20023FB6329
:10108000A0E22F4B1B6803F00063B3F1006F07D1A0
:1010900007F11803184600F0B9FABB69FB6391E247
:1010A0000023FB638EE2264B1B6803F00053B3F171
:1010B000005F07D107F10C03184600F0FBFBFB684B
:1010C000FB637FE20023FB637CE21D4BDB6C03F0E0
:1010D00040537B631A4B1B6803F00403042B0CD1B1
:1010E0007B6B002B09D1164B1B68DB0803F0030355
:1010F000144A22FA03F3FB631EE0114B1B6803F44E
:101100008073B3F5807F06D17B6BB3F1805F02D132
:101110000D4BFB6310E00A4B1B6803F40033B3F57F
:10112000003F06D17B6BB3F1005F02D1074BFB633D
:1011300002E00023FB6345E244E2054BFB6341E22E
:10114000004402580090D00300093D0040787D0122
:101150000080BB000023FB6334E27B68B3F5805F53
:1011600040F09C809B4B1B6D03F4E043BB63BB6B67
:10117000B3F5804F54D0BB6BB3F5804F00F28B803A
:10118000BB6BB3F5405F00F08380BB6BB3F5405F92
:1011900000F28180BB6BB3F5005F2FD0BB6BB3F562
:1011A000005F78D8BB6B002B04D0BB6BB3F5805FBE
:1011B00012D070E0874B1B6803F00073B3F1007F1F
:1011C00007D107F12403184600F0C8FCBB6AFB6393
:1011D000F8E10023FB63F5E17E4B1B6803F000633D
:1011E000B3F1006F07D107F11803184600F00EFAAB
:1011F000BB69FB63E6E10023FB63E3E1754B1B681E
:1012000003F00053B3F1005F07D107F10C03184658
:1012100000F050FBFB68FB63D4E10023FB63D1E1EA
:101220006C4BDB6C03F040537B636A4B1B6803F031
:101230000403042B0CD17B6B002B09D1654B1B687D
:10124000DB0803F00303644A22FA03F3FB631EE0A6
:10125000604B1B6803F48073B3F5807F06D17B6B12
:10126000B3F1805F02D15D4BFB6310E0594B1B680B
:1012700003F40033B3F5003F06D17B6BB3F1005F9D
:1012800002D1574BFB6302E00023FB639AE199E133
:10129000544BFB6396E10023FB6393E17B68B3F55A
:1012A000002F73D14B4B9B6D03F44033BB63BB6B7F
:1012B000B3F5003F2FD0BB6BB3F5003F63D8BB6BDA
:1012C000002B04D0BB6BB3F5803F12D05BE0414BE9
:1012D0001B6803F00063B3F1006F07D107F1180337
:1012E000184600F093F9BB69FB636BE10023FB63D5
:1012F00068E1384B1B6803F00053B3F1005F07D17E
:1013000007F10C03184600F0D5FA7B69FB6359E13D
:101310000023FB6356E12F4BDB6C03F040537B63F0
:101320002C4B1B6803F00403042B0CD17B6B002BAC
:1013300009D1284B1B68DB0803F00303264A22FA75
:1013400003F3FB631EE0234B1B6803F48073B3F5C8
:10135000807F06D17B6BB3F1805F02D11F4BFB63B3
:1013600010E01C4B1B6803F40033B3F5003F06D1BB
:101370007B6BB3F1005F02D1194BFB6302E00023EA
:10138000FB631FE11EE10023FB631BE17B68B3F5F8
:10139000803F3ED10F4BDB6C03F48033BB63BB6BF0
:1013A000002B04D0BB6BB3F5803F1DD02EE0094B62
:1013B0001B6803F00073B3F1007F07D107F124032A
:1013C000184600F0CBFBBB6AFB63FBE00023FB632A
:1013D000F8E000BF004402580090D00300093D002F
:1013E00040787D010080BB00794B1B6803F00063EF
:1013F000B3F1006F07D107F11803184600F006F9A2
:101400003B6AFB63DEE00023FB63DBE00023FB635E
:10141000D8E07B68B3F5804F40F085806C4B9B6DC6
:1014200003F0E043BB63BB6BB3F1A04F6BD0BB6B6E
:10143000B3F1A04F74D8BB6BB3F1804F56D0BB6BE8
:10144000B3F1804F6CD8BB6BB3F1405F3BD0BB6B4B
:10145000B3F1405F64D8BB6BB3F1005F21D0BB6BCD
:10146000B3F1005F5CD8BB6B002B04D0BB6BB3F156
:10147000805F04D054E000F0B3F8F863A2E0544B6E
:101480001B6803F00063B3F1006F07D107F1180385
:10149000184600F0BBF8FB69FB6393E00023FB6395
:1014A00090E04B4B1B6803F00053B3F1005F07D192
:1014B00007F10C03184600F0FDF93B69FB6381E07E
:1014C0000023FB637EE0424B1B6803F00403042B04
:1014D00009D13F4B1B68DB0803F003033D4A22FAA6
:1014E00003F3FB636EE00023FB636BE0384B1B6888
:1014F00003F48073B3F5807F02D1374BFB6361E067
:101500000023FB635EE0324B1B6803F40033B3F54A
:10151000003F02D1314BFB6354E00023FB6351E0F9
:101520000023FB634EE07B68B3F5004F48D1284BA6
:101530001B6D03F04053BB63BB6BB3F1005F2AD05C
:10154000BB6BB3F1005F38D8BB6B002B04D0BB6B17
:10155000B3F1805F0DD030E01D4B1B6803F4003306
:10156000B3F5003F02D11D4BFB632BE00023FB636F
:1015700028E0174B1B6803F00073B3F1007F07D11D
:1015800007F12403184600F0E9FABB6AFB6319E08F
:101590000023FB6316E00E4B1B6803F00063B3F1FE
:1015A000006F07D107F11803184600F02FF8FB6908
:1015B000FB6307E00023FB6304E00023FB6301E01F
:1015C0000023FB63FB6B18464037BD4680BD00BF60
:1015D000004402580090D00300093D0040787D018E
:1015E00080B500AFFEF788FB0246064B1B6A1B095D
:1015F00003F007030449CB5C03F01F0322FA03F353
:10160000184680BD00440258D44C040880B489B008
:1016100000AF7860A14B9B6A03F00303BB619F4B53
:101620009B6A1B0B03F03F037B619C4BDB6A1B092E
:1016300003F001033B61994BDB6BDB08C3F30C0345
:101640003A6902FB03F307EE903AF8EE677AC7EDCA
:10165000037A7B69002B00F01181BB69022B00F03B
:101660008380BB69022B00F2A180BB69002B03D0F1
:10167000BB69012B56D099E0884B1B6803F020030F
:10168000002B2DD0854B1B68DB0803F00303844A35
:1016900022FA03F3BB60BB6807EE903AF8EE676A84
:1016A0007B6907EE903AF8EE677A86EEA77A7B4B75
:1016B0009B6BC3F3080307EE903AF8EE676A97ED69
:1016C000036ADFED785AC6EE257A76EEA77AF7EE52
:1016D000006A77EEA67A67EE277AC7ED077A87E089
:1016E0007B6907EE903AF8EE677ADFED6F6A86EE77
:1016F000A77A6A4B9B6BC3F3080307EE903AF8EEA8
:10170000676A97ED036ADFED675AC6EE257A76EED3
:10171000A77AF7EE006A77EEA67A67EE277AC7ED2A
:10172000077A65E07B6907EE903AF8EE677ADFEDBD
:101730005F6A86EEA77A594B9B6BC3F3080307EEEB
:10174000903AF8EE676A97ED036ADFED565AC6EEF7
:10175000257A76EEA77AF7EE006A77EEA67A67EE3C
:10176000277AC7ED077A43E07B6907EE903AF8EEF7
:10177000677ADFED4F6A86EEA77A484B9B6BC3F31F
:10178000080307EE903AF8EE676A97ED036ADFED1B
:10179000455AC6EE257A76EEA77AF7EE006A77EE1E
:1017A000A67A67EE277AC7ED077A21E07B6907EE14
:1017B000903AF8EE677ADFED3D6A86EEA77A374B0E
:1017C0009B6BC3F3080307EE903AF8EE676A97ED58
:1017D000036ADFED345AC6EE257A76EEA77AF7EE85
:1017E000006A77EEA67A67EE277AC7ED077A00BF20
:1017F0002A4B9B6B5B0A03F07F0307EE903AF8EEEF
:10180000677AB7EE007A37EE877AD7ED076AC6EEC9
:10181000877AFCEEE77A17EE902A7B681A601F4BF6
:101820009B6B1B0C03F07F0307EE903AF8EE677A90
:10183000B7EE007A37EE877AD7ED076AC6EE877A79
:10184000FCEEE77A17EE902A7B685A60134B9B6B8D
:101850001B0E03F07F0307EE903AF8EE677AB7EEBF
:10186000007A37EE877AD7ED076AC6EE877AFCEE04
:10187000E77A17EE902A7B689A6008E07B6800227E
:101880001A607B6800225A607B6800229A6000BF61
:101890002437BD465DF8047B704700BF0044025802
:1018A0000090D003000000460024744C0024744AC9
:1018B00020BCBE4B80B489B000AF7860A14B9B6A5E
:1018C00003F00303BB619F4B9B6A1B0D03F03F03B7
:1018D0007B619C4BDB6A1B0A03F001033B61994B64
:1018E0005B6CDB08C3F30C033A6902FB03F307EEFE
:1018F000903AF8EE677AC7ED037A7B69002B00F027
:101900001181BB69022B00F08380BB69022B00F2BE
:10191000A180BB69002B03D0BB69012B56D099E095
:10192000884B1B6803F02003002B2DD0854B1B68D0
:10193000DB0803F00303844A22FA03F3BB60BB68AD
:1019400007EE903AF8EE676A7B6907EE903AF8EE98
:10195000677A86EEA77A7B4B1B6CC3F3080307EE0E
:10196000903AF8EE676A97ED036ADFED785AC6EEB3
:10197000257A76EEA77AF7EE006A77EEA67A67EE1A
:10198000277AC7ED077A87E07B6907EE903AF8EE91
:10199000677ADFED6F6A86EEA77A6A4B1B6CC3F33A
:1019A000080307EE903AF8EE676A97ED036ADFEDF9
:1019B000675AC6EE257A76EEA77AF7EE006A77EEDA
:1019C000A67A67EE277AC7ED077A65E07B6907EEAE
:1019D000903AF8EE677ADFED5F6A86EEA77A594BA8
:1019E0001B6CC3F3080307EE903AF8EE676A97EDB5
:1019F000036ADFED565AC6EE257A76EEA77AF7EE41
:101A0000006A77EEA67A67EE277AC7ED077A43E099
:101A10007B6907EE903AF8EE677ADFED4F6A86EE63
:101A2000A77A484B1B6CC3F3080307EE903AF8EE15
:101A3000676A97ED036ADFED455AC6EE257A76EEC2
:101A4000A77AF7EE006A77EEA67A67EE277AC7EDF7
:101A5000077A21E07B6907EE903AF8EE677ADFEDCE
:101A60003D6A86EEA77A374B1B6CC3F3080307EE7B
:101A7000903AF8EE676A97ED036ADFED345AC6EEE6
:101A8000257A76EEA77AF7EE006A77EEA67A67EE09
:101A9000277AC7ED077A00BF2A4B1B6C5B0A03F05D
:101AA0007F0307EE903AF8EE677AB7EE007A37EEEA
:101AB000877AD7ED076AC6EE877AFCEEE77A17EEEB
:101AC000902A7B681A601F4B1B6C1B0C03F07F0372
:101AD00007EE903AF8EE677AB7EE007A37EE877A3B
:101AE000D7ED076AC6EE877AFCEEE77A17EE902A02
:101AF0007B685A60134B1B6C1B0E03F07F0307EED1
:101B0000903AF8EE677AB7EE007A37EE877AD7ED3B
:101B1000076AC6EE877AFCEEE77A17EE902A7B68B2
:101B20009A6008E07B6800221A607B6800225A6095
:101B30007B6800229A6000BF2437BD465DF8047BB5
:101B4000704700BF004402580090D00300000046D8
:101B50000024744C0024744A20BCBE4B80B489B06D
:101B600000AF7860A04B9B6A03F00303BB619E4B00
:101B70009B6A1B0903F03F037B619B4BDB6A03F00D
:101B800001033B61984B5B6BDB08C3F30C033A69C1
:101B900002FB03F307EE903AF8EE677AC7ED037A9B
:101BA0007B69002B00F01181BB69022B00F0838060
:101BB000BB69022B00F2A180BB69002B03D0BB697B
:101BC000012B56D099E0884B1B6803F02003002BB3
:101BD0002DD0854B1B68DB0803F00303834A22FAF0
:101BE00003F3BB60BB6807EE903AF8EE676A7B6967
:101BF00007EE903AF8EE677A86EEA77A7A4B1B6B7F
:101C0000C3F3080307EE903AF8EE676A97ED036AAC
